** EXPERIMENTAL (HLL) ** Open Watcom Linker Version 2.0beta1 Limited Availability by SHL on Jul  2 2020
Portions Copyright (c) 1985-2002 Sybase, Inc. All Rights Reserved.
Created on:       21/06/16 19:55:27
Executable Image: stunnel.exe
creating an OS/2 EMX executable


                        +------------+
                        |   Groups   |
                        +------------+

Group                           Address              Size
=====                           =======              ====

CGROUP                          0001:00000000        002691b0
DGROUP                          0002:00000000        0000d840



                        +--------------+
                        |   Segments   |
                        +--------------+

Segment                Class          Group          Address         Size
=======                =====          =====          =======         ====

TEXT32                 CODE           CGROUP         0001:00000000   002691b0
________TEXT           CODE           CGROUP         0001:002691b0   00000000
DATA32                 DATA           DGROUP         0002:00000000   000047b0
SET1__os2dll           DATA           DGROUP         0002:000047b0   00000004
SET2__os2dll           DATA           DGROUP         0002:000047b4   00000000
SET3__os2dll           DATA           DGROUP         0002:000047b4   00000004
SET1___CTOR_LIST__     DATA           DGROUP         0002:000047b8   00000004
SET2___CTOR_LIST__     DATA           DGROUP         0002:000047bc   00000004
SET3___CTOR_LIST__     DATA           DGROUP         0002:000047c0   00000004
SET1___DTOR_LIST__     DATA           DGROUP         0002:000047c4   00000004
SET2___DTOR_LIST__     DATA           DGROUP         0002:000047c8   00000000
SET3___DTOR_LIST__     DATA           DGROUP         0002:000047c8   00000004
SET1___crtinit1__      DATA           DGROUP         0002:000047cc   00000004
SET2___crtinit1__      DATA           DGROUP         0002:000047d0   00000000
SET3___crtinit1__      DATA           DGROUP         0002:000047d0   00000004
SET1___crtexit1__      DATA           DGROUP         0002:000047d4   00000004
SET2___crtexit1__      DATA           DGROUP         0002:000047d8   00000000
SET3___crtexit1__      DATA           DGROUP         0002:000047d8   00000004
SET1___eh_frame__      DATA           DGROUP         0002:000047dc   00000004
SET2___eh_frame__      DATA           DGROUP         0002:000047e0   00000018
SET3___eh_frame__      DATA           DGROUP         0002:000047f8   00000004
SET1___eh_init__       DATA           DGROUP         0002:000047fc   00000004
SET2___eh_init__       DATA           DGROUP         0002:00004800   00000004
SET3___eh_init__       DATA           DGROUP         0002:00004804   00000004
SET1___eh_term__       DATA           DGROUP         0002:00004808   00000004
SET2___eh_term__       DATA           DGROUP         0002:0000480c   00000004
SET3___eh_term__       DATA           DGROUP         0002:00004810   00000004
SET1___fork_parent1__  DATA           DGROUP         0002:00004814   00000004
SET2___fork_parent1__  DATA           DGROUP         0002:00004818   00000000
SET3___fork_parent1__  DATA           DGROUP         0002:00004818   00000004
SET1___fork_child1__   DATA           DGROUP         0002:0000481c   00000004
SET2___fork_child1__   DATA           DGROUP         0002:00004820   00000000
SET3___fork_child1__   DATA           DGROUP         0002:00004820   00000004
________DATA           DATA           DGROUP         0002:00004830   00000000
BSS32                  BSS            DGROUP         0002:00004830   00008cc0
c_common               BSS            DGROUP         0002:0000d4f0   00000350
________BSS            BSS            DGROUP         0002:0000d840   00000000
STACK                  STACK          AUTO           0003:00000000   007d0000


                        +----------------+
                        |   Memory Map   |
                        +----------------+

* = unreferenced symbol
+ = symbol only referenced locally

Address        Symbol
=======        ======

Module: U:\usr\lib\crt0hi.obj({standard input})
0001:00000000* __text
0002:00000000* __data
0002:00000000* ___data_start
0002:00004830* ___bss_start
0002:000047b0+ __os2dll
0002:000047b8  ___CTOR_LIST__
0002:000047c4  ___DTOR_LIST__
0002:000047cc* ___crtinit1__
0002:000047d4* ___crtexit1__
0002:000047dc  ___eh_frame__
0002:000047fc  ___eh_init__
0002:00004808  ___eh_term__
0002:00004814+ ___fork_parent1__
0002:0000481c+ ___fork_child1__
Module: U:/tmp\ldconv_stunnel-tls_o_99560c9c37e164578.obj(tls.c)
0001:00000061  _tls_alloc
0001:00000193  _tls_init
0001:000001f6  _tls_cleanup
0001:0000025d* _tls_set
0001:00000279  _tls_get
0002:00004830  _tls_initialized
Module: U:/tmp\ldconv_stunnel-str_o_99560c9c37e169b68.obj(str.c)
0002:0000d4f0  _ui_tls
0001:00000500  _str_init
0001:0000051c  _str_canary_init
0001:00000618  _str_stats
0001:0000076e  _str_alloc_detached_debug
0001:00000834  _str_dup_detached_debug
0001:000008bd  _str_alloc_debug
0001:00000976  _str_dup_debug
0001:000009fa  _leak_table_utilization
0001:00000a4f  _safe_memcmp
0001:00000d4b  _str_realloc_debug
0001:00000d79  _str_vprintf
0001:00000dfa  _str_printf
0001:00000e14  _str_realloc_detached_debug
0001:00000e9b  _str_detach_debug
0001:00000f02  _str_free_debug
0001:00000fd0  _str_cleanup
Module: U:/tmp\ldconv_stunnel-file_o_99560c9c37e16c660.obj(file.c)
0001:00001017  _file_fdopen
0001:00001040  _file_open
0001:000010a3  _file_close
0001:000010e0  _file_getline
0001:00001164  _file_putline
0001:000011f3  _file_permissions
Module: U:/tmp\ldconv_stunnel-client_o_99560c9c37e175eb8.obj(client.c)
0001:0000133f  _alloc_client_session
0001:000013c7  _client_free
0001:0000140f  _throw_exception
0001:00006379  _client_main
0001:000064d9  _client_thread@4
Module: U:/tmp\ldconv_stunnel-log_o_99560c9c37e179d38.obj(log.c)
0001:000067b5  _log_close
0001:00006885  _s_log
0001:00006b14  _log_open
0001:00006beb  _log_flush
0001:00006cfe  _log_id
0001:00006f15  _fatal_debug
0001:00007019  _log_error
0001:00007053  _ioerror
0001:00007079  _sockerror
0001:0000709d  _s_strerror
0001:000070a2  _bin2hexstring
Module: U:/tmp\ldconv_stunnel-options_o_99560c9c37e17d3e8.obj(options.c)
0002:0000d500  _global_options
0002:0000d530  _service_options
0001:0000725c* _alphasort
0001:000085da* _scandir
0001:00008766  _options_defaults
0001:00008b4b  _options_apply
0001:00008bdb  _service_up_ref
0001:00008c2f  _service_free
0001:00011329  _options_free
0001:00011472  _options_parse
0001:000118f6  _options_cmdline
0002:00000200* _sock_opts_def
0002:000096f0  _number_of_sections
0002:000096f4* _configuration_file
Module: U:/tmp\ldconv_stunnel-protocol_o_99560c9c37e181e20.obj(protocol.c)
0001:00014234  _protocol
Module: U:/tmp\ldconv_stunnel-network_o_99560c9c37e185ca0.obj(network.c)
0001:00017131  _s_poll_alloc
0001:00017155  _s_poll_free
0001:00017164  _s_poll_add
0001:00017219  _s_poll_init
0001:0001728d  _s_poll_remove
0001:000172ee  _s_poll_canread
0001:00017322  _s_poll_canwrite
0001:00017356  _s_poll_hup
0001:0001738b  _s_poll_rdhup
0001:0001738d  _s_poll_err
0001:000173e4  _s_poll_dump
0001:0001743b  _s_poll_wait
0001:000174d6  _s_poll_sleep
0001:000175a4  _socket_options_set
0001:000176d3  _get_socket_error
0001:0001782a  _s_connect
0001:00017bf7  _s_write
0001:00017ddd  _s_read
0001:00017f38  _fd_putline
0001:00017fe0  _fd_getline
0001:00018116  _fd_printf
0001:000181a8  _s_ssl_write
0001:00018321  _s_ssl_read
0001:0001849d  _ssl_getstring
0001:00018588  _ssl_getline
0001:00018699  _ssl_putline
0001:0001873b  _ssl_printf
0001:00018866  _make_sockets
0001:00018adf  _original_dst
Module: U:/tmp\ldconv_stunnel-resolver_o_99560c9c37e188b80.obj(resolver.c)
0001:00018c40* _resolver_init
0001:00018cf4  _hostport2addrlist
0001:00018f71  _hostport2addr
0001:00019047  _name2addrlist
0001:00019162  _name2addr
0001:00019214  _addrlist_clear
0001:00019240  _addrlist_resolve
0001:000192c7  _addrlist_dup
0001:00019436  _s_ntop
0001:000195a6  _addr_len
0001:000195f6  _s_gai_strerror
Module: U:/tmp\ldconv_stunnel-ssl_o_99560c9c37e18b678.obj(ssl.c)
0002:0000d760  _index_ssl_cli
0002:0000d770  _index_ssl_ctx_opt
0002:0000d780  _index_session_authenticated
0002:0000d790  _index_session_connect_address
0001:00019c3c  _fips_available
0001:00019d38  _ssl_init
0001:0001a05e  _ssl_configure
Module: U:/tmp\ldconv_stunnel-ctx_o_99560c9c37e18e558.obj(ctx.c)
0001:0001c262  _psk_sort
0001:0001c311  _psk_find
0001:0001c4f0  _print_session_id
0001:0001c9b3  _sslerror
0001:0001ce50  _ui_stunnel
0001:0001d57e  _context_init
0002:00009d88* _current_section
0002:00009d84  _dh_params
0002:00009d80  _dh_temp_params
Module: U:/tmp\ldconv_stunnel-verify_o_99560c9c37e192ba8.obj(verify.c)
0001:0001f259  _X509_NAME2text
0001:0001fe38  _print_client_CA_list
0001:000200f2  _verify_init
Module: U:/tmp\ldconv_stunnel-sthreads_o_99560c9c37e1956a0.obj(sthreads.c)
0002:0000d7a0  _stunnel_locks
0001:0002043a  _stunnel_process_id
0001:0002043f  _stunnel_thread_id
0001:00020444* _thread_id_init
0001:00020445* _locking_init
0001:00020468  _sthreads_init
0001:000204e3  _create_client
0002:0000a1b0  _thread_head
Module: U:/tmp\ldconv_stunnel-fd_o_99560c9c37e198d50.obj(fd.c)
0001:0002061c  _get_limits
0001:0002070d  _set_nonblock
0001:00020819  _s_socket
0001:0002084f  _s_accept
0001:00020885* _s_socketpair
0001:00020901  _s_pipe
Module: U:/tmp\ldconv_stunnel-dhparam_o_99560c9c37e19bc30.obj(dhparam.c)
0001:00020980  _get_dh2048
Module: U:/tmp\ldconv_stunnel-cron_o_99560c9c37e19eb10.obj(cron.c)
0001:00020e0d  _cron_init
0002:0000a1d0  _cron_thread_id
Module: U:/tmp\ldconv_stunnel-stunnel_o_99560c9c37e1a1dd8.obj(stunnel.c)
0002:0000d7e0+ _fds
0002:0000d7f0+ _systemd_fds
0002:0000d800+ _listen_fds_start
0001:00022039  _main_configure
0001:00022177* _drop_privileges
0001:00022207  _main_cleanup
0001:000223f8* _pid_status_hang
0001:00022791  _daemon_loop
0001:0002300a  _signal_post
0001:000231a7  _stunnel_info
0001:00023473  _main_init
0002:000004e4  _num_clients
0002:000004e8  _terminate_pipe
0002:000004f0  _signal_pipe
0002:0000a1e0  _max_clients
Module: U:/tmp\ldconv_stunnel-pty_o_99560c9c37e1a4cb8.obj(pty.c)
0001:00023612  _pty_allocate
Module: U:/tmp\ldconv_stunnel-ui_unix_o_99560c9c37e1a9ec0.obj(ui_unix.c)
0001:00023792* _LoadExceptq
0001:00023949  _main
0001:00023b7a  _ui_config_reloaded
0001:00023b7b  _ui_new_chain
0001:00023b7c  _ui_clients
0001:00023b81  _ui_new_log
0001:00023ba5  _ui_passwd_cb
0001:00023baa  _ui_get_opener
0001:00023bbf  _ui_get_writer
0001:00023bd4  _ui_get_reader
0001:00023be9  _ui_get_closer
0001:00023949* main
Module: U:\usr\lib\libend.lib(src/libend/386/endlink386.asm)
0002:0000d840  _end
0002:00004830  _edata
Module: U:\usr\lib\libend.lib(src/libend/386/end.asm)
0001:002691b0* _etext
0001:002691b0* __etext
0000:00000000  WEAK$ZERO
0002:0000d840  __end
0002:00004830  __edata
Module: U:\tmp\ldconv_libcrypto_a_99560c9c37f156ab8.lib(mem.obj)
0001:00023c00  _CRYPTO_free
0001:00023c30  _CRYPTO_malloc
0001:00023c80  _CRYPTO_realloc
0001:00023d50  _CRYPTO_set_mem_functions
0001:00023d90* _CRYPTO_set_mem_debug
0001:00023da0  _CRYPTO_get_mem_functions
0001:00023de0  _CRYPTO_zalloc
0001:00023e70  _CRYPTO_clear_realloc
0001:00024050  _CRYPTO_clear_free
Module: U:\tmp\ldconv_libcrypto_a_99560c9c37f156ab8.lib(threads_pthread.obj)
0001:00024110  _CRYPTO_THREAD_lock_new
0001:00024180  _CRYPTO_THREAD_read_lock
0001:000241a0  _CRYPTO_THREAD_write_lock
0001:000241c0  _CRYPTO_THREAD_unlock
0001:000241e0  _CRYPTO_THREAD_lock_free
0001:00024220  _CRYPTO_THREAD_run_once
0001:00024250  _CRYPTO_THREAD_init_local
0001:00024280  _CRYPTO_THREAD_get_local
0001:00024290  _CRYPTO_THREAD_set_local
0001:000242c0  _CRYPTO_THREAD_cleanup_local
0001:000242e0  _CRYPTO_THREAD_get_current_id
0001:000242f0  _CRYPTO_THREAD_compare_id
0001:00024300  _CRYPTO_atomic_add
0001:00024320  _openssl_init_fork_handlers
0001:00024350  _openssl_get_fork_id
Module: U:\tmp\ldconv_libcrypto_a_99560c9c37f156ab8.lib(rand_lib.obj)
0001:000245e0  _rand_drbg_cleanup_entropy
0001:00024660  _rand_drbg_cleanup_nonce
0001:00024690  _rand_drbg_get_additional_data
0001:000246d0  _rand_drbg_cleanup_additional_data
0001:00024700  _rand_cleanup_int
0001:000247f0* _RAND_keep_random_devices_open
0001:00024830  _rand_pool_new
0001:000249a0  _rand_drbg_get_entropy
0001:00024da0  _rand_pool_attach
0001:00024e30  _rand_pool_free
0001:00024eb0* _rand_pool_buffer
0001:00024ec0* _rand_pool_entropy
0001:00024ed0* _rand_pool_length
0001:00024ee0* _rand_pool_detach
0001:00024f00* _rand_pool_reattach
0001:00024f30  _rand_pool_entropy_available
0001:00024f60* _rand_pool_entropy_needed
0001:00024f80  _rand_pool_bytes_needed
0001:00025210* _rand_pool_bytes_remaining
0001:00025220  _rand_pool_add
0001:00025330  _rand_drbg_get_nonce
0001:00025580* _rand_pool_add_begin
0001:000257c0* _rand_pool_add_end
0001:00025830  _RAND_set_rand_method
0001:000258b0  _RAND_get_rand_method
0001:00025950* _RAND_poll
0001:00025ad0* _RAND_set_rand_engine
0001:00025bd0* _RAND_seed
0001:00025ca0  _RAND_add
0001:00025d80  _RAND_priv_bytes
0001:00025ec0  _RAND_bytes
0001:00025fc0* _RAND_pseudo_bytes
0001:000260c0  _RAND_status
Module: U:\tmp\ldconv_libssl_a_99560c9c37e1aece0.lib(ssl_sess.obj)
0001:00026490  _SSL_get_session
0001:000264a0  _SSL_get1_session
0001:000264e0  _SSL_SESSION_set_ex_data
0001:000264f0  _SSL_SESSION_get_ex_data
0001:00026500  _SSL_SESSION_new
0001:00026670  _ssl_session_dup
0001:00026a30* _SSL_SESSION_dup
0001:00026a50  _SSL_SESSION_get_id
0001:00026a70* _SSL_SESSION_get0_id_context
0001:00026a90* _SSL_SESSION_get_compress_id
0001:00026aa0  _ssl_generate_session_id
0001:00026cd0  _ssl_get_new_session
0001:00026ef0  _SSL_CTX_add_session
0001:00027300  _lookup_sess_in_cache
0001:00027470  _SSL_CTX_remove_session
0001:00027610  _SSL_SESSION_free
0001:00027640  _ssl_get_prev_session
0001:00027be0  _SSL_SESSION_up_ref
0001:00027c00  _SSL_set_session
0001:00027e70* _SSL_SESSION_set1_id
0001:00027ef0* _SSL_SESSION_set_timeout
0001:00027f20  _SSL_SESSION_get_timeout
0001:00027f40  _SSL_SESSION_get_time
0001:00027f60* _SSL_SESSION_set_time
0001:00027f80* _SSL_SESSION_get_protocol_version
0001:00027f90  _SSL_SESSION_set_protocol_version
0001:00027fa0  _SSL_SESSION_get0_cipher
0001:00027fb0  _SSL_SESSION_set_cipher
0001:00027fd0* _SSL_SESSION_get0_hostname
0001:00027fe0* _SSL_SESSION_set1_hostname
0001:00028060* _SSL_SESSION_has_ticket
0001:00028080* _SSL_SESSION_get_ticket_lifetime_hint
0001:00028090* _SSL_SESSION_get0_ticket
0001:000280c0* _SSL_SESSION_get_max_early_data
0001:000280d0* _SSL_SESSION_set_max_early_data
0001:000280f0* _SSL_SESSION_get0_alpn_selected
0001:00028110* _SSL_SESSION_set1_alpn_selected
0001:000281b0* _SSL_SESSION_get0_peer
0001:000281c0* _SSL_SESSION_set1_id_context
0001:00028240  _SSL_SESSION_is_resumable
0001:00028270  _SSL_CTX_set_timeout
0001:00028290* _SSL_CTX_get_timeout
0001:000282b0* _SSL_set_session_secret_cb
0001:000282e0* _SSL_set_session_ticket_ext_cb
0001:00028310* _SSL_set_session_ticket_ext
0001:00028420  _SSL_CTX_flush_sessions
0001:000284b0  _ssl_clear_bad_session
0001:00028660  _SSL_CTX_sess_set_new_cb
0001:00028670* _SSL_CTX_sess_get_new_cb
0001:00028680  _SSL_CTX_sess_set_remove_cb
0001:00028690* _SSL_CTX_sess_get_remove_cb
0001:000286a0  _SSL_CTX_sess_set_get_cb
0001:000286b0* _SSL_CTX_sess_get_get_cb
0001:000286c0  _SSL_CTX_set_info_callback
0001:000286d0* _SSL_CTX_get_info_callback
0001:000286e0* _SSL_CTX_set_client_cert_cb
0001:000286f0* _SSL_CTX_get_client_cert_cb
0001:00028700  _SSL_CTX_set_client_cert_engine
0001:000287c0* _SSL_CTX_set_cookie_generate_cb
0001:000287d0* _SSL_CTX_set_cookie_verify_cb
0001:000287e0  _SSL_SESSION_set1_ticket_appdata
0001:00028880  _SSL_SESSION_get0_ticket_appdata
0001:000288b0* _SSL_CTX_set_stateless_cookie_generate_cb
0001:000288c0* _SSL_CTX_set_stateless_cookie_verify_cb
0001:000288f0* _PEM_read_bio_SSL_SESSION
0001:00028930* _PEM_read_SSL_SESSION
0001:00028970* _PEM_write_bio_SSL_SESSION
0001:000289d0* _PEM_write_SSL_SESSION
Module: U:\usr\lib\libc_dll.lib(setsockopt.obj)
0001:00028a30  _setsockopt
Module: U:\usr\lib\libc_dll.lib(sock_errno.obj)
0001:00028b60  _sock_errno
Module: U:\tmp\ldconv_ssp_a_99560c9c38216f540.lib(ssp.obj)
0001:00028d3a  ___stack_chk_fail
0001:00028d9f* ___chk_fail
0001:00028db9* ___stack_chk_fail_local
0002:0000a290  ___stack_chk_guard
Module: U:\tmp\ldconv_libssl_a_99560c9c37e1aece0.lib(ssl_lib.obj)
0001:00028e90  _ssl_undefined_function
0001:00029d20  _SSL_clear
0001:0002a0a0* _SSL_CTX_set_ssl_version
0001:0002a190* _SSL_is_dtls
0001:0002a1b0* _SSL_up_ref
0001:0002a1d0  _SSL_CTX_set_session_id_context
0001:0002a250* _SSL_set_session_id_context
0001:0002a2d0* _SSL_CTX_set_generate_session_id
0001:0002a310* _SSL_set_generate_session_id
0001:0002a350  _SSL_has_matching_session_id
0001:0002a3f0* _SSL_CTX_set_purpose
0001:0002a410* _SSL_set_purpose
0001:0002a430* _SSL_CTX_set_trust
0001:0002a450* _SSL_set_trust
0001:0002a470* _SSL_set1_host
0001:0002a4a0* _SSL_add1_host
0001:0002a4d0* _SSL_set_hostflags
0001:0002a4f0* _SSL_get0_peername
0001:0002a510* _SSL_CTX_dane_enable
0001:0002a640* _SSL_CTX_dane_set_flags
0001:0002a660* _SSL_CTX_dane_clear_flags
0001:0002a680* _SSL_dane_set_flags
0001:0002a6a0* _SSL_dane_clear_flags
0001:0002a6c0* _SSL_get0_dane_authority
0001:0002a740* _SSL_get0_dane_tlsa
0001:0002a7f0* _SSL_get0_dane
0001:0002a800* _SSL_dane_tlsa_add
0001:0002af50* _SSL_CTX_dane_mtype_set
0001:0002b1d0* _SSL_CTX_set1_param
0001:0002b1f0* _SSL_set1_param
0001:0002b210* _SSL_CTX_get0_param
0001:0002b220* _SSL_get0_param
0001:0002b230* _SSL_certs_clear
0001:0002b250  _SSL_free
0001:0002b280* _SSL_set0_rbio
0001:0002b2a0* _SSL_set0_wbio
0001:0002b2f0* _SSL_set_bio
0001:0002b430  _SSL_get_rbio
0001:0002b440  _SSL_get_wbio
0001:0002b460* _SSL_get_fd
0001:0002b4b0* _SSL_get_rfd
0001:0002b500* _SSL_get_wfd
0001:0002b570  _SSL_set_fd
0001:0002b600  _SSL_set_wfd
0001:0002b720  _SSL_set_rfd
0001:0002b820* _SSL_get_finished
0001:0002b870* _SSL_get_peer_finished
0001:0002b8c0* _SSL_get_verify_mode
0001:0002b8d0* _SSL_get_verify_depth
0001:0002b8f0* _SSL_get_verify_callback
0001:0002b900  _SSL_CTX_get_verify_mode
0001:0002b910* _SSL_CTX_get_verify_depth
0001:0002b930  _SSL_CTX_get_verify_callback
0001:0002b940  _SSL_set_verify
0001:0002b960* _SSL_set_verify_depth
0001:0002b980* _SSL_set_read_ahead
0001:0002b990* _SSL_get_read_ahead
0001:0002b9a0  _SSL_pending
0001:0002b9d0  _SSL_has_pending
0001:0002ba10  _SSL_get_peer_certificate
0001:0002ba50  _SSL_get_peer_cert_chain
0001:0002ba80* _SSL_copy_session_id
0001:0002bb70  _SSL_CTX_check_private_key
0001:0002bc10* _SSL_check_private_key
0001:0002bcf0* _SSL_waiting_for_async
0001:0002bd10* _SSL_get_all_async_fds
0001:0002bd40* _SSL_get_changed_async_fds
0001:0002bd70  _SSL_get_default_timeout
0001:0002bd80* _ssl_read_internal
0001:0002bed0  _SSL_read
0001:0002c060* _SSL_read_ex
0001:0002c1c0* _SSL_get_early_data_status
0001:0002c1d0* _SSL_peek
0001:0002c2f0* _SSL_peek_ex
0001:0002c3e0* _ssl_write_internal
0001:0002c560  _SSL_write
0001:0002c720* _SSL_write_ex
0001:0002c8b0  _SSL_shutdown
0001:0002c990* _SSL_key_update
0001:0002caa0* _SSL_get_key_update_type
0001:0002cab0  _SSL_renegotiate
0001:0002cb70  _SSL_renegotiate_abbreviated
0001:0002cc30* _SSL_renegotiate_pending
0001:0002cc50  _SSL_ctrl
0001:0002d090* _SSL_dane_enable
0001:0002d250  _SSL_new
0001:0002d900* _SSL_callback_ctrl
0001:0002d930* _SSL_CTX_sessions
0001:0002d940  _SSL_CTX_ctrl
0001:0002dde0  _SSL_CTX_callback_ctrl
0001:0002de10* _ssl_cipher_id_cmp
0001:0002de30  _ssl_cipher_ptr_id_cmp
0001:0002de50  _SSL_get_ciphers
0001:0002de90* _SSL_get_client_ciphers
0001:0002dec0  _SSL_get1_supported_ciphers
0001:0002dfa0  _ssl_get_ciphers_by_id
0001:0002dfe0* _SSL_get_cipher_list
0001:0002e040  _SSL_CTX_get_ciphers
0001:0002e050  _SSL_CTX_set_cipher_list
0001:0002e120  _SSL_set_cipher_list
0001:0002e200* _SSL_get_shared_ciphers
0001:0002e340  _SSL_get_servername
0001:0002e450* _SSL_get_servername_type
0001:0002e540* _SSL_select_next_proto
0001:0002e620* _SSL_get0_next_proto_negotiated
0001:0002e650* _SSL_CTX_set_next_protos_advertised_cb
0001:0002e670* _SSL_CTX_set_next_proto_select_cb
0001:0002e690* _SSL_CTX_set_alpn_protos
0001:0002e740* _SSL_set_alpn_protos
0001:0002e7f0* _SSL_CTX_set_alpn_select_cb
0001:0002e810* _SSL_get0_alpn_selected
0001:0002e850* _SSL_export_keying_material
0001:0002e8f0* _SSL_export_keying_material_early
0001:0002e920  _SSL_CTX_new
0001:0002eea0* _SSL_CTX_up_ref
0001:0002eec0  _SSL_CTX_free
0001:0002eef0  _SSL_CTX_set_default_passwd_cb
0001:0002ef00* _SSL_CTX_set_default_passwd_cb_userdata
0001:0002ef10* _SSL_CTX_get_default_passwd_cb
0001:0002ef20* _SSL_CTX_get_default_passwd_cb_userdata
0001:0002ef30* _SSL_set_default_passwd_cb
0001:0002ef40* _SSL_set_default_passwd_cb_userdata
0001:0002ef50* _SSL_get_default_passwd_cb
0001:0002ef60* _SSL_get_default_passwd_cb_userdata
0001:0002ef70* _SSL_CTX_set_cert_verify_callback
0001:0002ef90  _SSL_CTX_set_verify
0001:0002efb0* _SSL_CTX_set_verify_depth
0001:0002efd0* _SSL_CTX_set_cert_cb
0001:0002eff0* _SSL_set_cert_cb
0001:0002f010  _ssl_set_masks
0001:0002f2c0  _ssl_check_srvr_ecc_cert_and_alg
0001:0002f320  _ssl_get_server_cert_serverinfo
0001:0002f360  _ssl_update_cache
0001:0002f550* _SSL_CTX_get_ssl_method
0001:0002f560* _SSL_get_ssl_method
0001:0002f570  _SSL_set_ssl_method
0001:0002f5e0  _SSL_get_error
0001:0002f7c0* _SSL_do_handshake
0001:0002f890  _SSL_accept
0001:0002f980  _SSL_connect
0001:0002fa70* _SSL_write_early_data
0001:0002fe40* _SSL_read_early_data
0001:00030080  _SSL_set_accept_state
0001:00030150  _SSL_set_connect_state
0001:00030220  _ssl_undefined_void_function
0001:00030260* _ssl_undefined_const_function
0001:00030270* _ssl_bad_method
0001:000302f0  _ssl_protocol_to_string
0001:00030390  _SSL_get_version
0001:00030430* _SSL_dup
0001:000311b0* _ssl_clear_cipher_ctx
0001:00031230* _SSL_get_certificate
0001:00031250* _SSL_get_privatekey
0001:00031270* _SSL_CTX_get0_certificate
0001:00031290* _SSL_CTX_get0_privatekey
0001:000312b0  _SSL_get_current_cipher
0001:000312d0* _SSL_get_pending_cipher
0001:000312e0  _SSL_get_current_compression
0001:00031310  _SSL_get_current_expansion
0001:00031340  _ssl_init_wbio_buffer
0001:00031400  _ssl_free_wbio_buffer
0001:00031440* _SSL_CTX_set_quiet_shutdown
0001:00031450* _SSL_CTX_get_quiet_shutdown
0001:00031460* _SSL_set_quiet_shutdown
0001:00031470* _SSL_get_quiet_shutdown
0001:00031480  _SSL_set_shutdown
0001:00031490  _SSL_get_shutdown
0001:000314a0  _SSL_version
0001:000314b0  _SSL_client_version
0001:000314c0  _SSL_get_SSL_CTX
0001:000314d0  _SSL_set_SSL_CTX
0001:00031670* _SSL_CTX_set_default_verify_paths
0001:00031680* _SSL_CTX_set_default_verify_dir
0001:000316e0* _SSL_CTX_set_default_verify_file
0001:00031740  _SSL_CTX_load_verify_locations
0001:00031750* _SSL_set_info_callback
0001:00031760* _SSL_get_info_callback
0001:00031770* _SSL_set_verify_result
0001:00031780* _SSL_get_verify_result
0001:00031790* _SSL_get_client_random
0001:00031820* _SSL_get_server_random
0001:000318b0* _SSL_SESSION_get_master_key
0001:000318f0  _SSL_SESSION_set1_master_key
0001:00031930  _SSL_set_ex_data
0001:00031940  _SSL_get_ex_data
0001:00031950  _SSL_CTX_set_ex_data
0001:00031960  _SSL_CTX_get_ex_data
0001:00031970  _SSL_CTX_get_cert_store
0001:00031980* _SSL_CTX_set_cert_store
0001:000319a0* _SSL_CTX_set1_cert_store
0001:000319d0* _SSL_want
0001:000319e0* _SSL_CTX_set_tmp_dh_callback
0001:00031a10* _SSL_set_tmp_dh_callback
0001:00031a40* _SSL_CTX_use_psk_identity_hint
0001:00031b50* _SSL_use_psk_identity_hint
0001:00031c70* _SSL_get_psk_identity_hint
0001:00031ca0* _SSL_get_psk_identity
0001:00031cd0* _SSL_set_psk_client_callback
0001:00031ce0  _SSL_CTX_set_psk_client_callback
0001:00031cf0* _SSL_set_psk_server_callback
0001:00031d00  _SSL_CTX_set_psk_server_callback
0001:00031d10* _SSL_set_psk_find_session_callback
0001:00031d20* _SSL_CTX_set_psk_find_session_callback
0001:00031d30* _SSL_set_psk_use_session_callback
0001:00031d40* _SSL_CTX_set_psk_use_session_callback
0001:00031d50* _SSL_CTX_set_msg_callback
0001:00031d60* _SSL_set_msg_callback
0001:00031d70* _SSL_CTX_set_not_resumable_session_callback
0001:00031da0* _SSL_set_not_resumable_session_callback
0001:00031dd0* _SSL_CTX_set_record_padding_callback
0001:00031de0* _SSL_CTX_set_record_padding_callback_arg
0001:00031df0* _SSL_CTX_get_record_padding_callback_arg
0001:00031e00  _SSL_CTX_set_block_padding
0001:00031e40* _SSL_set_record_padding_callback
0001:00031e50* _SSL_set_record_padding_callback_arg
0001:00031e60* _SSL_get_record_padding_callback_arg
0001:00031e70  _SSL_set_block_padding
0001:00031eb0  _SSL_set_num_tickets
0001:00031ed0* _SSL_get_num_tickets
0001:00031ee0  _SSL_CTX_set_num_tickets
0001:00031f00* _SSL_CTX_get_num_tickets
0001:00031f10  _ssl_replace_hash
0001:00031f80* _ssl_clear_hash_ctx
0001:00031fa0  _ssl_handshake_hash
0001:000320b0  _SSL_session_reused
0001:000320c0* _SSL_is_server
0001:000320d0* _SSL_set_debug
0001:000320e0* _SSL_set_security_level
0001:00032100  _SSL_get_security_level
0001:00032120* _SSL_set_security_callback
0001:00032140* _SSL_get_security_callback
0001:00032160* _SSL_set0_security_ex_data
0001:00032180* _SSL_get0_security_ex_data
0001:000321a0  _SSL_CTX_set_security_level
0001:000321c0  _SSL_CTX_get_security_level
0001:000321e0* _SSL_CTX_set_security_callback
0001:00032200* _SSL_CTX_get_security_callback
0001:00032220* _SSL_CTX_set0_security_ex_data
0001:00032240* _SSL_CTX_get0_security_ex_data
0001:00032260  _SSL_CTX_get_options
0001:00032270  _SSL_get_options
0001:00032280  _SSL_CTX_set_options
0001:000322a0  _SSL_set_options
0001:000322c0  _SSL_CTX_clear_options
0001:000322e0* _SSL_clear_options
0001:00032300* _SSL_get0_verified_chain
0001:00032310  _OBJ_bsearch_ssl_cipher_id
0001:00032350* _SSL_get0_peer_scts
0001:00032560* _SSL_set_ct_validation_callback
0001:00032610* _SSL_CTX_set_ct_validation_callback
0001:00032690* _SSL_ct_is_enabled
0001:000326b0  _SSL_CTX_ct_is_enabled
0001:000326d0  _ssl_validate_ct
0001:000328f0* _SSL_CTX_enable_ct
0001:000329f0* _SSL_enable_ct
0001:00032b50* _SSL_CTX_set_default_ctlog_list_file
0001:00032b70* _SSL_CTX_set_ctlog_list_file
0001:00032b90* _SSL_CTX_set0_ctlog_store
0001:00032bc0* _SSL_CTX_get0_ctlog_store
0001:00032bd0* _SSL_CTX_set_client_hello_cb
0001:00032bf0* _SSL_client_hello_isv2
0001:00032c10* _SSL_client_hello_get0_legacy_version
0001:00032c30* _SSL_client_hello_get0_random
0001:00032c60* _SSL_client_hello_get0_session_id
0001:00032c90* _SSL_client_hello_get0_ciphers
0001:00032cc0* _SSL_client_hello_get0_compression_methods
0001:00032cf0* _SSL_client_hello_get1_extensions_present
0001:00032e70* _SSL_client_hello_get0_ext
0001:00032ef0* _SSL_free_buffers
0001:00032f40* _SSL_alloc_buffers
0001:00032f50* _SSL_CTX_set_keylog_callback
0001:00032f60* _SSL_CTX_get_keylog_callback
0001:00032f70  _ssl_log_rsa_client_key_exchange
0001:00033120  _ssl_log_secret
0001:000332e0  _ssl_cache_cipherlist
0001:000335e0* _SSL_bytes_to_cipher_list
0001:000338f0  _bytes_to_cipher_list
0001:00033d70* _SSL_CTX_set_max_early_data
0001:00033d90* _SSL_CTX_get_max_early_data
0001:00033da0* _SSL_set_max_early_data
0001:00033dc0* _SSL_get_max_early_data
0001:00033dd0* _SSL_CTX_set_recv_max_early_data
0001:00033df0* _SSL_CTX_get_recv_max_early_data
0001:00033e00* _SSL_set_recv_max_early_data
0001:00033e20* _SSL_get_recv_max_early_data
0001:00033e30  _ssl_get_max_send_fragment
0001:00033e70  _ssl_get_split_send_fragment
0001:00033ec0* _SSL_stateless
0001:00034000* _SSL_CTX_set_post_handshake_auth
0001:00034010* _SSL_set_post_handshake_auth
0001:00034020* _SSL_verify_client_post_handshake
0001:000342b0  _SSL_CTX_set_session_ticket_cb
0001:000342e0* _SSL_CTX_set_allow_early_data_cb
0001:00034300* _SSL_set_allow_early_data_cb
0001:0003431c* _SSL_version_str
0002:00000530* _ssl3_undef_enc_method
Module: U:\tmp\ldconv_libcrypto_a_99560c9c37f156ab8.lib(x509_cmp.obj)
0001:00034420* _X509_issuer_and_serial_cmp
0001:000344f0* _X509_issuer_and_serial_hash
0001:000345d0* _X509_issuer_name_cmp
0001:00034670  _X509_subject_name_cmp
0001:00034710  _X509_CRL_cmp
0001:000347b0  _X509_CRL_match
0001:000347e0  _X509_get_issuer_name
0001:000347f0* _X509_issuer_name_hash
0001:00034850* _X509_issuer_name_hash_old
0001:00034900  _X509_get_subject_name
0001:00034910  _X509_get_serialNumber
0001:00034920  _X509_get0_serialNumber
0001:00034930* _X509_subject_name_hash
0001:00034990* _X509_subject_name_hash_old
0001:00034a40  _X509_cmp
0001:00034b10  _X509_NAME_cmp
0001:00034ba0  _X509_NAME_hash
0001:00034c00* _X509_NAME_hash_old
0001:00034cb0  _X509_find_by_issuer_and_serial
0001:00034d60  _X509_find_by_subject
0001:00034e20  _X509_get0_pubkey
0001:00034e40  _X509_get_pubkey
0001:00034e60  _X509_check_private_key
0001:00034f60  _X509_chain_check_suiteb
0001:00035250  _X509_CRL_check_suiteb
0001:00035330  _X509_chain_up_ref
Module: U:\tmp\ldconv_libcrypto_a_99560c9c37f156ab8.lib(x_x509.obj)
0001:00035610* _d2i_X509_CINF
0001:00035bc0  _X509_CINF_it
0001:00035640* _i2d_X509_CINF
0001:00035670* _X509_CINF_new
0001:00035690* _X509_CINF_free
0001:000356b0  _d2i_X509
0001:00035b18  _X509_it
0001:000356e0  _i2d_X509
0001:00035710* _X509_new
0001:00035730  _X509_free
0001:00035750  _X509_dup
0001:00035770* _X509_set_ex_data
0001:00035780* _X509_get_ex_data
0001:00035790  _d2i_X509_AUX
0001:00035880  _i2d_X509_AUX
0001:00035aa0  _i2d_re_X509_tbs
0001:00035ad0  _X509_get0_signature
0001:00035b00  _X509_get_signature_nid
Module: U:\tmp\ldconv_libssl_a_99560c9c37e1aece0.lib(ssl_ciph.obj)
0001:00037340  _ssl_load_ciphers
0001:000377e0  _ssl_cipher_get_evp
0001:00037b40  _ssl_md
0001:00037b60  _ssl_handshake_md
0001:00037b90  _ssl_prf_md
0001:00037bc0  _SSL_CTX_set_ciphersuites
0001:00037c70  _SSL_set_ciphersuites
0001:00037e40  _ssl_create_cipher_list
0001:000389a0  _SSL_CIPHER_description
0001:000390a0* _SSL_CIPHER_get_version
0001:000390e0  _SSL_CIPHER_get_name
0001:00039100* _SSL_CIPHER_standard_name
0001:00039120* _OPENSSL_cipher_name
0001:00039150  _SSL_CIPHER_get_bits
0001:00039170  _SSL_CIPHER_get_id
0001:00039180* _SSL_CIPHER_get_protocol_id
0001:00039190  _ssl3_comp_find
0001:000391f0  _SSL_COMP_get_compression_methods
0001:00039210* _SSL_COMP_set0_compression_methods
0001:00039220  _ssl_comp_free_compression_methods_int
0001:00039250  _SSL_COMP_add_compression_method
0001:00039440  _SSL_COMP_get_name
0001:00039460  _SSL_COMP_get0_name
0001:00039470  _SSL_COMP_get_id
0001:00039480  _ssl_get_cipher_by_char
0001:000394b0  _SSL_CIPHER_find
0001:000394d0  _SSL_CIPHER_get_cipher_nid
0001:00039500* _SSL_CIPHER_get_digest_nid
0001:00039590* _SSL_CIPHER_get_kx_nid
0001:00039620* _SSL_CIPHER_get_auth_nid
0001:000396a0* _SSL_CIPHER_get_handshake_digest
0001:000396c0* _SSL_CIPHER_is_aead
0001:000396d0  _ssl_cipher_get_overhead
0001:000398a0  _ssl_cert_is_disabled
Module: U:\tmp\ldconv_libcrypto_a_99560c9c37f156ab8.lib(p_lib.obj)
0001:0003af80  _EVP_PKEY_bits
0001:0003afb0  _EVP_PKEY_security_bits
0001:0003afe0  _EVP_PKEY_size
0001:0003b010* _EVP_PKEY_save_parameters
0001:0003b060  _EVP_PKEY_copy_parameters
0001:0003b2f0  _EVP_PKEY_missing_parameters
0001:0003b320  _EVP_PKEY_cmp_parameters
0001:0003b360  _EVP_PKEY_cmp
0001:0003b3d0  _EVP_PKEY_new
0001:0003b4b0  _EVP_PKEY_up_ref
0001:0003b4d0* _EVP_PKEY_get_raw_private_key
0001:0003b580* _EVP_PKEY_get_raw_public_key
0001:0003b630  _EVP_PKEY_set_type
0001:0003b750  _EVP_PKEY_set_type_str
0001:0003b890* _EVP_PKEY_set_alias_type
0001:0003b980* _EVP_PKEY_set1_engine
0001:0003ba50* _EVP_PKEY_get0_engine
0001:0003ba60  _EVP_PKEY_assign
0001:0003bb80  _EVP_PKEY_get0
0001:0003bb90* _EVP_PKEY_get0_hmac
0001:0003bbf0  _EVP_PKEY_get0_poly1305
0001:0003bc50  _EVP_PKEY_get0_siphash
0001:0003bcb0  _EVP_PKEY_set1_RSA
0001:0003bdd0  _EVP_PKEY_get0_RSA
0001:0003be20  _EVP_PKEY_get1_RSA
0001:0003be80  _EVP_PKEY_set1_DSA
0001:0003bfa0* _EVP_PKEY_get0_DSA
0001:0003bff0  _EVP_PKEY_get1_DSA
0001:0003c050  _EVP_PKEY_set1_EC_KEY
0001:0003c170  _EVP_PKEY_get0_EC_KEY
0001:0003c1d0  _EVP_PKEY_get1_EC_KEY
0001:0003c240  _EVP_PKEY_set1_DH
0001:0003c370  _EVP_PKEY_get0_DH
0001:0003c3c0* _EVP_PKEY_get1_DH
0001:0003c420  _EVP_PKEY_type
0001:0003c460  _EVP_PKEY_id
0001:0003c470  _EVP_PKEY_base_id
0001:0003c4b0  _EVP_PKEY_free
0001:0003c560  _EVP_PKEY_new_raw_private_key
0001:0003c710* _EVP_PKEY_new_raw_public_key
0001:0003c8c0* _EVP_PKEY_new_CMAC_key
0001:0003caa0  _EVP_PKEY_print_public
0001:0003cb30* _EVP_PKEY_print_private
0001:0003cbb0* _EVP_PKEY_print_params
0001:0003cc30  _EVP_PKEY_get_default_digest_nid
0001:0003cc70  _EVP_PKEY_set1_tls_encodedpoint
0001:0003ccc0  _EVP_PKEY_get1_tls_encodedpoint
Module: U:\tmp\ldconv_libcrypto_a_99560c9c37f156ab8.lib(obj_dat.obj)
0001:0003cf30  _obj_cleanup_int
0001:0003cfc0* _OBJ_new_nid
0001:0003cfe0* _OBJ_add_object
0001:0003d1e0  _OBJ_nid2obj
0001:0003d2c0  _OBJ_nid2sn
0001:0003d3a0  _OBJ_nid2ln
0001:0003d480  _OBJ_obj2nid
0001:0003d590  _OBJ_obj2txt
0001:0003da20  _OBJ_ln2nid
0001:0003dae0  _OBJ_sn2nid
0001:0003dba0  _OBJ_txt2obj
0001:0003dde0  _OBJ_txt2nid
0001:0003e020  _OBJ_bsearch_
0001:0003e080  _OBJ_bsearch_ex_
0001:0003e160  _OBJ_create
0001:0003e280* _OBJ_create_objects
0001:0003e410  _OBJ_length
0001:0003e430  _OBJ_get0_data
Module: U:\tmp\ldconv_libcrypto_a_99560c9c37f156ab8.lib(ec_key.obj)
0001:00051550  _EC_KEY_new
0001:00051580  _EC_KEY_free
0001:00051650  _EC_KEY_new_by_curve_name
0001:000516b0* _EC_KEY_copy
0001:000518b0  _EC_KEY_dup
0001:00051900  _EC_KEY_up_ref
0001:00051920* _EC_KEY_get0_engine
0001:00051930  _EC_KEY_generate_key
0001:000519c0  _ossl_ec_key_gen
0001:000519d0  _ec_key_simple_generate_key
0001:00051af0  _ec_key_simple_generate_public_key
0001:00051b30  _EC_KEY_check_key
0001:00051bd0  _ec_key_simple_check_key
0001:00051f20* _EC_KEY_set_public_key_affine_coordinates
0001:00052140  _EC_KEY_get0_group
0001:00052150  _EC_KEY_set_group
0001:000521a0  _EC_KEY_get0_private_key
0001:000521b0* _EC_KEY_set_private_key
0001:000522a0  _EC_KEY_get0_public_key
0001:000522b0* _EC_KEY_set_public_key
0001:00052300  _EC_KEY_get_enc_flags
0001:00052310  _EC_KEY_set_enc_flags
0001:00052320  _EC_KEY_get_conv_form
0001:00052330* _EC_KEY_set_conv_form
0001:00052360* _EC_KEY_set_asn1_flag
0001:00052380* _EC_KEY_precompute_mult
0001:000523a0  _EC_KEY_get_flags
0001:000523b0  _EC_KEY_set_flags
0001:000523c0  _EC_KEY_clear_flags
0001:000523d0  _EC_KEY_decoded_from_explicit_params
0001:000523f0  _EC_KEY_key2buf
0001:00052440  _EC_KEY_oct2key
0001:000524d0* _EC_KEY_priv2oct
0001:00052530  _ec_key_simple_priv2oct
0001:000525c0  _EC_KEY_oct2priv
0001:00052620  _ec_key_simple_oct2priv
0001:000526e0  _EC_KEY_priv2buf
0001:00052860  _EC_KEY_can_sign
Module: U:\tmp\ldconv_libcrypto_a_99560c9c37f156ab8.lib(ec_lib.obj)
0001:000528b0  _EC_GROUP_new
0001:00052a30  _EC_pre_comp_free
0001:00052a80  _EC_GROUP_free
0001:00052b70  _EC_GROUP_clear_free
0001:00052ca0  _EC_GROUP_method_of
0001:00052cb0  _EC_METHOD_get_field_type
0001:00052cc0  _EC_GROUP_get0_generator
0001:00052cd0* _EC_GROUP_get_mont_data
0001:00052ce0  _EC_GROUP_get_order
0001:00052d30  _EC_GROUP_get0_order
0001:00052d40  _EC_GROUP_order_bits
0001:00052d50  _EC_GROUP_get_cofactor
0001:00052da0  _EC_GROUP_get0_cofactor
0001:00052db0  _EC_GROUP_set_curve_name
0001:00052dc0  _EC_GROUP_get_curve_name
0001:00052dd0  _EC_GROUP_set_asn1_flag
0001:00052de0  _EC_GROUP_get_asn1_flag
0001:00052df0  _EC_GROUP_set_point_conversion_form
0001:00052e00  _EC_GROUP_get_point_conversion_form
0001:00052e10  _EC_GROUP_set_seed
0001:00052ed0  _EC_GROUP_get0_seed
0001:00052ee0  _EC_GROUP_get_seed_len
0001:00052ef0  _EC_GROUP_set_curve
0001:00052f40  _EC_GROUP_get_curve
0001:00052f90* _EC_GROUP_set_curve_GFp
0001:00052fe0* _EC_GROUP_get_curve_GFp
0001:00053030* _EC_GROUP_set_curve_GF2m
0001:00053080* _EC_GROUP_get_curve_GF2m
0001:000530d0  _EC_GROUP_get_degree
0001:00053120  _EC_GROUP_check_discriminant
0001:00053170  _EC_POINT_new
0001:00053290  _EC_GROUP_copy
0001:000536a0  _EC_GROUP_set_generator
0001:00053ba0  _EC_GROUP_dup
0001:00053fc0  _EC_POINT_free
0001:00054000  _EC_POINT_clear_free
0001:00054050  _EC_POINT_copy
0001:00054120  _EC_POINT_dup
0001:00054340* _EC_POINT_method_of
0001:00054350  _EC_POINT_set_to_infinity
0001:000543e0  _EC_POINT_set_Jprojective_coordinates_GFp
0001:000544d0* _EC_POINT_get_Jprojective_coordinates_GFp
0001:000545c0  _EC_POINT_set_affine_coordinates
0001:00054780* _EC_POINT_set_affine_coordinates_GFp
0001:00054940* _EC_POINT_set_affine_coordinates_GF2m
0001:00054b00  _EC_POINT_get_affine_coordinates
0001:00054c70* _EC_POINT_get_affine_coordinates_GFp
0001:00054de0* _EC_POINT_get_affine_coordinates_GF2m
0001:00054f50  _EC_POINT_add
0001:00055070  _EC_POINT_dbl
0001:00055160  _EC_POINT_invert
0001:00055210  _EC_POINT_is_at_infinity
0001:000552c0  _EC_POINT_is_on_curve
0001:00055370  _EC_POINT_cmp
0001:00055460  _EC_GROUP_cmp
0001:000556b0  _EC_POINT_make_affine
0001:00055760  _EC_POINTs_make_affine
0001:00055840* _EC_POINTs_mul
0001:00055a80  _EC_POINT_mul
0001:00055c90  _EC_GROUP_precompute_mult
0001:00055cd0* _EC_GROUP_have_precompute_mult
0001:00055d00* _EC_KEY_set_ex_data
0001:00055d10* _EC_KEY_get_ex_data
0001:00055d20  _ec_group_simple_order_bits
0001:00055d40  _ec_group_do_inverse_ord
0001:00055e50  _ec_point_blind_coordinates
Module: U:\tmp\ldconv_libcrypto_a_99560c9c37f156ab8.lib(ec_curve.obj)
0001:00055e90  _EC_GROUP_new_by_curve_name
0001:00056430* _EC_get_builtin_curves
0001:00056480  _EC_curve_nid2nist
0001:000565c0  _EC_curve_nist2nid
0001:000567e0  _ec_curve_nid_from_params
Module: U:\usr\lib\libc_dll.lib(bind.obj)
0001:0005bb50  _bind
Module: U:\usr\lib\libc_dll.lib(getsockname.obj)
0001:0005bc50  _getsockname
Module: U:\usr\lib\libc_dll.lib(getpeername.obj)
0001:0005bd70  _getpeername
Module: U:\usr\lib\libc_dll.lib(send.obj)
0001:0005be90  _send
Module: U:\usr\lib\libc_dll.lib(recv.obj)
0001:0005bf50  _recv
Module: U:\usr\lib\libc_dll.lib(so_ioctl.obj)
0001:0005c010  _so_ioctl
Module: U:\usr\lib\libc_dll.lib(shutdown.obj)
0001:0005c090  _shutdown
Module: U:\usr\lib\libc_dll.lib(syslog.obj)
0001:0005c27c* _vsyslog
0001:0005c6b0  _syslog
0001:0005c6d1  _openlog
0001:0005c804  _closelog
0001:0005c838* _setlogmask
Module: U:\tmp\ldconv_libgcc_a_99560c9c382191438.lib(_chkstk_ms.obj)
0001:0005c850  ___chkstk_ms
Module: U:\tmp\ldconv_libcrypto_a_99560c9c37f156ab8.lib(o_str.obj)
0001:0005c880* _OPENSSL_memcmp
0001:0005c8c0  _CRYPTO_strdup
0001:0005c920  _CRYPTO_strndup
0001:0005c9b0  _CRYPTO_memdup
0001:0005ca40  _OPENSSL_strnlen
0001:0005ca70  _OPENSSL_strlcpy
0001:0005cad0  _OPENSSL_strlcat
0001:0005cb50  _OPENSSL_hexchar2int
0001:0005cb70  _OPENSSL_hexstr2buf
0001:0005cd20  _OPENSSL_buf2hexstr
0001:0005ce00  _openssl_strerror_r
Module: U:\tmp\ldconv_libcrypto_a_99560c9c37f156ab8.lib(eng_lib.obj)
0002:0000d810  _global_engine_lock
0001:0005cec0  _do_engine_lock_init_ossl_
0001:0005cf50  _ENGINE_new
0001:0005d020  _engine_set_all_null
0001:0005d0a0  _engine_free_util
0001:0005d140  _ENGINE_free
0001:0005d1d0  _engine_cleanup_add_first
0001:0005d260  _engine_cleanup_add_last
0001:0005d310  _engine_cleanup_int
0001:0005d360  _ENGINE_set_ex_data
0001:0005d370  _ENGINE_get_ex_data
0001:0005d380  _ENGINE_set_id
0001:0005d3d0  _ENGINE_set_name
0001:0005d420  _ENGINE_set_destroy_function
0001:0005d440  _ENGINE_set_init_function
0001:0005d460  _ENGINE_set_finish_function
0001:0005d480  _ENGINE_set_ctrl_function
0001:0005d4a0  _ENGINE_set_flags
0001:0005d4c0  _ENGINE_set_cmd_defns
0001:0005d4e0  _ENGINE_get_id
0001:0005d4f0* _ENGINE_get_name
0001:0005d500* _ENGINE_get_destroy_function
0001:0005d510* _ENGINE_get_init_function
0001:0005d520* _ENGINE_get_finish_function
0001:0005d530* _ENGINE_get_ctrl_function
0001:0005d540* _ENGINE_get_flags
0001:0005d550* _ENGINE_get_cmd_defns
0001:0005d560  _ENGINE_get_static_state
0002:000005d0  _engine_lock_init
0002:0000a400  _do_engine_lock_init_ossl_ret_
Module: U:\tmp\ldconv_libcrypto_a_99560c9c37f156ab8.lib(eng_init.obj)
0001:0005d570  _engine_unlocked_init
0001:0005d5d0  _engine_unlocked_finish
0001:0005d690  _ENGINE_init
0001:0005d790  _ENGINE_finish
Module: U:\tmp\ldconv_libcrypto_a_99560c9c37f156ab8.lib(err.obj)
0001:0005dfe0  _err_cleanup
0001:0005e030  _ERR_load_ERR_strings
0001:0005e070* _ERR_load_strings
0001:0005e120  _ERR_load_strings_const
0001:0005e1b0* _ERR_unload_strings
0001:0005e230  _err_free_strings_int
0001:0005e250  _ERR_error_string_n
0001:0005e270* _ERR_error_string
0001:0005e2a0* _ERR_lib_error_string
0001:0005e320  _ERR_func_error_string
0001:0005e3a0* _ERR_reason_error_string
0001:0005e470  _err_delete_thread_state
0001:0005e930* _ERR_remove_thread_state
0001:0005e940* _ERR_remove_state
0001:0005e950* _ERR_get_state
0001:0005eed0  _ERR_put_error
0001:0005efc0  _ERR_clear_error
0001:0005f690  _ERR_get_error_line_data
0001:0005f930  _ERR_peek_last_error
0001:0005fab0  _ERR_peek_error
0001:0005fc30* _ERR_peek_last_error_line
0001:0005fe10  _ERR_get_error
0001:0005fff0* _ERR_peek_error_line
0001:000601d0  _ERR_get_error_line
0001:00060410* _ERR_peek_last_error_line_data
0001:00060640* _ERR_peek_error_line_data
0001:00060870* _err_shelve_state
0001:00060910* _err_unshelve_state
0001:00060930* _ERR_get_next_error_library
0001:00060990* _ERR_set_error_data
0001:00060a00* _ERR_add_error_vdata
0001:00060b80  _ERR_add_error_data
0001:00060ba0  _ERR_set_mark
0001:00061150  _ERR_pop_to_mark
0001:00061260  _ERR_clear_last_mark
0001:00061300  _err_clear_last_constant_time
Module: U:\tmp\ldconv_libcrypto_a_99560c9c37f156ab8.lib(o_fips.obj)
0001:000617f0  _FIPS_mode
0001:00061810  _FIPS_mode_set
Module: U:\tmp\ldconv_libcrypto_a_99560c9c37f156ab8.lib(cversion.obj)
0001:00061860  _OpenSSL_version_num
0001:00061880  _OpenSSL_version
Module: U:\tmp\ldconv_libcrypto_a_99560c9c37f156ab8.lib(eng_ctrl.obj)
0001:00061aa0  _ENGINE_ctrl
0001:00061ea0* _ENGINE_cmd_is_executable
0001:00062080  _ENGINE_ctrl_cmd
0001:000622b0  _ENGINE_ctrl_cmd_string
Module: U:\tmp\ldconv_libcrypto_a_99560c9c37f156ab8.lib(eng_fat.obj)
0001:000628c0* _ENGINE_set_default
0001:00062a20  _ENGINE_set_default_string
0001:00062ad0* _ENGINE_register_complete
0001:00062b30  _ENGINE_register_all_complete
Module: U:\tmp\ldconv_libcrypto_a_99560c9c37f156ab8.lib(eng_list.obj)
0001:00062be0  _ENGINE_get_first
0001:00062c70* _ENGINE_get_last
0001:00062d00  _ENGINE_get_next
0001:00062d80* _ENGINE_get_prev
0001:00062e00  _ENGINE_add
0001:00063000* _ENGINE_remove
0001:000631f0  _ENGINE_by_id
0001:00063520* _ENGINE_up_ref
Module: U:\usr\lib\libc_dll.lib(socket.obj)
0001:00063580  _socket
Module: U:\usr\lib\libc_dll.lib(getsockopt.obj)
0001:00063610  _getsockopt
Module: U:\tmp\ldconv_libcrypto_a_99560c9c37f156ab8.lib(bio_b64.obj)
0001:000649b0  _BIO_f_base64
Module: U:\tmp\ldconv_libcrypto_a_99560c9c37f156ab8.lib(bio_lib.obj)
0001:00064a40  _BIO_new
0001:00064be0  _BIO_free
0001:00064d00  _BIO_set_data
0001:00064d10  _BIO_get_data
0001:00064d20  _BIO_set_init
0001:00064d30  _BIO_get_init
0001:00064d40* _BIO_set_shutdown
0001:00064d50* _BIO_get_shutdown
0001:00064d60  _BIO_vfree
0001:00064e70  _BIO_up_ref
0001:00064e90  _BIO_clear_flags
0001:00064ea0  _BIO_test_flags
0001:00064eb0  _BIO_set_flags
0001:00064ec0  _BIO_get_callback
0001:00064ed0* _BIO_set_callback
0001:00064ee0* _BIO_get_callback_ex
0001:00064ef0* _BIO_set_callback_ex
0001:00064f00* _BIO_set_callback_arg
0001:00064f10* _BIO_get_callback_arg
0001:00064f20* _BIO_method_name
0001:00064f30  _BIO_method_type
0001:00064f40  _BIO_read
0001:00065190* _BIO_read_ex
0001:000653c0  _BIO_write
0001:000655c0* _BIO_write_ex
0001:000657c0  _BIO_puts
0001:00065a30  _BIO_gets
0001:00065c90  _BIO_indent
0001:00065f60  _BIO_int_ctrl
0001:000660f0* _BIO_ptr_ctrl
0001:00066290  _BIO_ctrl
0001:00066400  _BIO_callback_ctrl
0001:000665b0* _BIO_ctrl_pending
0001:00066760* _BIO_ctrl_wpending
0001:00066910  _BIO_push
0001:00066ac0  _BIO_pop
0001:00066c90* _BIO_get_retry_BIO
0001:00066cc0  _BIO_get_retry_reason
0001:00066cd0* _BIO_set_retry_reason
0001:00066ce0  _BIO_find_type
0001:00066d20  _BIO_next
0001:00066d40* _BIO_set_next
0001:00066d50  _BIO_free_all
0001:00066e80* _BIO_dup_chain
0001:00066fb0  _BIO_copy_next_retry
0001:00066fd0* _BIO_set_ex_data
0001:00066fe0* _BIO_get_ex_data
0001:00066ff0* _BIO_number_read
0001:00067010* _BIO_number_written
0001:00067030* _bio_free_ex_data
0001:00067060  _bio_cleanup
Module: U:\tmp\ldconv_libcrypto_a_99560c9c37f156ab8.lib(bss_mem.obj)
0001:00067980  _BIO_s_mem
0001:00067990  _BIO_s_secmem
0001:000679a0  _BIO_new_mem_buf
Module: U:\tmp\ldconv_libcrypto_a_99560c9c37f156ab8.lib(set_key.obj)
0001:00067ae0  _DES_set_odd_parity
0001:00067b60* _DES_check_key_parity
0001:00067be0* _DES_is_weak_key
0001:00067e90  _DES_set_key_unchecked
0001:000680a0* _DES_set_key_checked
0001:00068400* _DES_set_key
0001:00068730* _DES_key_sched
0002:0000c9b0* __shadow_DES_check_key
Module: U:\tmp\ldconv_libcrypto_a_99560c9c37f156ab8.lib(ecb_enc.obj)
0001:00069430* _DES_options
0001:00069480  _DES_ecb_encrypt
Module: U:\tmp\ldconv_libcrypto_a_99560c9c37f156ab8.lib(md4_dgst.obj)
0001:000694d0  _MD4_Init
0001:00069520* _md4_block_data_order
0001:00069a80  _MD4_Update
0001:00069be0* _MD4_Transform
0001:00069c10  _MD4_Final
Module: U:\usr\lib\libc_dll.lib(connect.obj)
0001:00069d50  _connect
Module: U:\usr\lib\libc_dll.lib(listen.obj)
0001:00069e40  _listen
Module: U:\tmp\ldconv_libcrypto_a_99560c9c37f156ab8.lib(ex_data.obj)
0001:00069fa0  _crypto_cleanup_all_ex_data_int
0001:0006a000* _CRYPTO_free_ex_index
0001:0006a150  _CRYPTO_get_ex_new_index
0001:0006a3b0  _CRYPTO_new_ex_data
0001:0006a620  _CRYPTO_free_ex_data
0001:0006a920  _CRYPTO_set_ex_data
0001:0006aa20  _CRYPTO_dup_ex_data
0001:0006ad80  _CRYPTO_get_ex_data
Module: U:\tmp\ldconv_libcrypto_a_99560c9c37f156ab8.lib(randfile.obj)
0001:0006adf0  _RAND_load_file
0001:0006b060  _RAND_write_file
0001:0006b1e0  _RAND_file_name
Module: U:\tmp\ldconv_libcrypto_a_99560c9c37f156ab8.lib(conf_lib.obj)
0001:0006b2d0  _CONF_set_nconf
0001:0006b310* _CONF_set_default_method
0001:0006b340* _CONF_load
0001:0006b3f0* _CONF_load_fp
0001:0006b4a0* _CONF_load_bio
0001:0006b500  _CONF_get_section
0001:0006b5a0  _CONF_get_string
0001:0006b6d0  _CONF_free
0001:0006b710* _CONF_dump_fp
0001:0006b7c0* _CONF_dump_bio
0001:0006b810  _NCONF_new
0001:0006b880  _NCONF_free
0001:0006b8a0* _NCONF_free_data
0001:0006b8c0  _NCONF_load
0001:0006b910* _NCONF_load_fp
0001:0006b9e0* _NCONF_load_bio
0001:0006ba30  _NCONF_get_section
0001:0006bac0  _NCONF_get_string
0001:0006bb90  _NCONF_get_number_e
0001:0006bd90* _CONF_get_number
0001:0006be40* _NCONF_dump_fp
0001:0006bef0* _NCONF_dump_bio
0001:0006bf40  _OPENSSL_INIT_new
0001:0006bf70* _OPENSSL_INIT_set_config_filename
0001:0006bfb0* _OPENSSL_INIT_set_config_file_flags
0001:0006bfc0* _OPENSSL_INIT_set_config_appname
0001:0006c000  _OPENSSL_INIT_free
Module: U:\tmp\ldconv_libcrypto_a_99560c9c37f156ab8.lib(init.obj)
0001:0006c2b0* _OPENSSL_cleanup
0001:0006c930* _OPENSSL_thread_stop
0001:0006c9c0  _ossl_init_thread_start
0001:0006caf0  _OPENSSL_init_crypto
0001:0006cba0  _OPENSSL_atexit
0001:0006cc10  _OPENSSL_fork_prepare
0001:0006cc20  _OPENSSL_fork_parent
0001:0006cc30  _OPENSSL_fork_child
Module: U:\tmp\ldconv_libcrypto_a_99560c9c37f156ab8.lib(stack.obj)
0001:0006cc40  _OPENSSL_sk_set_cmp_func
0001:0006cc80  _OPENSSL_sk_dup
0001:0006cdb0  _OPENSSL_sk_deep_copy
0001:0006cf50  _OPENSSL_sk_new_null
0001:0006cf80  _OPENSSL_sk_new
0001:0006cfb0  _OPENSSL_sk_new_reserve
0001:0006d0f0  _OPENSSL_sk_reserve
0001:0006d1d0  _OPENSSL_sk_insert
0001:0006d370  _OPENSSL_sk_delete_ptr
0001:0006d3f0  _OPENSSL_sk_delete
0001:0006d480  _OPENSSL_sk_find
0001:0006d560* _OPENSSL_sk_find_ex
0001:0006d640  _OPENSSL_sk_push
0001:0006d7d0* _OPENSSL_sk_unshift
0001:0006d950  _OPENSSL_sk_shift
0001:0006d9b0  _OPENSSL_sk_pop
0001:0006d9e0* _OPENSSL_sk_zero
0001:0006da30  _OPENSSL_sk_pop_free
0001:0006dab0  _OPENSSL_sk_free
0001:0006db00  _OPENSSL_sk_num
0001:0006db20  _OPENSSL_sk_value
0001:0006db50  _OPENSSL_sk_set
0001:0006db90  _OPENSSL_sk_sort
0001:0006dbf0  _OPENSSL_sk_is_sorted
Module: U:\tmp\ldconv_libcrypto_a_99560c9c37f156ab8.lib(c_zlib.obj)
0001:0006dc10  _COMP_zlib
0001:0006dc20  _comp_zlib_cleanup_int
Module: U:\tmp\ldconv_libcrypto_a_99560c9c37f156ab8.lib(comp_lib.obj)
0001:0006dc50  _COMP_CTX_new
0001:0006dcf0  _COMP_CTX_get_method
0001:0006dd00  _COMP_get_type
0001:0006dd10  _COMP_get_name
0001:0006dd20  _COMP_CTX_free
0001:0006dd60  _COMP_compress_block
0001:0006ddb0  _COMP_expand_block
0001:0006de00* _COMP_CTX_get_type
Module: U:\tmp\ldconv_libcrypto_a_99560c9c37f156ab8.lib(eng_all.obj)
0001:0006de10  _ENGINE_load_builtin_engines
Module: U:\tmp\ldconv_libssl_a_99560c9c37e1aece0.lib(ssl_init.obj)
0001:0006e130  _OPENSSL_init_ssl
Module: U:\tmp\ldconv_libssl_a_99560c9c37e1aece0.lib(statem.obj)
0001:0006e270  _SSL_get_state
0001:0006e280  _SSL_in_init
0001:0006e290  _SSL_is_init_finished
0001:0006e2b0  _SSL_in_before
0001:0006e2d0  _ossl_statem_clear
0001:0006e300  _ossl_statem_set_renegotiate
0001:0006e320  _ossl_statem_fatal
0001:0006f1a0  _ossl_statem_in_error
0001:0006f1b0  _ossl_statem_set_in_init
0001:0006f1c0  _ossl_statem_get_in_handshake
0001:0006f1d0  _ossl_statem_set_in_handshake
0001:0006f1f0  _ossl_statem_skip_early_data
0001:0006f220  _ossl_statem_check_finish_init
0001:0006f2c0  _ossl_statem_set_hello_verify_done
0001:0006f2e0  _ossl_statem_connect
0001:0006f300  _ossl_statem_accept
0001:0006f320  _statem_flush
0001:0006f370  _ossl_statem_app_data_allowed
0001:0006f3c0  _ossl_statem_export_allowed
0001:0006f3e0  _ossl_statem_export_early_allowed
Module: U:\tmp\ldconv_libssl_a_99560c9c37e1aece0.lib(ssl_stat.obj)
0001:0006f430  _SSL_state_string_long
0001:0006f480* _SSL_state_string
0001:0006f4e0  _SSL_alert_type_string_long
0001:0006f510* _SSL_alert_type_string
0001:0006f540* _SSL_alert_desc_string
0001:0006f560  _SSL_alert_desc_string_long
Module: U:\tmp\ldconv_libssl_a_99560c9c37e1aece0.lib(ssl_cert.obj)
0001:00070870  _SSL_get_ex_data_X509_STORE_CTX_idx
0001:000708b0  _ssl_cert_new
0001:000709a0  _ssl_cert_clear_certs
0001:00070a40  _ssl_cert_free
0001:00070bd0  _ssl_cert_dup
0001:00070fe0  _ssl_cert_set0_chain
0001:000710f0  _ssl_cert_set1_chain
0001:00071170  _ssl_cert_add0_chain_cert
0001:00071230  _ssl_cert_add1_chain_cert
0001:00071300  _ssl_cert_select_current
0001:000714c0  _ssl_cert_set_current
0001:00071540  _ssl_cert_set_cert_cb
0001:00071570  _ssl_verify_cert_chain
0001:00071860* _SSL_dup_CA_list
0001:00071950  _SSL_set0_CA_list
0001:00071980  _SSL_CTX_set0_CA_list
0001:000719b0* _SSL_CTX_get0_CA_list
0001:000719c0  _SSL_get0_CA_list
0001:000719e0  _SSL_CTX_set_client_CA_list
0001:00071a10* _SSL_CTX_get_client_CA_list
0001:00071a20* _SSL_set_client_CA_list
0001:00071a50* _SSL_get0_peer_CA_list
0001:00071a70  _SSL_get_client_CA_list
0001:00071ab0* _SSL_add1_to_CA_list
0001:00071b40* _SSL_CTX_add1_to_CA_list
0001:00071bd0* _SSL_add_client_CA
0001:00071c60* _SSL_CTX_add_client_CA
0001:00071cf0  _SSL_load_client_CA_file
0001:00071ef0  _SSL_add_file_cert_subjects_to_stack
0001:00072080  _SSL_add_dir_cert_subjects_to_stack
0001:00072220  _ssl_build_cert_chain
0001:000726a0  _ssl_cert_set_cert_store
0001:00072720  _ssl_security
0001:00072770  _ssl_ctx_security
0001:000727c0  _ssl_cert_lookup_by_nid
0001:00072850  _ssl_cert_lookup_by_pkey
0001:00072910  _ssl_cert_lookup_by_idx
Module: U:\usr\lib\libc_dll.lib(sendto.obj)
0001:000729b0  _sendto
Module: U:\tmp\ldconv_libssl_a_99560c9c37e1aece0.lib(ssl_asn1.obj)
0001:00072a80  _i2d_SSL_SESSION
0001:00072ed0  _d2i_SSL_SESSION
Module: U:\tmp\ldconv_libcrypto_a_99560c9c37f156ab8.lib(m_sha1.obj)
0001:00073d60  _EVP_sha1
0001:00073d70  _EVP_sha224
0001:00073d80  _EVP_sha256
0001:00073d90  _EVP_sha512_224
0001:00073da0  _EVP_sha512_256
0001:00073db0  _EVP_sha384
0001:00073dc0  _EVP_sha512
Module: U:\tmp\ldconv_libcrypto_a_99560c9c37f156ab8.lib(hmac.obj)
0001:00073fa0  _HMAC_Init_ex
0001:00074320  _HMAC_Update
0001:00074350  _HMAC_Final
0001:000743f0  _HMAC_size
0001:00074430  _HMAC_CTX_free
0001:000744b0* _HMAC_CTX_reset
0001:00074570* _HMAC_Init
0001:000745d0  _HMAC_CTX_new
0001:00074680  _HMAC_CTX_copy
0001:00074780  _HMAC
0001:000749a0  _HMAC_CTX_set_flags
0001:000749e0* _HMAC_CTX_get_md
Module: U:\tmp\ldconv_libcrypto_a_99560c9c37f156ab8.lib(e_aes.obj)
0001:00077680  _EVP_aes_128_cbc
0001:00077690  _EVP_aes_128_ecb
0001:000776a0  _EVP_aes_128_ofb
0001:000776b0  _EVP_aes_128_cfb128
0001:000776c0  _EVP_aes_128_cfb1
0001:000776d0  _EVP_aes_128_cfb8
0001:000776e0  _EVP_aes_128_ctr
0001:000776f0  _EVP_aes_192_cbc
0001:00077700  _EVP_aes_192_ecb
0001:00077710  _EVP_aes_192_ofb
0001:00077720  _EVP_aes_192_cfb128
0001:00077730  _EVP_aes_192_cfb1
0001:00077740  _EVP_aes_192_cfb8
0001:00077750  _EVP_aes_192_ctr
0001:00077760  _EVP_aes_256_cbc
0001:00077770  _EVP_aes_256_ecb
0001:00077780  _EVP_aes_256_ofb
0001:00077790  _EVP_aes_256_cfb128
0001:000777a0  _EVP_aes_256_cfb1
0001:000777b0  _EVP_aes_256_cfb8
0001:000777c0  _EVP_aes_256_ctr
0001:000777d0  _EVP_aes_128_gcm
0001:000777e0  _EVP_aes_192_gcm
0001:000777f0  _EVP_aes_256_gcm
0001:00077800  _EVP_aes_128_xts
0001:00077810  _EVP_aes_256_xts
0001:00077820  _EVP_aes_128_ccm
0001:00077830  _EVP_aes_192_ccm
0001:00077840  _EVP_aes_256_ccm
0001:00077850  _EVP_aes_128_wrap
0001:00077860  _EVP_aes_192_wrap
0001:00077870  _EVP_aes_256_wrap
0001:00077880  _EVP_aes_128_wrap_pad
0001:00077890  _EVP_aes_192_wrap_pad
0001:000778a0  _EVP_aes_256_wrap_pad
0001:000778b0  _EVP_aes_128_ocb
0001:000778c0  _EVP_aes_192_ocb
0001:000778d0  _EVP_aes_256_ocb
Module: U:\tmp\ldconv_libcrypto_a_99560c9c37f156ab8.lib(evp_enc.obj)
0001:00078650  _EVP_CIPHER_CTX_reset
0001:00078710  _EVP_CIPHER_CTX_new
0001:00078740  _EVP_CIPHER_CTX_free
0001:000788b0* _EVP_CipherInit
0001:00078d90  _EVP_CipherInit_ex
0001:000792e0  _EVP_CipherUpdate
0001:00079680  _EVP_CipherFinal_ex
0001:00079a30* _EVP_CipherFinal
0001:00079de0* _EVP_EncryptInit
0001:0007a290  _EVP_EncryptInit_ex
0001:0007a790* _EVP_DecryptInit
0001:0007ac40  _EVP_DecryptInit_ex
0001:0007b140  _is_partially_overlapping
0001:0007b170  _EVP_EncryptUpdate
0001:0007b540  _EVP_EncryptFinal
0001:0007b6b0  _EVP_EncryptFinal_ex
0001:0007b820  _EVP_DecryptUpdate
0001:0007bb90  _EVP_DecryptFinal
0001:0007bea0  _EVP_DecryptFinal_ex
0001:0007c1b0  _EVP_CIPHER_CTX_set_key_length
0001:0007c2b0  _EVP_CIPHER_CTX_set_padding
0001:0007c2d0  _EVP_CIPHER_CTX_ctrl
0001:0007c3b0  _EVP_CIPHER_CTX_rand_key
0001:0007c480  _EVP_CIPHER_CTX_copy
Module: U:\tmp\ldconv_libcrypto_a_99560c9c37f156ab8.lib(evp_lib.obj)
0001:0007c6c0  _EVP_CIPHER_param_to_asn1
0001:0007c8d0  _EVP_CIPHER_get_asn1_iv
0001:0007c9b0  _EVP_CIPHER_asn1_to_param
0001:0007cac0  _EVP_CIPHER_set_asn1_iv
0001:0007cb70  _EVP_CIPHER_type
0001:0007ccc0  _EVP_CIPHER_block_size
0001:0007ccd0  _EVP_CIPHER_CTX_block_size
0001:0007cce0* _EVP_CIPHER_impl_ctx_size
0001:0007ccf0  _EVP_Cipher
0001:0007cd00  _EVP_CIPHER_CTX_cipher
0001:0007cd10  _EVP_CIPHER_CTX_encrypting
0001:0007cd20  _EVP_CIPHER_flags
0001:0007cd30* _EVP_CIPHER_CTX_get_app_data
0001:0007cd40* _EVP_CIPHER_CTX_set_app_data
0001:0007cd50  _EVP_CIPHER_CTX_get_cipher_data
0001:0007cd60* _EVP_CIPHER_CTX_set_cipher_data
0001:0007cd80  _EVP_CIPHER_iv_length
0001:0007cd90  _EVP_CIPHER_CTX_iv_length
0001:0007cdf0  _EVP_CIPHER_CTX_original_iv
0001:0007ce00* _EVP_CIPHER_CTX_iv
0001:0007ce10  _EVP_CIPHER_CTX_iv_noconst
0001:0007ce20  _EVP_CIPHER_CTX_buf_noconst
0001:0007ce30  _EVP_CIPHER_CTX_num
0001:0007ce40  _EVP_CIPHER_CTX_set_num
0001:0007ce50  _EVP_CIPHER_key_length
0001:0007ce60  _EVP_CIPHER_CTX_key_length
0001:0007ce70  _EVP_CIPHER_nid
0001:0007ce80* _EVP_CIPHER_CTX_nid
0001:0007ce90  _EVP_MD_block_size
0001:0007cea0  _EVP_MD_type
0001:0007ceb0  _EVP_MD_pkey_type
0001:0007cec0  _EVP_MD_size
0001:0007cf10* _EVP_MD_flags
0001:0007cf20  _EVP_MD_meth_new
0001:0007cf60* _EVP_MD_meth_dup
0001:0007cff0  _EVP_MD_meth_free
0001:0007d020  _EVP_MD_meth_set_input_blocksize
0001:0007d040  _EVP_MD_meth_set_result_size
0001:0007d060  _EVP_MD_meth_set_app_datasize
0001:0007d080  _EVP_MD_meth_set_flags
0001:0007d0a0  _EVP_MD_meth_set_init
0001:0007d0c0  _EVP_MD_meth_set_update
0001:0007d0e0  _EVP_MD_meth_set_final
0001:0007d100* _EVP_MD_meth_set_copy
0001:0007d120* _EVP_MD_meth_set_cleanup
0001:0007d140* _EVP_MD_meth_set_ctrl
0001:0007d160* _EVP_MD_meth_get_input_blocksize
0001:0007d170* _EVP_MD_meth_get_result_size
0001:0007d180* _EVP_MD_meth_get_app_datasize
0001:0007d190  _EVP_MD_meth_get_flags
0001:0007d1a0* _EVP_MD_meth_get_init
0001:0007d1b0* _EVP_MD_meth_get_update
0001:0007d1c0* _EVP_MD_meth_get_final
0001:0007d1d0* _EVP_MD_meth_get_copy
0001:0007d1e0* _EVP_MD_meth_get_cleanup
0001:0007d1f0* _EVP_MD_meth_get_ctrl
0001:0007d200  _EVP_MD_CTX_md
0001:0007d220  _EVP_MD_CTX_pkey_ctx
0001:0007d230* _EVP_MD_CTX_set_pkey_ctx
0001:0007d270  _EVP_MD_CTX_md_data
0001:0007d280* _EVP_MD_CTX_update_fn
0001:0007d290  _EVP_MD_CTX_set_update_fn
0001:0007d2a0  _EVP_MD_CTX_set_flags
0001:0007d2b0  _EVP_MD_CTX_clear_flags
0001:0007d2c0  _EVP_MD_CTX_test_flags
0001:0007d2d0  _EVP_CIPHER_CTX_set_flags
0001:0007d2e0* _EVP_CIPHER_CTX_clear_flags
0001:0007d2f0  _EVP_CIPHER_CTX_test_flags
Module: U:\tmp\ldconv_libcrypto_a_99560c9c37f156ab8.lib(evp_key.obj)
0001:0007d300  _EVP_set_pw_prompt
0001:0007d340  _EVP_get_pw_prompt
0001:0007d360  _EVP_read_pw_string_min
0001:0007d480* _EVP_read_pw_string
0001:0007d530  _EVP_BytesToKey
Module: U:\tmp\ldconv_libcrypto_a_99560c9c37f156ab8.lib(pem_x509.obj)
0001:0007d840  _PEM_read_bio_X509
0001:0007d880* _PEM_read_X509
0001:0007d8c0  _PEM_write_bio_X509
0001:0007d920* _PEM_write_X509
Module: U:\tmp\ldconv_libcrypto_a_99560c9c37f156ab8.lib(bss_file.obj)
0001:0007e070  _BIO_new_file
0001:0007e1f0  _BIO_new_fp
0001:0007e240  _BIO_s_file
Module: U:\tmp\ldconv_libcrypto_a_99560c9c37f156ab8.lib(p12_utl.obj)
0001:0007e2c0  _OPENSSL_asc2uni
0001:0007e390* _OPENSSL_uni2asc
0001:0007e450  _OPENSSL_utf82uni
0001:0007e670  _OPENSSL_uni2utf8
0001:0007e910* _i2d_PKCS12_bio
0001:0007e940* _i2d_PKCS12_fp
0001:0007e970  _d2i_PKCS12_bio
0001:0007e9a0* _d2i_PKCS12_fp
Module: U:\tmp\ldconv_libcrypto_a_99560c9c37f156ab8.lib(p12_kiss.obj)
0001:0007ec40  _PKCS12_parse
Module: U:\tmp\ldconv_libcrypto_a_99560c9c37f156ab8.lib(p12_asn.obj)
0001:0007f060  _d2i_PKCS12
0001:0007f684  _PKCS12_it
0001:0007f090* _i2d_PKCS12
0001:0007f0c0* _PKCS12_new
0001:0007f0e0  _PKCS12_free
0001:0007f100* _d2i_PKCS12_MAC_DATA
0001:0007f60c* _PKCS12_MAC_DATA_it
0001:0007f130* _i2d_PKCS12_MAC_DATA
0001:0007f160  _PKCS12_MAC_DATA_new
0001:0007f180  _PKCS12_MAC_DATA_free
0001:0007f1a0* _d2i_PKCS12_BAGS
0001:0007f4fc* _PKCS12_BAGS_it
0001:0007f1d0* _i2d_PKCS12_BAGS
0001:0007f200  _PKCS12_BAGS_new
0001:0007f220  _PKCS12_BAGS_free
0001:0007f240* _d2i_PKCS12_SAFEBAG
0001:0007f36c* _PKCS12_SAFEBAG_it
0001:0007f270* _i2d_PKCS12_SAFEBAG
0001:0007f2a0  _PKCS12_SAFEBAG_new
0001:0007f2c0  _PKCS12_SAFEBAG_free
0001:0007f2ec  _PKCS12_AUTHSAFES_it
0001:0007f32c  _PKCS12_SAFEBAGS_it
Module: U:\tmp\ldconv_libssl_a_99560c9c37e1aece0.lib(ssl_rsa.obj)
0001:000804f0  _SSL_use_certificate
0001:000805b0* _SSL_use_certificate_file
0001:000807a0* _SSL_use_certificate_ASN1
0001:00080880* _SSL_use_RSAPrivateKey
0001:00080970* _SSL_use_RSAPrivateKey_file
0001:00080b20* _SSL_use_RSAPrivateKey_ASN1
0001:00080bb0  _SSL_use_PrivateKey
0001:00080d50  _SSL_use_PrivateKey_file
0001:00080f10* _SSL_use_PrivateKey_ASN1
0001:00080fb0  _SSL_CTX_use_certificate
0001:00081070* _SSL_CTX_use_certificate_file
0001:00081250* _SSL_CTX_use_certificate_ASN1
0001:00081330* _SSL_CTX_use_RSAPrivateKey
0001:00081420* _SSL_CTX_use_RSAPrivateKey_file
0001:000815c0* _SSL_CTX_use_RSAPrivateKey_ASN1
0001:00081650  _SSL_CTX_use_PrivateKey
0001:000817f0  _SSL_CTX_use_PrivateKey_file
0001:000819a0* _SSL_CTX_use_PrivateKey_ASN1
0001:00081a40  _SSL_CTX_use_certificate_chain_file
0001:00081a50  _SSL_use_certificate_chain_file
0001:00081a60* _SSL_CTX_use_serverinfo_ex
0001:00081c60* _SSL_CTX_use_serverinfo
0001:00081e80  _SSL_CTX_use_serverinfo_file
0001:00082410* _SSL_use_cert_and_key
0001:00082440* _SSL_CTX_use_cert_and_key
Module: U:\tmp\ldconv_libcrypto_a_99560c9c37f156ab8.lib(ui_lib.obj)
0001:000828e0  _UI_new
0001:000829f0* _UI_new_method
0001:00082b10  _UI_free
0001:00082b90  _UI_add_input_string
0001:00082e20* _UI_dup_input_string
0001:00083110  _UI_add_verify_string
0001:000833a0* _UI_dup_verify_string
0001:00083690* _UI_add_input_boolean
0001:000836d0* _UI_dup_input_boolean
0001:000838e0* _UI_add_info_string
0001:00083b20* _UI_dup_info_string
0001:00083db0* _UI_add_error_string
0001:00083ff0* _UI_dup_error_string
0001:00084280  _UI_construct_prompt
0001:00084430  _UI_add_user_data
0001:00084480* _UI_dup_user_data
0001:00084550* _UI_get0_user_data
0001:00084560* _UI_get0_result
0001:00084630* _UI_get_result_length
0001:00084750  _UI_process
0001:00084920* _UI_ctrl
0001:000849e0* _UI_set_ex_data
0001:000849f0* _UI_get_ex_data
0001:00084a00* _UI_get_method
0001:00084a10  _UI_set_method
0001:00084a20  _UI_create_method
0001:00084b00* _UI_destroy_method
0001:00084b60  _UI_method_set_opener
0001:00084b80  _UI_method_set_writer
0001:00084ba0* _UI_method_set_flusher
0001:00084bc0  _UI_method_set_reader
0001:00084be0  _UI_method_set_closer
0001:00084c00* _UI_method_set_data_duplicator
0001:00084c30* _UI_method_set_prompt_constructor
0001:00084c50* _UI_method_set_ex_data
0001:00084c60  _UI_method_get_opener
0001:00084c70  _UI_method_get_writer
0001:00084c80* _UI_method_get_flusher
0001:00084c90  _UI_method_get_reader
0001:00084ca0  _UI_method_get_closer
0001:00084cb0* _UI_method_get_prompt_constructor
0001:00084cc0* _UI_method_get_data_duplicator
0001:00084cd0* _UI_method_get_data_destructor
0001:00084ce0* _UI_method_get_ex_data
0001:00084cf0  _UI_get_string_type
0001:00084d00  _UI_get_input_flags
0001:00084d10  _UI_get0_output_string
0001:00084d20  _UI_get0_action_string
0001:00084d30  _UI_get0_result_string
0001:00084d50* _UI_get_result_string_length
0001:00084d70  _UI_get0_test_string
0001:00084d80* _UI_get_result_minsize
0001:00084da0* _UI_get_result_maxsize
0001:00084df0* _UI_set_result_ex
0001:00085020  _UI_set_result
Module: U:\tmp\ldconv_libssl_a_99560c9c37e1aece0.lib(methods.obj)
0001:00085060  _TLS_method
0001:00085070* _tlsv1_3_method
0001:00085080* _tlsv1_2_method
0001:00085090* _tlsv1_1_method
0001:000850a0* _tlsv1_method
0001:000850b0  _TLS_server_method
0001:000850c0  _tlsv1_3_server_method
0001:000850d0  _tlsv1_2_server_method
0001:000850e0  _tlsv1_1_server_method
0001:000850f0  _tlsv1_server_method
0001:00085100  _TLS_client_method
0001:00085110  _tlsv1_3_client_method
0001:00085120  _tlsv1_2_client_method
0001:00085130  _tlsv1_1_client_method
0001:00085140  _tlsv1_client_method
0001:00085150* _dtlsv1_method
0001:00085160* _dtlsv1_2_method
0001:00085170  _DTLS_method
0001:00085180  _dtlsv1_server_method
0001:00085190  _dtlsv1_2_server_method
0001:000851a0* _DTLS_server_method
0001:000851b0  _dtlsv1_client_method
0001:000851c0  _dtls_bad_ver_client_method
0001:000851d0  _dtlsv1_2_client_method
0001:000851e0* _DTLS_client_method
0001:000851f0* _TLSv1_2_method
0001:00085200* _TLSv1_2_server_method
0001:00085210* _TLSv1_2_client_method
0001:00085220* _TLSv1_1_method
0001:00085230* _TLSv1_1_server_method
0001:00085240* _TLSv1_1_client_method
0001:00085250* _TLSv1_method
0001:00085260* _TLSv1_server_method
0001:00085270* _TLSv1_client_method
0001:00085280* _DTLSv1_2_method
0001:00085290* _DTLSv1_2_server_method
0001:000852a0* _DTLSv1_2_client_method
0001:000852b0* _DTLSv1_method
0001:000852c0* _DTLSv1_server_method
0001:000852d0* _DTLSv1_client_method
Module: U:\tmp\ldconv_libssl_a_99560c9c37e1aece0.lib(ssl_conf.obj)
0001:00087480  _SSL_CONF_cmd
0001:00087740* _SSL_CONF_cmd_argv
0001:000879f0* _SSL_CONF_cmd_value_type
0001:00087ac0  _SSL_CONF_CTX_new
0001:00087af0  _SSL_CONF_CTX_finish
0001:00088000  _SSL_CONF_CTX_free
0001:00088090  _SSL_CONF_CTX_set_flags
0001:000880a0* _SSL_CONF_CTX_clear_flags
0001:000880b0* _SSL_CONF_CTX_set1_prefix
0001:00088160  _SSL_CONF_CTX_set_ssl
0001:000881e0  _SSL_CONF_CTX_set_ssl_ctx
Module: U:\tmp\ldconv_libcrypto_a_99560c9c37f156ab8.lib(eng_pkey.obj)
0001:00088ce0  _ENGINE_set_load_privkey_function
0001:00088d00* _ENGINE_set_load_pubkey_function
0001:00088d20* _ENGINE_set_load_ssl_client_cert_function
0001:00088d40* _ENGINE_get_load_privkey_function
0001:00088d50* _ENGINE_get_load_pubkey_function
0001:00088d60  _ENGINE_get_ssl_client_cert_function
0001:00088d90  _ENGINE_load_private_key
0001:00088ef0* _ENGINE_load_public_key
0001:00089050  _ENGINE_load_ssl_client_cert
Module: U:\tmp\ldconv_libcrypto_a_99560c9c37f156ab8.lib(pem_pkey.obj)
0001:000891f0  _PEM_read_bio_PrivateKey
0001:00089530* _PEM_write_bio_PrivateKey
0001:00089670* _PEM_write_bio_PrivateKey_traditional
0001:00089770* _PEM_read_bio_Parameters
0001:000898f0* _PEM_write_bio_Parameters
0001:00089990  _PEM_read_PrivateKey
0001:00089a30* _PEM_write_PrivateKey
0001:00089bf0  _PEM_read_bio_DHparams
0001:00089d30* _PEM_read_DHparams
Module: U:\tmp\ldconv_libcrypto_a_99560c9c37f156ab8.lib(dh_lib.obj)
0001:00089dd0* _DH_set_method
0001:00089e30  _DH_free
0001:00089f20* _DH_new_method
0001:0008a110  _DH_new
0001:0008a130  _DH_up_ref
0001:0008a150* _DH_set_ex_data
0001:0008a160* _DH_get_ex_data
0001:0008a170* _DH_bits
0001:0008a180  _DH_size
0001:0008a1b0  _DH_security_bits
0001:0008a200  _DH_get0_pqg
0001:0008a230  _DH_set0_pqg
0001:0008a300* _DH_get_length
0001:0008a310* _DH_set_length
0001:0008a330  _DH_get0_key
0001:0008a360  _DH_set0_key
0001:0008a3b0* _DH_get0_p
0001:0008a3c0  _DH_get0_q
0001:0008a3d0* _DH_get0_g
0001:0008a3e0* _DH_get0_priv_key
0001:0008a3f0* _DH_get0_pub_key
0001:0008a400* _DH_clear_flags
0001:0008a410* _DH_test_flags
0001:0008a420* _DH_set_flags
0001:0008a430* _DH_get0_engine
Module: U:\tmp\ldconv_libcrypto_a_99560c9c37f156ab8.lib(a_time.obj)
0001:0008a440* _d2i_ASN1_TIME
0001:0008bdbc  _ASN1_TIME_it
0001:0008a470* _i2d_ASN1_TIME
0001:0008a4a0* _ASN1_TIME_new
0001:0008a4c0  _ASN1_TIME_free
0001:0008a4e0  _asn1_time_to_tm
0001:0008aba0  _asn1_time_from_tm
0001:0008ad30* _ASN1_TIME_set
0001:0008aee0  _ASN1_TIME_adj
0001:0008b0d0  _ASN1_TIME_check
0001:0008b100* _ASN1_TIME_to_generalizedtime
0001:0008b2b0* _ASN1_TIME_set_string
0001:0008b300* _ASN1_TIME_set_string_X509
0001:0008b440* _ASN1_TIME_to_tm
0001:0008b4c0  _ASN1_TIME_diff
0001:0008b600  _ASN1_TIME_print
0001:0008b7f0* _ASN1_TIME_cmp_time_t
0001:0008b8d0* _ASN1_TIME_normalize
0001:0008bb40* _ASN1_TIME_compare
Module: U:\tmp\ldconv_libcrypto_a_99560c9c37f156ab8.lib(ocsp_asn.obj)
0001:0008bde0* _d2i_OCSP_SIGNATURE
0001:0008cfc0* _OCSP_SIGNATURE_it
0001:0008be10* _i2d_OCSP_SIGNATURE
0001:0008be40  _OCSP_SIGNATURE_new
0001:0008be60  _OCSP_SIGNATURE_free
0001:0008be80* _d2i_OCSP_CERTID
0001:0008cef4  _OCSP_CERTID_it
0001:0008beb0* _i2d_OCSP_CERTID
0001:0008bee0  _OCSP_CERTID_new
0001:0008bf00  _OCSP_CERTID_free
0001:0008bf20* _d2i_OCSP_ONEREQ
0001:0008ce7c* _OCSP_ONEREQ_it
0001:0008bf50* _i2d_OCSP_ONEREQ
0001:0008bf80  _OCSP_ONEREQ_new
0001:0008bfa0  _OCSP_ONEREQ_free
0001:0008bfc0* _d2i_OCSP_REQINFO
0001:0008cdd8  _OCSP_REQINFO_it
0001:0008bff0* _i2d_OCSP_REQINFO
0001:0008c020* _OCSP_REQINFO_new
0001:0008c040* _OCSP_REQINFO_free
0001:0008c060* _d2i_OCSP_REQUEST
0001:0008cd58  _OCSP_REQUEST_it
0001:0008c090* _i2d_OCSP_REQUEST
0001:0008c0c0  _OCSP_REQUEST_new
0001:0008c0e0  _OCSP_REQUEST_free
0001:0008c100* _d2i_OCSP_RESPBYTES
0001:0008ccd8* _OCSP_RESPBYTES_it
0001:0008c130* _i2d_OCSP_RESPBYTES
0001:0008c160* _OCSP_RESPBYTES_new
0001:0008c180* _OCSP_RESPBYTES_free
0001:0008c1a0  _d2i_OCSP_RESPONSE
0001:0008cc58  _OCSP_RESPONSE_it
0001:0008c1d0* _i2d_OCSP_RESPONSE
0001:0008c200* _OCSP_RESPONSE_new
0001:0008c220  _OCSP_RESPONSE_free
0001:0008c240  _d2i_OCSP_RESPID
0001:0008cbd4* _OCSP_RESPID_it
0001:0008c270  _i2d_OCSP_RESPID
0001:0008c2a0* _OCSP_RESPID_new
0001:0008c2c0  _OCSP_RESPID_free
0001:0008c2e0* _d2i_OCSP_REVOKEDINFO
0001:0008cb50* _OCSP_REVOKEDINFO_it
0001:0008c310* _i2d_OCSP_REVOKEDINFO
0001:0008c340* _OCSP_REVOKEDINFO_new
0001:0008c360* _OCSP_REVOKEDINFO_free
0001:0008c380* _d2i_OCSP_CERTSTATUS
0001:0008cab4* _OCSP_CERTSTATUS_it
0001:0008c3b0* _i2d_OCSP_CERTSTATUS
0001:0008c3e0* _OCSP_CERTSTATUS_new
0001:0008c400* _OCSP_CERTSTATUS_free
0001:0008c420* _d2i_OCSP_SINGLERESP
0001:0008c9d4* _OCSP_SINGLERESP_it
0001:0008c450* _i2d_OCSP_SINGLERESP
0001:0008c480* _OCSP_SINGLERESP_new
0001:0008c4a0* _OCSP_SINGLERESP_free
0001:0008c4c0* _d2i_OCSP_RESPDATA
0001:0008c900  _OCSP_RESPDATA_it
0001:0008c4f0* _i2d_OCSP_RESPDATA
0001:0008c520* _OCSP_RESPDATA_new
0001:0008c540* _OCSP_RESPDATA_free
0001:0008c560* _d2i_OCSP_BASICRESP
0001:0008c84c  _OCSP_BASICRESP_it
0001:0008c590* _i2d_OCSP_BASICRESP
0001:0008c5c0* _OCSP_BASICRESP_new
0001:0008c5e0  _OCSP_BASICRESP_free
0001:0008c600* _d2i_OCSP_CRLID
0001:0008c7b4  _OCSP_CRLID_it
0001:0008c630* _i2d_OCSP_CRLID
0001:0008c660  _OCSP_CRLID_new
0001:0008c680  _OCSP_CRLID_free
0001:0008c6a0* _d2i_OCSP_SERVICELOC
0001:0008c74c  _OCSP_SERVICELOC_it
0001:0008c6d0* _i2d_OCSP_SERVICELOC
0001:0008c700  _OCSP_SERVICELOC_new
0001:0008c720  _OCSP_SERVICELOC_free
Module: U:\tmp\ldconv_libcrypto_a_99560c9c37f156ab8.lib(ocsp_lib.obj)
0001:0008d040* _OCSP_cert_id_new
0001:0008d1e0  _OCSP_cert_to_id
0001:0008d260  _OCSP_id_issuer_cmp
0001:0008d2c0  _OCSP_id_cmp
0001:0008d350  _OCSP_parse_url
0001:0008d680  _OCSP_CERTID_dup
Module: U:\tmp\ldconv_libcrypto_a_99560c9c37f156ab8.lib(ocsp_cl.obj)
0001:0008d6a0  _OCSP_request_add0_id
0001:0008d700* _OCSP_request_set1_name
0001:0008d770* _OCSP_request_add1_cert
0001:0008d830* _OCSP_request_sign
0001:0008da70  _OCSP_response_status
0001:0008da80  _OCSP_response_get1_basic
0001:0008db30* _OCSP_resp_get0_signature
0001:0008db40* _OCSP_resp_get0_tbs_sigalg
0001:0008db50* _OCSP_resp_get0_respdata
0001:0008db60  _OCSP_resp_count
0001:0008db80  _OCSP_resp_get0
0001:0008dba0* _OCSP_resp_get0_produced_at
0001:0008dbb0* _OCSP_resp_get0_certs
0001:0008dbc0* _OCSP_resp_get0_id
0001:0008dc10* _OCSP_resp_get1_id
0001:0008dc90* _OCSP_resp_find
0001:0008dd00* _OCSP_single_get0_status
0001:0008dd90  _OCSP_resp_find_status
0001:0008dea0  _OCSP_check_validity
0001:0008e0e0* _OCSP_SINGLERESP_get0_id
Module: U:\tmp\ldconv_libcrypto_a_99560c9c37f156ab8.lib(bss_sock.obj)
0001:0008e470  _BIO_s_socket
0001:0008e480  _BIO_new_socket
0001:0008e4c0  _BIO_sock_should_retry
0001:0008e520* _BIO_sock_non_fatal_error
Module: U:\tmp\ldconv_libcrypto_a_99560c9c37f156ab8.lib(ocsp_ht.obj)
0001:0008e5d0* _OCSP_REQ_CTX_new
0001:0008e6c0  _OCSP_REQ_CTX_free
0001:0008e710* _OCSP_REQ_CTX_get0_mem_bio
0001:0008e720* _OCSP_set_max_response_length
0001:0008e740* _OCSP_REQ_CTX_i2d
0001:0008e7c0* _OCSP_REQ_CTX_http
0001:0008e810  _OCSP_REQ_CTX_set1_req
0001:0008e890  _OCSP_REQ_CTX_add1_header
0001:0008e940  _OCSP_sendreq_new
0001:0008ea60* _OCSP_REQ_CTX_nbio
0001:0008f100  _OCSP_REQ_CTX_nbio_d2i
0001:0008f180  _OCSP_sendreq_nbio
0001:0008f200* _OCSP_sendreq_bio
Module: U:\tmp\ldconv_libcrypto_a_99560c9c37f156ab8.lib(ocsp_ext.obj)
0001:0008f4d0* _OCSP_REQUEST_get_ext_count
0001:0008f4e0* _OCSP_REQUEST_get_ext_by_NID
0001:0008f4f0* _OCSP_REQUEST_get_ext_by_OBJ
0001:0008f500* _OCSP_REQUEST_get_ext_by_critical
0001:0008f510* _OCSP_REQUEST_get_ext
0001:0008f520* _OCSP_REQUEST_delete_ext
0001:0008f530* _OCSP_REQUEST_get1_ext_d2i
0001:0008f540* _OCSP_REQUEST_add1_ext_i2d
0001:0008f550* _OCSP_REQUEST_add_ext
0001:0008f580* _OCSP_ONEREQ_get_ext_count
0001:0008f590* _OCSP_ONEREQ_get_ext_by_NID
0001:0008f5a0* _OCSP_ONEREQ_get_ext_by_OBJ
0001:0008f5b0* _OCSP_ONEREQ_get_ext_by_critical
0001:0008f5c0* _OCSP_ONEREQ_get_ext
0001:0008f5d0* _OCSP_ONEREQ_delete_ext
0001:0008f5e0* _OCSP_ONEREQ_get1_ext_d2i
0001:0008f5f0* _OCSP_ONEREQ_add1_ext_i2d
0001:0008f600* _OCSP_ONEREQ_add_ext
0001:0008f630* _OCSP_BASICRESP_get_ext_count
0001:0008f640* _OCSP_BASICRESP_get_ext_by_NID
0001:0008f650* _OCSP_BASICRESP_get_ext_by_OBJ
0001:0008f660* _OCSP_BASICRESP_get_ext_by_critical
0001:0008f670* _OCSP_BASICRESP_get_ext
0001:0008f680* _OCSP_BASICRESP_delete_ext
0001:0008f690* _OCSP_BASICRESP_get1_ext_d2i
0001:0008f6a0* _OCSP_BASICRESP_add1_ext_i2d
0001:0008f6b0* _OCSP_BASICRESP_add_ext
0001:0008f6e0* _OCSP_SINGLERESP_get_ext_count
0001:0008f6f0* _OCSP_SINGLERESP_get_ext_by_NID
0001:0008f700* _OCSP_SINGLERESP_get_ext_by_OBJ
0001:0008f710* _OCSP_SINGLERESP_get_ext_by_critical
0001:0008f720* _OCSP_SINGLERESP_get_ext
0001:0008f730* _OCSP_SINGLERESP_delete_ext
0001:0008f740  _OCSP_SINGLERESP_get1_ext_d2i
0001:0008f750* _OCSP_SINGLERESP_add1_ext_i2d
0001:0008f760* _OCSP_SINGLERESP_add_ext
0001:0008f7b0  _OCSP_request_add1_nonce
0001:0008f8e0* _OCSP_basic_add1_nonce
0001:0008fa10  _OCSP_check_nonce
0001:0008fae0* _OCSP_copy_nonce
0001:0008fb50* _OCSP_crlID_new
0001:0008fc20* _OCSP_accept_responses_new
0001:0008fcb0* _OCSP_archive_cutoff_new
0001:0008fd20* _OCSP_url_svcloc_new
Module: U:\tmp\ldconv_libcrypto_a_99560c9c37f156ab8.lib(x509_vfy.obj)
0001:00090d30* _X509_cmp_current_time
0001:00090e30  _X509_cmp_time
0001:00090f40  _x509_check_cert_time
0001:00092310  _X509_gmtime_adj
0001:000923a0* _X509_time_adj
0001:00092450* _X509_time_adj_ex
0001:00092500* _X509_get_pubkey_parameters
0001:00093d50  _X509_verify_cert
0001:000941d0* _X509_CRL_diff
0001:00094670  _X509_STORE_CTX_set_ex_data
0001:00094680  _X509_STORE_CTX_get_ex_data
0001:00094690  _X509_STORE_CTX_get_error
0001:000946a0  _X509_STORE_CTX_set_error
0001:000946b0  _X509_STORE_CTX_get_error_depth
0001:000946c0* _X509_STORE_CTX_set_error_depth
0001:000946d0  _X509_STORE_CTX_get_current_cert
0001:000946e0* _X509_STORE_CTX_set_current_cert
0001:000946f0  _X509_STORE_CTX_get0_chain
0001:00094700  _X509_STORE_CTX_get1_chain
0001:00094720* _X509_STORE_CTX_get0_current_issuer
0001:00094730* _X509_STORE_CTX_get0_current_crl
0001:00094740* _X509_STORE_CTX_get0_parent_ctx
0001:00094750* _X509_STORE_CTX_set_cert
0001:00094760* _X509_STORE_CTX_set0_crls
0001:00094770  _X509_STORE_CTX_set_purpose
0001:000948c0  _X509_STORE_CTX_set_trust
0001:00094930* _X509_STORE_CTX_purpose_inherit
0001:00094ae0  _X509_STORE_CTX_new
0001:00094b50  _X509_STORE_CTX_free
0001:00094c10  _X509_STORE_CTX_init
0001:00095320* _X509_STORE_CTX_set0_trusted_stack
0001:00095340  _X509_STORE_CTX_cleanup
0001:000953d0* _X509_STORE_CTX_set_depth
0001:000953e0  _X509_STORE_CTX_set_flags
0001:000953f0* _X509_STORE_CTX_set_time
0001:00095410* _X509_STORE_CTX_get0_cert
0001:00095420* _X509_STORE_CTX_get0_untrusted
0001:00095430* _X509_STORE_CTX_set0_untrusted
0001:00095440* _X509_STORE_CTX_set0_verified_chain
0001:00095470  _X509_STORE_CTX_set_verify_cb
0001:00095480* _X509_STORE_CTX_get_verify_cb
0001:00095490* _X509_STORE_CTX_set_verify
0001:000954a0* _X509_STORE_CTX_get_verify
0001:000954b0* _X509_STORE_CTX_get_get_issuer
0001:000954c0* _X509_STORE_CTX_get_check_issued
0001:000954d0* _X509_STORE_CTX_get_check_revocation
0001:000954e0* _X509_STORE_CTX_get_get_crl
0001:000954f0* _X509_STORE_CTX_get_check_crl
0001:00095500* _X509_STORE_CTX_get_cert_crl
0001:00095510* _X509_STORE_CTX_get_check_policy
0001:00095520* _X509_STORE_CTX_get_lookup_certs
0001:00095530* _X509_STORE_CTX_get_lookup_crls
0001:00095540* _X509_STORE_CTX_get_cleanup
0001:00095550* _X509_STORE_CTX_get0_policy_tree
0001:00095560* _X509_STORE_CTX_get_explicit_policy
0001:00095570* _X509_STORE_CTX_get_num_untrusted
0001:00095580  _X509_STORE_CTX_set_default
0001:000955c0  _X509_STORE_CTX_get0_param
0001:000955d0* _X509_STORE_CTX_set0_param
0001:000955f0  _X509_STORE_CTX_set0_dane
Module: U:\tmp\ldconv_libcrypto_a_99560c9c37f156ab8.lib(ocsp_vfy.obj)
0001:000957d0  _OCSP_basic_verify
0001:00096030* _OCSP_resp_get0_signer
0001:000961b0* _OCSP_request_verify
Module: U:\tmp\ldconv_libcrypto_a_99560c9c37f156ab8.lib(ocsp_prn.obj)
0001:00096650  _OCSP_response_status_str
0001:000966b0  _OCSP_cert_status_str
0001:000966f0  _OCSP_crl_reason_str
0001:000967f0* _OCSP_REQUEST_print
0001:00096b20* _OCSP_RESPONSE_print
Module: U:\tmp\ldconv_libcrypto_a_99560c9c37f156ab8.lib(a_strex.obj)
0001:00098ff0  _X509_NAME_print_ex
0001:00099030* _X509_NAME_print_ex_fp
0001:000990b0  _ASN1_STRING_print_ex
0001:00099530* _ASN1_STRING_print_ex_fp
0001:000999f0  _ASN1_STRING_to_UTF8
Module: U:\tmp\ldconv_libcrypto_a_99560c9c37f156ab8.lib(x509_txt.obj)
0001:00099be0  _X509_verify_cert_error_string
Module: U:\tmp\ldconv_libcrypto_a_99560c9c37f156ab8.lib(v3_utl.obj)
0001:0009aef0  _X509V3_conf_free
0001:0009b800  _X509V3_add_value
0001:0009ba10  _X509V3_add_value_uchar
0001:0009bc20  _X509V3_add_value_bool
0001:0009be40* _X509V3_add_value_bool_nf
0001:0009c050  _i2s_ASN1_ENUMERATED
0001:0009c100  _i2s_ASN1_INTEGER
0001:0009c1b0  _s2i_ASN1_INTEGER
0001:0009c3d0  _X509V3_add_value_int
0001:0009c4e0  _X509V3_get_value_bool
0001:0009c6b0  _X509V3_get_value_int
0001:0009c910  _X509V3_parse_list
0001:0009cbf0  _name_cmp
0001:0009cc40* _X509_get1_email
0001:0009cca0  _X509_get1_ocsp
0001:0009cd50* _X509_REQ_get1_email
0001:0009cdc0  _X509_email_free
0001:0009cde0  _X509_check_host
0001:0009ceb0  _X509_check_email
0001:0009cf70  _X509_check_ip
0001:0009cfb0  _X509_check_ip_asc
0001:0009d250  _a2i_IPADDRESS
0001:0009d4d0  _a2i_ipadd
0001:0009d720  _a2i_IPADDRESS_NC
0001:0009d840  _X509V3_NAME_from_section
Module: U:\tmp\ldconv_libcrypto_a_99560c9c37f156ab8.lib(x509_lu.obj)
0001:0009dac0* _X509_OBJECT_free
0001:0009db20* _X509_LOOKUP_new
0001:0009dbc0* _X509_LOOKUP_free
0001:0009dc00  _X509_STORE_lock
0001:0009dc10  _X509_STORE_unlock
0001:0009dc20* _X509_LOOKUP_init
0001:0009dc50* _X509_LOOKUP_shutdown
0001:0009dc80  _X509_LOOKUP_ctrl
0001:0009dcb0* _X509_LOOKUP_by_subject
0001:0009dce0* _X509_LOOKUP_by_issuer_serial
0001:0009dd00* _X509_LOOKUP_by_fingerprint
0001:0009dd20* _X509_LOOKUP_by_alias
0001:0009dd40* _X509_LOOKUP_set_method_data
0001:0009dd60* _X509_LOOKUP_get_method_data
0001:0009dd70* _X509_LOOKUP_get_store
0001:0009dd80  _X509_STORE_new
0001:0009df20  _X509_STORE_free
0001:0009e030  _X509_STORE_up_ref
0001:0009e050  _X509_STORE_add_lookup
0001:0009e1e0* _X509_STORE_CTX_get_by_subject
0001:0009e350* _X509_STORE_CTX_get_obj_by_subject
0001:0009e440* _X509_OBJECT_up_ref_count
0001:0009e480* _X509_OBJECT_get0_X509
0001:0009e4a0* _X509_OBJECT_get0_X509_CRL
0001:0009e4c0* _X509_OBJECT_get_type
0001:0009e4d0* _X509_OBJECT_new
0001:0009e540* _X509_OBJECT_set1_X509
0001:0009e5b0* _X509_OBJECT_set1_X509_CRL
0001:0009e620* _X509_OBJECT_idx_by_subject
0001:0009e640* _X509_OBJECT_retrieve_by_subject
0001:0009e680* _X509_STORE_get0_objects
0001:0009e690  _X509_STORE_CTX_get1_certs
0001:0009e900  _X509_STORE_CTX_get1_crls
0001:0009eb60* _X509_OBJECT_retrieve_match
0001:0009ec80  _X509_STORE_add_crl
0001:0009ee30  _X509_STORE_add_cert
0001:0009efe0  _X509_STORE_CTX_get1_issuer
0001:0009f310  _X509_STORE_set_flags
0001:0009f320* _X509_STORE_set_depth
0001:0009f350* _X509_STORE_set_purpose
0001:0009f360* _X509_STORE_set_trust
0001:0009f370* _X509_STORE_set1_param
0001:0009f380* _X509_STORE_get0_param
0001:0009f390* _X509_STORE_set_verify
0001:0009f3a0* _X509_STORE_get_verify
0001:0009f3b0* _X509_STORE_set_verify_cb
0001:0009f3c0* _X509_STORE_get_verify_cb
0001:0009f3d0* _X509_STORE_set_get_issuer
0001:0009f3e0* _X509_STORE_get_get_issuer
0001:0009f3f0* _X509_STORE_set_check_issued
0001:0009f400* _X509_STORE_get_check_issued
0001:0009f410* _X509_STORE_set_check_revocation
0001:0009f420* _X509_STORE_get_check_revocation
0001:0009f430* _X509_STORE_set_get_crl
0001:0009f440* _X509_STORE_get_get_crl
0001:0009f450* _X509_STORE_set_check_crl
0001:0009f460* _X509_STORE_get_check_crl
0001:0009f470* _X509_STORE_set_cert_crl
0001:0009f480* _X509_STORE_get_cert_crl
0001:0009f490* _X509_STORE_set_check_policy
0001:0009f4a0* _X509_STORE_get_check_policy
0001:0009f4b0* _X509_STORE_set_lookup_certs
0001:0009f4c0* _X509_STORE_get_lookup_certs
0001:0009f4d0* _X509_STORE_set_lookup_crls
0001:0009f4e0* _X509_STORE_get_lookup_crls
0001:0009f4f0* _X509_STORE_set_cleanup
0001:0009f500* _X509_STORE_get_cleanup
0001:0009f510* _X509_STORE_set_ex_data
0001:0009f520* _X509_STORE_get_ex_data
0001:0009f530* _X509_STORE_CTX_get0_store
Module: U:\tmp\ldconv_libcrypto_a_99560c9c37f156ab8.lib(x_pubkey.obj)
0001:000a0510  _X509_PUBKEY_it
0001:0009f860* _d2i_X509_PUBKEY
0001:0009f890  _i2d_X509_PUBKEY
0001:0009f8c0* _X509_PUBKEY_new
0001:0009f8e0  _X509_PUBKEY_free
0001:0009f900  _X509_PUBKEY_set
0001:0009fa30  _X509_PUBKEY_get0
0001:0009fac0  _X509_PUBKEY_get
0001:0009fb80  _d2i_PUBKEY
0001:0009fd00  _i2d_PUBKEY
0001:0009fd70  _d2i_RSA_PUBKEY
0001:0009fee0  _i2d_RSA_PUBKEY
0001:0009ffb0  _d2i_DSA_PUBKEY
0001:000a0120  _i2d_DSA_PUBKEY
0001:000a01f0  _d2i_EC_PUBKEY
0001:000a0360  _i2d_EC_PUBKEY
0001:000a0430  _X509_PUBKEY_set0_param
0001:000a04b0  _X509_PUBKEY_get0_param
0001:000a04f0  _X509_get0_pubkey_bitstr
Module: U:\tmp\ldconv_libcrypto_a_99560c9c37f156ab8.lib(by_file.obj)
0001:000a0720  _X509_LOOKUP_file
0001:000a0730  _X509_load_cert_file
0001:000a0a10  _X509_load_crl_file
0001:000a0c00* _X509_load_cert_crl_file
Module: U:\tmp\ldconv_libcrypto_a_99560c9c37f156ab8.lib(by_dir.obj)
0001:000a17c0  _X509_LOOKUP_hash_dir
Module: U:\usr\lib\libc_dll.lib(accept.obj)
0001:000a17f0  _accept
Module: U:\usr\lib\libc_dll.lib(socketpair.obj)
0001:000a1970  _socketpair
Module: U:\tmp\ldconv_libcrypto_a_99560c9c37f156ab8.lib(bn_lib.obj)
0001:000a1c10* _BN_set_params
0001:000a1c80* _BN_get_params
0001:000a1cd0  _BN_value_one
0001:000a1ce0  _BN_num_bits_word
0001:000a1d70  _BN_num_bits
0001:000a1ed0  _BN_clear_free
0001:000a1f80  _BN_free
0001:000a2010  _bn_init
0001:000a2050  _BN_new
0001:000a20c0  _BN_secure_new
0001:000a2130  _bn_expand2
0001:000a22e0  _BN_dup
0001:000a2460  _BN_copy
0001:000a24e0* _BN_swap
0001:000a2570* _BN_clear
0001:000a25b0  _BN_get_word
0001:000a25e0  _BN_set_word
0001:000a2780  _BN_bin2bn
0001:000a2980  _BN_bn2binpad
0001:000a2ac0  _BN_bn2bin
0001:000a2b70* _BN_lebin2bn
0001:000a2d80* _BN_bn2lebinpad
0001:000a2ed0  _BN_ucmp
0001:000a2f20  _BN_cmp
0001:000a2fc0  _BN_set_bit
0001:000a3080  _BN_clear_bit
0001:000a30e0  _BN_is_bit_set
0001:000a3110  _BN_mask_bits
0001:000a3190  _BN_set_negative
0001:000a31b0  _bn_cmp_words
0001:000a3230  _bn_cmp_part_words
0001:000a3310  _BN_consttime_swap
0001:000a33a0  _BN_security_bits
0001:000a3430* _BN_zero_ex
0001:000a3450  _BN_abs_is_word
0001:000a3480  _BN_is_zero
0001:000a3490  _BN_is_one
0001:000a34c0  _BN_is_word
0001:000a3500  _BN_is_odd
0001:000a3520  _BN_is_negative
0001:000a3530  _BN_to_montgomery
0001:000a3570  _BN_with_flags
0001:000a35b0  _BN_GENCB_new
0001:000a3620  _BN_GENCB_free
0001:000a3650  _BN_set_flags
0001:000a3660  _BN_get_flags
0001:000a3670* _BN_GENCB_set_old
0001:000a3690  _BN_GENCB_set
0001:000a36b0  _BN_GENCB_get_arg
0001:000a36c0  _bn_wexpand
0001:000a3870  _bn_correct_top
Module: U:\tmp\ldconv_libcrypto_a_99560c9c37f156ab8.lib(dh_gen.obj)
0001:000a38f0  _DH_generate_parameters_ex
Module: U:\tmp\ldconv_libgcc_a_99560c9c382191438.lib(__main.obj)
0001:000a3b40* ___do_global_dtors
0001:000a3b45* ___do_global_ctors
0001:000a3b5e  ___main
Module: U:\tmp\ldconv_libcrypto_a_99560c9c37f156ab8.lib(pem_lib.obj)
0001:000a3d40  _PEM_def_callback
0001:000a3e50  _PEM_proc_type
0001:000a3ed0  _PEM_dek_info
0001:000a3f70  _PEM_ASN1_read
0001:000a4020  _PEM_do_header
0001:000a42b0  _PEM_get_EVP_CIPHER_INFO
0001:000a46b0  _PEM_write_bio
0001:000a49c0  _PEM_ASN1_write_bio
0001:000a4f30  _PEM_ASN1_write
0001:000a5010* _PEM_write
0001:000a50c0  _PEM_read_bio_ex
0001:000a5cf0* _PEM_read
0001:000a65b0  _PEM_bytes_read_bio
0001:000a65f0  _PEM_bytes_read_bio_secmem
0001:000a6630  _PEM_read_bio
0001:000a6670  _pem_check_suffix
Module: U:\tmp\ldconv_libcrypto_a_99560c9c37f156ab8.lib(ui_openssl.obj)
0001:000a6f30  _UI_OpenSSL
0001:000a6f40* _UI_set_default_method
0001:000a6f50  _UI_get_default_method
Module: U:\tmp\ldconv_libcrypto_a_99560c9c37f156ab8.lib(mem_clr.obj)
0001:000a6f80  _OPENSSL_cleanse
Module: U:\tmp\ldconv_libcrypto_a_99560c9c37f156ab8.lib(rand_unix.obj)
0001:000a6fb0  _rand_pool_init
0001:000a6fc0  _rand_pool_acquire_entropy
0001:000a7070  _rand_pool_cleanup
0001:000a7080  _rand_pool_keep_random_devices_open
0001:000a7090  _rand_pool_add_nonce_data
0001:000a7110  _rand_pool_add_additional_data
0001:000a71a0* _clock_gettime
Module: U:\tmp\ldconv_libcrypto_a_99560c9c37f156ab8.lib(mem_sec.obj)
0001:000a7ed0* _CRYPTO_secure_malloc_init
0001:000a82a0  _CRYPTO_secure_malloc_done
0001:000a8370* _CRYPTO_secure_malloc_initialized
0001:000a84d0  _CRYPTO_secure_malloc
0001:000a8930  _CRYPTO_secure_zalloc
0001:000a8950  _CRYPTO_secure_free
0001:000a8a20  _CRYPTO_secure_clear_free
0001:000a8b00  _CRYPTO_secure_allocated
0001:000a8b60* _CRYPTO_secure_used
0001:000a8b70* _CRYPTO_secure_actual_size
Module: U:\tmp\ldconv_libcrypto_a_99560c9c37f156ab8.lib(drbg_lib.obj)
0001:000a8fe0* _RAND_DRBG_set
0001:000a9140* _RAND_DRBG_set_defaults
0001:000a91f0* _RAND_DRBG_new
0001:000a9540* _RAND_DRBG_secure_new
0001:000a98a0* _RAND_DRBG_free
0001:000a9940* _RAND_DRBG_instantiate
0001:000a9c70* _RAND_DRBG_uninstantiate
0001:000a9dd0* _RAND_DRBG_reseed
0001:000aa820  _rand_drbg_restart
0001:000aaaf0  _RAND_DRBG_generate
0001:000aadd0  _RAND_DRBG_bytes
0001:000ab160* _RAND_DRBG_set_callbacks
0001:000ab1a0* _RAND_DRBG_set_reseed_interval
0001:000ab1c0* _RAND_DRBG_set_reseed_time_interval
0001:000ab1e0* _RAND_DRBG_set_reseed_defaults
0001:000ab240  _rand_drbg_lock
0001:000ab260  _rand_drbg_unlock
0001:000ab280* _rand_drbg_enable_locking
0001:000ab6c0* _RAND_DRBG_set_ex_data
0001:000ab6d0* _RAND_DRBG_get_ex_data
0001:000ab6e0  _rand_drbg_cleanup_int
0001:000ab7b0  _drbg_delete_thread_state
0001:000ab920* _rand_drbg_seedlen
0001:000ab970  _RAND_DRBG_get0_master
0001:000ab9b0* _RAND_DRBG_get0_public
0001:000abb30  _RAND_DRBG_get0_private
0001:000abcb0  _RAND_OpenSSL
0002:00000b70  _rand_meth
Module: U:\tmp\ldconv_libcrypto_a_99560c9c37f156ab8.lib(tb_rand.obj)
0001:000abd00* _ENGINE_unregister_RAND
0001:000abd20  _ENGINE_register_RAND
0001:000abd80* _ENGINE_register_all_RAND
0001:000abde0  _ENGINE_set_default_RAND
0001:000abe40  _ENGINE_get_default_RAND
0001:000abe60  _ENGINE_get_RAND
0001:000abe70  _ENGINE_set_RAND
Module: U:\tmp\ldconv_libcrypto_a_99560c9c37f156ab8.lib(lhash.obj)
0001:000abf20  _OPENSSL_LH_strhash
0001:000abf90  _OPENSSL_LH_new
0001:000ac070  _OPENSSL_LH_free
0001:000ac110  _OPENSSL_LH_insert
0001:000ac2d0  _OPENSSL_LH_delete
0001:000ac430  _OPENSSL_LH_retrieve
0001:000ac470  _OPENSSL_LH_doall
0001:000ac4c0  _OPENSSL_LH_doall_arg
0001:000ac530  _openssl_lh_strcasehash
0001:000ac5a0  _OPENSSL_LH_num_items
0001:000ac5b0  _OPENSSL_LH_get_down_load
0001:000ac5c0  _OPENSSL_LH_set_down_load
0001:000ac5d0  _OPENSSL_LH_error
Module: U:\tmp\ldconv_libcrypto_a_99560c9c37f156ab8.lib(x509_set.obj)
0001:000ac5e0* _X509_set_version
0001:000ac650* _X509_set_serialNumber
0001:000ac690  _X509_set_issuer_name
0001:000ac6b0* _X509_set_subject_name
0001:000ac6d0  _x509_set1_time
0001:000ac710* _X509_set1_notBefore
0001:000ac760* _X509_set1_notAfter
0001:000ac7b0* _X509_set_pubkey
0001:000ac7d0  _X509_up_ref
0001:000ac7f0  _X509_get_version
0001:000ac800  _X509_get0_notBefore
0001:000ac810  _X509_get0_notAfter
0001:000ac820* _X509_getm_notBefore
0001:000ac830* _X509_getm_notAfter
0001:000ac840* _X509_get_signature_type
0001:000ac860  _X509_get_X509_PUBKEY
0001:000ac870  _X509_get0_extensions
0001:000ac880  _X509_get0_uids
0001:000ac8b0  _X509_get0_tbs_sigalg
0001:000ac8c0* _X509_SIG_INFO_get
0001:000ac910  _X509_SIG_INFO_set
0001:000ac930  _X509_get_signature_info
0001:000ac9a0  _x509_init_sig_info
Module: U:\tmp\ldconv_libssl_a_99560c9c37e1aece0.lib(t1_lib.obj)
0001:000ad5d0  _tls1_default_timeout
0001:000ad5e0  _tls1_new
0001:000ad620  _tls1_free
0001:000ad660  _tls1_clear
0001:000ad6a0  _tls1_group_id_lookup
0001:000ad6d0  _tls1_get_supported_groups
0001:000ad780  _tls_curve_allowed
0001:000ad7f0  _tls1_shared_group
0001:000ad810  _tls1_set_groups
0001:000ad950  _tls1_set_groups_list
0001:000ad9d0  _tls1_check_group_id
0001:000adcd0  _tls1_get_formatlist
0001:000add20  _tls1_check_ec_tmp_key
0001:000addb0  _tls1_lookup_md
0001:000ade00  _tls12_get_psigalgs
0001:000adeb0  _tls_check_sigalg_curve
0001:000adf40  _tls12_check_peer_sigalg
0001:000ae540* _SSL_get_peer_signature_type_nid
0001:000ae570* _SSL_get_signature_type_nid
0001:000ae5a0  _ssl_cipher_disabled
0001:000aeac0  _tls1_set_peer_legacy_sigalg
0001:000aeb10  _tls_use_ticket
0001:000aeb50  _tls_decrypt_ticket
0001:000af270  _tls_get_ticket_from_client
0001:000af330  _ssl_set_sig_mask
0001:000af490  _ssl_set_client_disabled
0001:000af550  _tls12_copy_sigalgs
0001:000af6a0  _tls1_save_u16
0001:000af7e0  _tls1_save_sigalgs
0001:000afa60  _tls1_process_sigalgs
0001:000aff70  _tls1_set_server_sigalgs
0001:000b01a0* _SSL_get_sigalgs
0001:000b02c0* _SSL_get_shared_sigalgs
0001:000b0350  _tls1_set_sigalgs_list
0001:000b04a0* _tls1_set_raw_sigalgs
0001:000b05b0  _tls1_set_sigalgs
0001:000b0730  _tls1_check_chain
0001:000b0fe0  _tls1_set_cert_validity
0001:000b1160* _SSL_check_chain
0001:000b11a0  _ssl_get_auto_dh
0001:000b1350  _ssl_security_cert
0001:000b1550  _ssl_security_cert_chain
0001:000b1750  _tls_choose_sigalg
0001:000b1d30* _SSL_CTX_set_tlsext_max_fragment_length
0001:000b1d90* _SSL_set_tlsext_max_fragment_length
0001:000b1df0* _SSL_SESSION_get_max_fragment_length
0001:000b24d0  _TLSv1_3_enc_data
0001:000b2510  _TLSv1_2_enc_data
0001:000b2550  _TLSv1_1_enc_data
0001:000b2590  _TLSv1_enc_data
Module: U:\tmp\ldconv_libssl_a_99560c9c37e1aece0.lib(extensions.obj)
0001:000b36f0  _tls_validate_all_contexts
0001:000b37e0  _extension_is_relevant
0001:000b38d0  _tls_collect_extensions
0001:000b3d70  _tls_parse_extension
0001:000b3f70  _tls_parse_all_extensions
0001:000b40e0  _should_add_extension
0001:000b4220  _tls_construct_extensions
0001:000b45a0  _tls_psk_do_binder
Module: U:\tmp\ldconv_libcrypto_a_99560c9c37f156ab8.lib(pem_oth.obj)
0001:000b4ff0  _PEM_ASN1_read_bio
Module: U:\tmp\ldconv_libcrypto_a_99560c9c37f156ab8.lib(async.obj)
0001:000b50d0* _async_get_ctx
0001:000b5100* _async_start_func
0001:000b5160* _ASYNC_pause_job
0001:000b51e0  _async_init
0001:000b5240  _async_deinit
0001:000b5260* _ASYNC_init_thread
0001:000b5540  _ASYNC_start_job
0001:000b59f0  _async_delete_thread_state
0001:000b5af0* _ASYNC_cleanup_thread
0001:000b5b30  _ASYNC_get_current_job
0001:000b5b80* _ASYNC_get_wait_ctx
0001:000b5b90* _ASYNC_block_pause
0001:000b5be0* _ASYNC_unblock_pause
Module: U:\tmp\ldconv_libcrypto_a_99560c9c37f156ab8.lib(async_wait.obj)
0001:000b5c60  _ASYNC_WAIT_CTX_new
0001:000b5c90  _ASYNC_WAIT_CTX_free
0001:000b5d20* _ASYNC_WAIT_CTX_set_wait_fd
0001:000b5db0* _ASYNC_WAIT_CTX_get_fd
0001:000b5e00  _ASYNC_WAIT_CTX_get_all_fds
0001:000b5e50  _ASYNC_WAIT_CTX_get_changed_fds
0001:000b5ef0* _ASYNC_WAIT_CTX_clear_fd
0001:000b5f90* _async_wait_ctx_reset_counts
Module: U:\tmp\ldconv_libcrypto_a_99560c9c37f156ab8.lib(x_name.obj)
0001:000b6040  _X509_NAME_ENTRY_free
0001:000b7100  _X509_NAME_ENTRY_it
0001:000b7020  _X509_NAME_it
0001:000b6c30* _d2i_X509_NAME_ENTRY
0001:000b6c60* _i2d_X509_NAME_ENTRY
0001:000b6c90  _X509_NAME_ENTRY_new
0001:000b6cb0  _X509_NAME_ENTRY_dup
0001:000b6cd0  _d2i_X509_NAME
0001:000b6d00  _i2d_X509_NAME
0001:000b6d30  _X509_NAME_new
0001:000b6d50  _X509_NAME_free
0001:000b6d70  _X509_NAME_dup
0001:000b6d90  _X509_NAME_set
0001:000b6e00  _X509_NAME_print
0001:000b6fc0* _X509_NAME_get0_der
Module: U:\tmp\ldconv_libcrypto_a_99560c9c37f156ab8.lib(ct_sct.obj)
0001:000b71a0  _SCT_free
0001:000b7240  _SCT_new
0001:000b72b0  _SCT_LIST_free
0001:000b72d0  _SCT_set_version
0001:000b7330  _SCT_set_log_entry_type
0001:000b7390  _SCT_set0_log_id
0001:000b7420* _SCT_set1_log_id
0001:000b7530  _SCT_set_timestamp
0001:000b7550* _SCT_set_signature_nid
0001:000b75e0  _SCT_set0_extensions
0001:000b7620* _SCT_set1_extensions
0001:000b76f0* _SCT_set0_signature
0001:000b7730  _SCT_set1_signature
0001:000b7800* _SCT_get_version
0001:000b7810* _SCT_get_log_entry_type
0001:000b7820* _SCT_get0_log_id
0001:000b7840* _SCT_get_timestamp
0001:000b7850  _SCT_get_signature_nid
0001:000b7890* _SCT_get0_extensions
0001:000b78b0* _SCT_get0_signature
0001:000b78d0  _SCT_is_complete
0001:000b7930  _SCT_signature_is_complete
0001:000b7970* _SCT_get_source
0001:000b7980  _SCT_set_source
0001:000b79d0  _SCT_get_validation_status
0001:000b79e0* _SCT_validate
0001:000b7b90  _SCT_LIST_validate
Module: U:\tmp\ldconv_libcrypto_a_99560c9c37f156ab8.lib(x509_vpm.obj)
0001:000b7eb0  _X509_VERIFY_PARAM_free
0001:000b7f60  _X509_VERIFY_PARAM_new
0001:000b7fe0* _X509_VERIFY_PARAM_set1_name
0001:000b8030  _X509_VERIFY_PARAM_set_flags
0001:000b8060* _X509_VERIFY_PARAM_clear_flags
0001:000b8080* _X509_VERIFY_PARAM_get_flags
0001:000b8090* _X509_VERIFY_PARAM_get_inh_flags
0001:000b80a0* _X509_VERIFY_PARAM_set_inh_flags
0001:000b80c0  _X509_VERIFY_PARAM_set_purpose
0001:000b80d0  _X509_VERIFY_PARAM_set_trust
0001:000b80e0  _X509_VERIFY_PARAM_set_depth
0001:000b80f0  _X509_VERIFY_PARAM_set_auth_level
0001:000b8100* _X509_VERIFY_PARAM_get_time
0001:000b8110  _X509_VERIFY_PARAM_set_time
0001:000b8120* _X509_VERIFY_PARAM_add0_policy
0001:000b8160* _X509_VERIFY_PARAM_set1_policies
0001:000b8230  _X509_VERIFY_PARAM_inherit
0001:000b8700  _X509_VERIFY_PARAM_set1
0001:000b8ac0  _X509_VERIFY_PARAM_set1_host
0001:000b8cc0  _X509_VERIFY_PARAM_add1_host
0001:000b8e40  _X509_VERIFY_PARAM_set_hostflags
0001:000b8e50* _X509_VERIFY_PARAM_get_hostflags
0001:000b8e60  _X509_VERIFY_PARAM_get0_peername
0001:000b8e70  _X509_VERIFY_PARAM_move_peername
0001:000b8ef0* _X509_VERIFY_PARAM_set1_email
0001:000b8f80* _X509_VERIFY_PARAM_set1_ip
0001:000b9030* _X509_VERIFY_PARAM_set1_ip_asc
0001:000b90c0  _X509_VERIFY_PARAM_get_depth
0001:000b90d0* _X509_VERIFY_PARAM_get_auth_level
0001:000b90e0* _X509_VERIFY_PARAM_get0_name
0001:000b90f0* _X509_VERIFY_PARAM_add0_table
0001:000b9210* _X509_VERIFY_PARAM_get_count
0001:000b9240* _X509_VERIFY_PARAM_get0
0001:000b9280  _X509_VERIFY_PARAM_lookup
0001:000b9300* _X509_VERIFY_PARAM_table_cleanup
Module: U:\tmp\ldconv_libcrypto_a_99560c9c37f156ab8.lib(ct_log.obj)
0001:000b96b0* _CTLOG_free
0001:000b9700  _CTLOG_STORE_new
0001:000b9790  _CTLOG_STORE_free
0001:000b97e0  _CTLOG_STORE_load_file
0001:000b99b0  _CTLOG_STORE_load_default_file
0001:000b99e0  _CTLOG_new
0001:000b9b90  _CTLOG_get0_name
0001:000b9ba0* _CTLOG_get0_log_id
0001:000b9bc0  _CTLOG_get0_public_key
0001:000b9bd0  _CTLOG_STORE_get0_log_by_id
Module: U:\tmp\ldconv_libssl_a_99560c9c37e1aece0.lib(tls_srp.obj)
0001:000b9c40  _SSL_CTX_SRP_CTX_free
0001:000b9d50  _SSL_SRP_CTX_free
0001:000b9e60  _SSL_SRP_CTX_init
0001:000ba1c0  _SSL_CTX_SRP_CTX_init
0001:000ba210  _SSL_srp_server_param_with_username
0001:000ba320* _SSL_set_srp_server_param_pw
0001:000ba3f0* _SSL_set_srp_server_param
0001:000ba610  _srp_generate_server_master_secret
0001:000ba770  _srp_generate_client_master_secret
0001:000baa20  _srp_verify_server_param
0001:000bab90  _SRP_Calc_A_param
0001:000bac20* _SSL_get_srp_g
0001:000bac40* _SSL_get_srp_N
0001:000bac60* _SSL_get_srp_username
0001:000bac80* _SSL_get_srp_userinfo
0001:000baca0* _SSL_CTX_set_srp_username
0001:000bacd0* _SSL_CTX_set_srp_password
0001:000bad00* _SSL_CTX_set_srp_strength
0001:000bad30* _SSL_CTX_set_srp_verify_param_callback
0001:000bad60* _SSL_CTX_set_srp_cb_arg
0001:000bad90* _SSL_CTX_set_srp_username_callback
0001:000badc0* _SSL_CTX_set_srp_client_pwd_callback
Module: U:\tmp\ldconv_libcrypto_a_99560c9c37f156ab8.lib(buffer.obj)
0001:000bae10  _BUF_MEM_new_ex
0001:000bae80  _BUF_MEM_new
0001:000baef0  _BUF_MEM_free
0001:000baf70  _BUF_MEM_grow
0001:000bb0f0  _BUF_MEM_grow_clean
0001:000bb2a0  _BUF_reverse
Module: U:\tmp\ldconv_libcrypto_a_99560c9c37f156ab8.lib(digest.obj)
0001:000bb320  _EVP_MD_CTX_reset
0001:000bb400  _EVP_MD_CTX_new
0001:000bb430  _EVP_MD_CTX_free
0001:000bb520  _EVP_DigestInit_ex
0001:000bb7d0  _EVP_DigestInit
0001:000bb8c0  _EVP_DigestUpdate
0001:000bb920  _EVP_DigestFinal
0001:000bb9b0  _EVP_DigestFinal_ex
0001:000bba40  _EVP_DigestFinalXOF
0001:000bbb00  _EVP_MD_CTX_copy
0001:000bbd20  _EVP_MD_CTX_copy_ex
0001:000bbf40  _EVP_Digest
0001:000bc080  _EVP_MD_CTX_ctrl
Module: U:\tmp\ldconv_libcrypto_a_99560c9c37f156ab8.lib(x_exten.obj)
0001:000bc0c0* _d2i_X509_EXTENSION
0001:000bc238  _X509_EXTENSION_it
0001:000bc0f0* _i2d_X509_EXTENSION
0001:000bc120  _X509_EXTENSION_new
0001:000bc140  _X509_EXTENSION_free
0001:000bc160  _d2i_X509_EXTENSIONS
0001:000bc1ec  _X509_EXTENSIONS_it
0001:000bc190  _i2d_X509_EXTENSIONS
0001:000bc1c0  _X509_EXTENSION_dup
Module: U:\tmp\ldconv_libssl_a_99560c9c37e1aece0.lib(rec_layer_s3.obj)
0001:000bc2c0  _RECORD_LAYER_init
0001:000bc2f0  _RECORD_LAYER_clear
0001:000bc3e0  _RECORD_LAYER_release
0001:000bc430  _RECORD_LAYER_read_pending
0001:000bc440  _RECORD_LAYER_processed_read_pending
0001:000bc480  _RECORD_LAYER_write_pending
0001:000bc4a0  _RECORD_LAYER_reset_read_sequence
0001:000bc4c0  _RECORD_LAYER_reset_write_sequence
0001:000bc4e0  _ssl3_pending
0001:000bc530* _SSL_CTX_set_default_read_buffer_len
0001:000bc540  _SSL_set_default_read_buffer_len
0001:000bc560* _SSL_rstate_string_long
0001:000bc590* _SSL_rstate_string
0001:000bc5d0  _ssl3_read_n
0001:000bc990  _ssl3_write_pending
0001:000bcb60  _do_ssl3_write
0001:000bda90  _ssl3_write_bytes
0001:000bdfc0  _ssl3_read_bytes
0001:000bed10  _ssl3_record_sequence_update
0001:000bed50  _RECORD_LAYER_is_sslv2_record
0001:000bed70  _RECORD_LAYER_get_rrec_length
Module: U:\tmp\ldconv_libcrypto_a_99560c9c37f156ab8.lib(names.obj)
0001:000bee80  _EVP_add_cipher
0001:000beee0  _EVP_add_digest
0001:000bef90  _EVP_get_cipherbyname
0001:000befd0  _EVP_get_digestbyname
0001:000bf010  _evp_cleanup_int
0001:000bf050* _EVP_CIPHER_do_all
0001:000bf0a0* _EVP_CIPHER_do_all_sorted
0001:000bf0f0* _EVP_MD_do_all
0001:000bf140* _EVP_MD_do_all_sorted
Module: U:\tmp\ldconv_libssl_a_99560c9c37e1aece0.lib(statem_lib.obj)
0001:000bf540  _ssl3_do_write
0001:000bf660  _tls_close_construct_packet
0001:000bf6c0  _tls_construct_cert_verify
0001:000bfbb0  _tls_process_cert_verify
0001:000c02e0  _tls_construct_finished
0001:000c0510  _tls_construct_key_update
0001:000c0590  _tls_process_key_update
0001:000c06c0  _ssl3_take_mac
0001:000c0730  _tls_process_change_cipher_spec
0001:000c08e0  _tls_construct_change_cipher_spec
0001:000c0950  _ssl3_output_cert_chain
0001:000c0cc0  _tls_finish_handshake
0001:000c1040  _tls_get_message_header
0001:000c12e0  _tls_get_message_body
0001:000c3a70  _hrrrandom
0001:000c1590  _ssl_x509err2alert
0001:000c15d0  _ssl_allow_compression
0001:000c1610  _ssl_version_supported
0001:000c1950  _ssl_check_version_downgrade
0001:000c1b10  _ssl_set_version_bound
0001:000c1ba0  _ssl_choose_server_version
0001:000c2200  _ssl_get_min_max_version
0001:000c24e0  _tls_setup_handshake
0001:000c27a0  _ssl_choose_client_version
0001:000c2b50  _ssl_set_client_hello_version
0001:000c2bc0  _check_in_list
0001:000c2c60  _create_synthetic_message_hash
0001:000c2d90  _parse_ca_names
0001:000c2fd0  _get_ca_names
0001:000c3020  _construct_ca_names
0001:000c3190  _construct_key_exchange_tbs
0001:000c32b0  _tls13_save_handshake_digest_for_pha
0001:000c3390  _tls_process_finished
0001:000c3740  _tls13_restore_handshake_digest_for_pha
Module: U:\tmp\ldconv_libssl_a_99560c9c37e1aece0.lib(extensions_cust.obj)
0001:000c3b40  _custom_ext_find
0001:000c3bd0  _custom_ext_init
0001:000c3c10  _custom_ext_parse
0001:000c3d80  _custom_ext_add
0001:000c3ff0  _custom_exts_copy_flags
0001:000c40a0  _custom_exts_copy
0001:000c4270  _custom_exts_free
0001:000c4310  _SSL_CTX_has_client_custom_ext
0001:000c4370* _SSL_CTX_add_client_custom_ext
0001:000c4690  _SSL_CTX_add_server_custom_ext
0001:000c49b0  _SSL_CTX_add_custom_ext
0001:000c4bf0* _SSL_extension_supported
Module: U:\tmp\ldconv_libssl_a_99560c9c37e1aece0.lib(tls13_enc.obj)
0001:000c4d10  _tls13_hkdf_expand
0001:000c5500* _tls13_derive_key
0001:000c5560* _tls13_derive_iv
0001:000c55c0  _tls13_derive_finishedkey
0001:000c5620  _tls13_generate_secret
0001:000c59e0  _tls13_generate_handshake_secret
0001:000c5d30  _tls13_generate_master_secret
0001:000c5d90  _tls13_final_finish_mac
0001:000c5fc0  _tls13_setup_key_block
0001:000c6140  _tls13_change_cipher_state
0001:000c6b80  _tls13_update_key
0001:000c6ca0  _tls13_alert_code
0001:000c6cc0  _tls13_export_keying_material
0001:000c6e80  _tls13_export_keying_material_early
Module: U:\tmp\ldconv_libssl_a_99560c9c37e1aece0.lib(ssl_mcnf.obj)
0001:000c74e0* _SSL_add_ssl_module
0001:000c74f0* _SSL_config
0001:000c7510* _SSL_CTX_config
0001:000c7530  _ssl_ctx_system_config
Module: U:\tmp\ldconv_libcrypto_a_99560c9c37f156ab8.lib(v3_purp.obj)
0001:000c7d40  _X509_PURPOSE_set
0001:000c7dc0* _X509_PURPOSE_get_count
0001:000c7df0  _X509_PURPOSE_get0
0001:000c7e40* _X509_PURPOSE_get_by_sname
0001:000c7ee0  _X509_PURPOSE_get_by_id
0001:000c7f30* _X509_PURPOSE_add
0001:000c8260* _X509_PURPOSE_cleanup
0001:000c8290* _X509_PURPOSE_get_id
0001:000c82a0* _X509_PURPOSE_get0_name
0001:000c82b0* _X509_PURPOSE_get0_sname
0001:000c82c0  _X509_PURPOSE_get_trust
0001:000c82d0* _X509_supported_extension
0001:000c8330* _X509_set_proxy_flag
0001:000c8340* _X509_set_proxy_pathlen
0001:000c8350  _x509_signing_allowed
0001:000c83b0  _X509_check_akid
0001:000c8e70  _X509_check_purpose
0001:000c8f20  _X509_check_ca
0001:000c8fb0  _x509_likely_issued
0001:000c9050* _X509_check_issued
0001:000c9140  _X509_get_extension_flags
0001:000c9160  _X509_get_key_usage
0001:000c91a0  _X509_get_extended_key_usage
0001:000c91e0  _X509_get0_subject_key_id
0001:000c9210* _X509_get0_authority_key_id
0001:000c9250* _X509_get0_authority_issuer
0001:000c9290* _X509_get0_authority_serial
0001:000c92d0* _X509_get_pathlen
0001:000c9300* _X509_get_proxy_pathlen
Module: U:\tmp\ldconv_libcrypto_a_99560c9c37f156ab8.lib(bf_buff.obj)
0001:000ca1b0  _BIO_f_buffer
Module: U:\tmp\ldconv_libcrypto_a_99560c9c37f156ab8.lib(x509_d2.obj)
0001:000ca210  _X509_STORE_set_default_paths
0001:000ca2b0  _X509_STORE_load_locations
Module: U:\tmp\ldconv_libcrypto_a_99560c9c37f156ab8.lib(ct_oct.obj)
0001:000ca390  _o2i_SCT_signature
0001:000ca4c0* _o2i_SCT
0001:000ca760* _i2o_SCT_signature
0001:000ca8c0* _i2o_SCT
0001:000caae0  _o2i_SCT_LIST
0001:000cacb0* _i2o_SCT_LIST
0001:000cb0c0  _d2i_SCT_LIST
0001:000cb150  _i2d_SCT_LIST
Module: U:\tmp\ldconv_libcrypto_a_99560c9c37f156ab8.lib(x509_ext.obj)
0001:000cb1c0  _X509_CRL_get_ext_count
0001:000cb1d0  _X509_CRL_get_ext_by_NID
0001:000cb1e0* _X509_CRL_get_ext_by_OBJ
0001:000cb1f0* _X509_CRL_get_ext_by_critical
0001:000cb200  _X509_CRL_get_ext
0001:000cb210* _X509_CRL_delete_ext
0001:000cb220  _X509_CRL_get_ext_d2i
0001:000cb230  _X509_CRL_add1_ext_i2d
0001:000cb240  _X509_CRL_add_ext
0001:000cb270  _X509_get_ext_count
0001:000cb280  _X509_get_ext_by_NID
0001:000cb290* _X509_get_ext_by_OBJ
0001:000cb2a0* _X509_get_ext_by_critical
0001:000cb2b0  _X509_get_ext
0001:000cb2c0  _X509_delete_ext
0001:000cb2d0* _X509_add_ext
0001:000cb300  _X509_get_ext_d2i
0001:000cb310* _X509_add1_ext_i2d
0001:000cb320* _X509_REVOKED_get_ext_count
0001:000cb330* _X509_REVOKED_get_ext_by_NID
0001:000cb340* _X509_REVOKED_get_ext_by_OBJ
0001:000cb350* _X509_REVOKED_get_ext_by_critical
0001:000cb360* _X509_REVOKED_get_ext
0001:000cb370* _X509_REVOKED_delete_ext
0001:000cb380* _X509_REVOKED_add_ext
0001:000cb3b0  _X509_REVOKED_get_ext_d2i
0001:000cb3c0* _X509_REVOKED_add1_ext_i2d
Module: U:\tmp\ldconv_libcrypto_a_99560c9c37f156ab8.lib(ct_policy.obj)
0001:000cb3f0  _CT_POLICY_EVAL_CTX_new
0001:000cb470  _CT_POLICY_EVAL_CTX_free
0001:000cb4b0  _CT_POLICY_EVAL_CTX_set1_cert
0001:000cb4e0  _CT_POLICY_EVAL_CTX_set1_issuer
0001:000cb510  _CT_POLICY_EVAL_CTX_set_shared_CTLOG_STORE
0001:000cb520  _CT_POLICY_EVAL_CTX_set_time
0001:000cb540* _CT_POLICY_EVAL_CTX_get0_cert
0001:000cb550* _CT_POLICY_EVAL_CTX_get0_issuer
0001:000cb560* _CT_POLICY_EVAL_CTX_get0_log_store
0001:000cb570* _CT_POLICY_EVAL_CTX_get_time
Module: U:\tmp\ldconv_libssl_a_99560c9c37e1aece0.lib(ssl3_buffer.obj)
0001:000cb580* _SSL3_BUFFER_set_data
0001:000cb5c0  _SSL3_BUFFER_clear
0001:000cb5f0  _SSL3_BUFFER_release
0001:000cb620  _ssl3_setup_read_buffer
0001:000cb6f0  _ssl3_setup_write_buffer
0001:000cb840  _ssl3_setup_buffers
0001:000cbaa0  _ssl3_release_write_buffer
0001:000cbb10  _ssl3_release_read_buffer
Module: U:\tmp\ldconv_libssl_a_99560c9c37e1aece0.lib(statem_srvr.obj)
0001:000cbbb0* _tls_construct_server_hello
0001:000cc050* _tls_construct_server_key_exchange
0001:000ccc40* _tls_construct_certificate_request
0001:000cd1f0* _tls_construct_server_certificate
0001:000cd2f0* _tls_construct_new_session_ticket
0001:000cdf60* _tls_construct_server_done
0001:000cef10* _tls_construct_cert_status
0001:000cefb0* _dtls_construct_hello_verify_request
0001:000cf0b0* _d2i_GOST_KX_MESSAGE
0001:000d3884* _GOST_KX_MESSAGE_it
0001:000cf0e0* _i2d_GOST_KX_MESSAGE
0001:000cf110* _GOST_KX_MESSAGE_new
0001:000cf130* _GOST_KX_MESSAGE_free
0001:000cf150  _ossl_statem_server_read_transition
0001:000cf600  _send_certificate_request
0001:000cf690  _ossl_statem_server_write_transition
0001:000cfc80  _ossl_statem_server_pre_work
0001:000cff60  _ossl_statem_server_post_work
0001:000d0360  _ossl_statem_server_construct_message
0001:000d0630  _ossl_statem_server_max_message_size
0001:000d0720  _dtls_raw_hello_verify_request
0001:000d0780* _tls_process_client_hello
0001:000d10d0  _tls_handle_alpn
0001:000d1340  _ossl_statem_server_post_process_message
0001:000d1840* _tls_post_process_client_hello
0001:000d1c70* _tls_process_client_key_exchange
0001:000d2ae0* _tls_post_process_client_key_exchange
0001:000d2b90* _tls_process_client_certificate
0001:000d33b0  _tls_construct_cert_status_body
0001:000d3450* _tls_process_next_proto
0001:000d3590* _tls_process_end_of_early_data
0001:000d36c0  _ossl_statem_server_process_message
Module: U:\tmp\ldconv_libcrypto_a_99560c9c37f156ab8.lib(a_int.obj)
0001:000d3ac0  _ASN1_INTEGER_dup
0001:000d3ad0  _ASN1_INTEGER_cmp
0001:000d3b30  _i2c_ASN1_INTEGER
0001:000d3c90  _c2i_ASN1_INTEGER
0001:000d3f00* _d2i_ASN1_UINTEGER
0001:000d41b0* _ASN1_INTEGER_get_int64
0001:000d4480  _ASN1_INTEGER_set_int64
0001:000d4520  _ASN1_INTEGER_get_uint64
0001:000d4750  _ASN1_INTEGER_set_uint64
0001:000d47b0  _ASN1_INTEGER_set
0001:000d4850  _ASN1_INTEGER_get
0001:000d4ae0  _BN_to_ASN1_INTEGER
0001:000d4c40  _ASN1_INTEGER_to_BN
0001:000d4d20* _ASN1_ENUMERATED_get_int64
0001:000d4ff0* _ASN1_ENUMERATED_set_int64
0001:000d5090* _ASN1_ENUMERATED_set
0001:000d5130  _ASN1_ENUMERATED_get
0001:000d5260* _BN_to_ASN1_ENUMERATED
0001:000d53c0  _ASN1_ENUMERATED_to_BN
0001:000d54a0  _c2i_uint64_int
0001:000d5700  _i2c_uint64_int
Module: U:\tmp\ldconv_libcrypto_a_99560c9c37f156ab8.lib(x509_obj.obj)
0001:000d58a0  _X509_NAME_oneline
Module: U:\tmp\ldconv_libcrypto_a_99560c9c37f156ab8.lib(m_md5.obj)
0001:000d5dc0  _EVP_md5
Module: U:\tmp\ldconv_libcrypto_a_99560c9c37f156ab8.lib(x_x509a.obj)
0001:000d5e20  _d2i_X509_CERT_AUX
0001:000d62e0* _X509_CERT_AUX_it
0001:000d5e50  _i2d_X509_CERT_AUX
0001:000d5e80* _X509_CERT_AUX_new
0001:000d5ea0  _X509_CERT_AUX_free
0001:000d5ec0  _X509_trusted
0001:000d5ee0  _X509_alias_set1
0001:000d5fb0  _X509_keyid_set1
0001:000d6080  _X509_alias_get0
0001:000d60b0  _X509_keyid_get0
0001:000d60e0* _X509_add1_trust_object
0001:000d6190* _X509_add1_reject_object
0001:000d6220* _X509_trust_clear
0001:000d6260* _X509_reject_clear
0001:000d62a0  _X509_get0_trust_objects
0001:000d62c0  _X509_get0_reject_objects
Module: U:\tmp\ldconv_libcrypto_a_99560c9c37f156ab8.lib(tasn_typ.obj)
0001:000d63a0  _d2i_ASN1_OCTET_STRING
0001:000d7420  _ASN1_OCTET_STRING_it
0001:000d63d0  _i2d_ASN1_OCTET_STRING
0001:000d6400  _ASN1_OCTET_STRING_new
0001:000d6420  _ASN1_OCTET_STRING_free
0001:000d6430  _d2i_ASN1_INTEGER
0001:000d73f0  _ASN1_INTEGER_it
0001:000d6460  _i2d_ASN1_INTEGER
0001:000d6490  _ASN1_INTEGER_new
0001:000d64b0  _ASN1_INTEGER_free
0001:000d64c0  _d2i_ASN1_ENUMERATED
0001:000d73c4  _ASN1_ENUMERATED_it
0001:000d64f0* _i2d_ASN1_ENUMERATED
0001:000d6520* _ASN1_ENUMERATED_new
0001:000d6540  _ASN1_ENUMERATED_free
0001:000d6550* _d2i_ASN1_BIT_STRING
0001:000d7398  _ASN1_BIT_STRING_it
0001:000d6580* _i2d_ASN1_BIT_STRING
0001:000d65b0  _ASN1_BIT_STRING_new
0001:000d65d0  _ASN1_BIT_STRING_free
0001:000d65e0* _d2i_ASN1_UTF8STRING
0001:000d736c  _ASN1_UTF8STRING_it
0001:000d6610* _i2d_ASN1_UTF8STRING
0001:000d6640  _ASN1_UTF8STRING_new
0001:000d6660  _ASN1_UTF8STRING_free
0001:000d6670* _d2i_ASN1_PRINTABLESTRING
0001:000d7340  _ASN1_PRINTABLESTRING_it
0001:000d66a0* _i2d_ASN1_PRINTABLESTRING
0001:000d66d0* _ASN1_PRINTABLESTRING_new
0001:000d66f0  _ASN1_PRINTABLESTRING_free
0001:000d6700* _d2i_ASN1_T61STRING
0001:000d730c* _ASN1_T61STRING_it
0001:000d6730* _i2d_ASN1_T61STRING
0001:000d6760* _ASN1_T61STRING_new
0001:000d6780* _ASN1_T61STRING_free
0001:000d6790* _d2i_ASN1_IA5STRING
0001:000d72e0  _ASN1_IA5STRING_it
0001:000d67c0* _i2d_ASN1_IA5STRING
0001:000d67f0  _ASN1_IA5STRING_new
0001:000d6810  _ASN1_IA5STRING_free
0001:000d6820* _d2i_ASN1_GENERALSTRING
0001:000d72b4* _ASN1_GENERALSTRING_it
0001:000d6850* _i2d_ASN1_GENERALSTRING
0001:000d6880* _ASN1_GENERALSTRING_new
0001:000d68a0* _ASN1_GENERALSTRING_free
0001:000d68b0* _d2i_ASN1_UTCTIME
0001:000d7284* _ASN1_UTCTIME_it
0001:000d68e0* _i2d_ASN1_UTCTIME
0001:000d6910* _ASN1_UTCTIME_new
0001:000d6930* _ASN1_UTCTIME_free
0001:000d6940* _d2i_ASN1_GENERALIZEDTIME
0001:000d7258  _ASN1_GENERALIZEDTIME_it
0001:000d6970* _i2d_ASN1_GENERALIZEDTIME
0001:000d69a0  _ASN1_GENERALIZEDTIME_new
0001:000d69c0  _ASN1_GENERALIZEDTIME_free
0001:000d69d0* _d2i_ASN1_VISIBLESTRING
0001:000d7224* _ASN1_VISIBLESTRING_it
0001:000d6a00* _i2d_ASN1_VISIBLESTRING
0001:000d6a30* _ASN1_VISIBLESTRING_new
0001:000d6a50* _ASN1_VISIBLESTRING_free
0001:000d6a60* _d2i_ASN1_UNIVERSALSTRING
0001:000d71f4* _ASN1_UNIVERSALSTRING_it
0001:000d6a90* _i2d_ASN1_UNIVERSALSTRING
0001:000d6ac0* _ASN1_UNIVERSALSTRING_new
0001:000d6ae0* _ASN1_UNIVERSALSTRING_free
0001:000d6af0* _d2i_ASN1_BMPSTRING
0001:000d71c0* _ASN1_BMPSTRING_it
0001:000d6b20* _i2d_ASN1_BMPSTRING
0001:000d6b50* _ASN1_BMPSTRING_new
0001:000d6b70* _ASN1_BMPSTRING_free
0001:000d6b80* _d2i_ASN1_NULL
0001:000d7194  _ASN1_NULL_it
0001:000d6bb0* _i2d_ASN1_NULL
0001:000d6be0  _ASN1_NULL_new
0001:000d6c00* _ASN1_NULL_free
0001:000d6c20  _d2i_ASN1_TYPE
0001:000d7144  _ASN1_ANY_it
0001:000d6c50  _i2d_ASN1_TYPE
0001:000d6c80  _ASN1_TYPE_new
0001:000d6ca0  _ASN1_TYPE_free
0001:000d6cc0* _d2i_ASN1_PRINTABLE
0001:000d70f0  _ASN1_PRINTABLE_it
0001:000d6cf0* _i2d_ASN1_PRINTABLE
0001:000d6d20* _ASN1_PRINTABLE_new
0001:000d6d40* _ASN1_PRINTABLE_free
0001:000d6d60* _d2i_DISPLAYTEXT
0001:000d70c4  _DISPLAYTEXT_it
0001:000d6d90* _i2d_DISPLAYTEXT
0001:000d6dc0* _DISPLAYTEXT_new
0001:000d6de0* _DISPLAYTEXT_free
0001:000d6e00* _d2i_DIRECTORYSTRING
0001:000d709c  _DIRECTORYSTRING_it
0001:000d6e30* _i2d_DIRECTORYSTRING
0001:000d6e60* _DIRECTORYSTRING_new
0001:000d6e80* _DIRECTORYSTRING_free
0001:000d6ea0  _d2i_ASN1_SEQUENCE_ANY
0001:000d6fa4* _ASN1_SEQUENCE_ANY_it
0001:000d6ed0  _i2d_ASN1_SEQUENCE_ANY
0001:000d6f00* _d2i_ASN1_SET_ANY
0001:000d6f60* _ASN1_SET_ANY_it
0001:000d6f30  _i2d_ASN1_SET_ANY
0001:000d6fec  _ASN1_OCTET_STRING_NDEF_it
0001:000d7018  _ASN1_FBOOLEAN_it
0001:000d7044* _ASN1_TBOOLEAN_it
0001:000d7070  _ASN1_BOOLEAN_it
0001:000d711c  _ASN1_SEQUENCE_it
0001:000d716c  _ASN1_OBJECT_it
Module: U:\tmp\ldconv_libcrypto_a_99560c9c37f156ab8.lib(v3_akeya.obj)
0001:000d7440* _d2i_AUTHORITY_KEYID
0001:000d74ec  _AUTHORITY_KEYID_it
0001:000d7470* _i2d_AUTHORITY_KEYID
0001:000d74a0  _AUTHORITY_KEYID_new
0001:000d74c0  _AUTHORITY_KEYID_free
Module: U:\tmp\ldconv_libcrypto_a_99560c9c37f156ab8.lib(v3_crld.obj)
0001:000d77d0* _DIST_POINT_free
0001:000d8b5c* _DIST_POINT_it
0001:000d8bcc* _DIST_POINT_NAME_it
0001:000d8a4c* _ISSUING_DIST_POINT_it
0001:000d86b0* _d2i_DIST_POINT_NAME
0001:000d86e0* _i2d_DIST_POINT_NAME
0001:000d8710* _DIST_POINT_NAME_new
0001:000d8730* _DIST_POINT_NAME_free
0001:000d8750* _d2i_DIST_POINT
0001:000d8780* _i2d_DIST_POINT
0001:000d87b0* _DIST_POINT_new
0001:000d87d0* _d2i_CRL_DIST_POINTS
0001:000d8b08* _CRL_DIST_POINTS_it
0001:000d8800* _i2d_CRL_DIST_POINTS
0001:000d8830* _CRL_DIST_POINTS_new
0001:000d8850  _CRL_DIST_POINTS_free
0001:000d8870* _d2i_ISSUING_DIST_POINT
0001:000d88a0* _i2d_ISSUING_DIST_POINT
0001:000d88d0* _ISSUING_DIST_POINT_new
0001:000d88f0  _ISSUING_DIST_POINT_free
0001:000d8910  _DIST_POINT_set_dpname
0001:000d8a00  _v3_idp
0001:000d8e00  _v3_freshest_crl
0001:000d8e40  _v3_crld
Module: U:\tmp\ldconv_libcrypto_a_99560c9c37f156ab8.lib(pcy_cache.obj)
0001:000d8ec0  _policy_cache_free
0001:000d8f10  _policy_cache_set
0001:000d9380  _policy_cache_find_data
Module: U:\tmp\ldconv_libcrypto_a_99560c9c37f156ab8.lib(v3_genn.obj)
0001:000d93c0* _d2i_GENERAL_NAME
0001:000d99d4  _GENERAL_NAME_it
0001:000d93f0* _i2d_GENERAL_NAME
0001:000d9420* _d2i_OTHERNAME
0001:000d9bb4* _OTHERNAME_it
0001:000d9450* _i2d_OTHERNAME
0001:000d9480  _OTHERNAME_new
0001:000d94a0* _OTHERNAME_free
0001:000d94c0* _d2i_EDIPARTYNAME
0001:000d9b44* _EDIPARTYNAME_it
0001:000d94f0* _i2d_EDIPARTYNAME
0001:000d9520* _EDIPARTYNAME_new
0001:000d9540* _EDIPARTYNAME_free
0001:000d9560  _GENERAL_NAME_new
0001:000d9580  _GENERAL_NAME_free
0001:000d95a0* _d2i_GENERAL_NAMES
0001:000d9984  _GENERAL_NAMES_it
0001:000d95d0* _i2d_GENERAL_NAMES
0001:000d9600  _GENERAL_NAMES_new
0001:000d9620  _GENERAL_NAMES_free
0001:000d9640* _GENERAL_NAME_dup
0001:000d9670  _GENERAL_NAME_cmp
0001:000d97f0* _OTHERNAME_cmp
0001:000d9850* _GENERAL_NAME_set0_value
0001:000d98a0* _GENERAL_NAME_get0_value
0001:000d98f0* _GENERAL_NAME_set0_othername
0001:000d9940* _GENERAL_NAME_get0_otherName
Module: U:\tmp\ldconv_libcrypto_a_99560c9c37f156ab8.lib(v3_ncons.obj)
0001:000daaf8* _NAME_CONSTRAINTS_it
0001:000dab78* _GENERAL_SUBTREE_it
0001:000da6c0* _GENERAL_SUBTREE_new
0001:000da6e0* _GENERAL_SUBTREE_free
0001:000da700* _NAME_CONSTRAINTS_new
0001:000da720  _NAME_CONSTRAINTS_free
0001:000da740  _NAME_CONSTRAINTS_check
0001:000da900  _NAME_CONSTRAINTS_check_CN
0001:000dac00  _v3_name_constraints
Module: U:\tmp\ldconv_libcrypto_a_99560c9c37f156ab8.lib(v3_addr.obj)
0001:000dac40  _IPAddressFamily_free
0001:000def08* _IPAddressFamily_it
0001:000def98* _IPAddressChoice_it
0001:000df01c* _IPAddressOrRange_it
0001:000df098* _IPAddressRange_it
0001:000dccd0* _d2i_IPAddressRange
0001:000dcd00* _i2d_IPAddressRange
0001:000dcd30* _IPAddressRange_new
0001:000dcd50* _IPAddressRange_free
0001:000dcd70* _d2i_IPAddressOrRange
0001:000dcda0* _i2d_IPAddressOrRange
0001:000dcdd0* _IPAddressOrRange_new
0001:000dcdf0* _IPAddressOrRange_free
0001:000dce10* _d2i_IPAddressChoice
0001:000dce40* _i2d_IPAddressChoice
0001:000dce70* _IPAddressChoice_new
0001:000dce90* _IPAddressChoice_free
0001:000dceb0* _d2i_IPAddressFamily
0001:000dcee0* _i2d_IPAddressFamily
0001:000dcf10* _IPAddressFamily_new
0001:000dcf30* _X509v3_addr_get_afi
0001:000dcf70* _X509v3_addr_add_inherit
0001:000dcff0* _X509v3_addr_add_prefix
0001:000dd110* _X509v3_addr_add_range
0001:000dd280* _X509v3_addr_get_range
0001:000dd300* _X509v3_addr_is_canonical
0001:000dddf0* _X509v3_addr_canonize
0001:000deb80* _X509v3_addr_inherits
0001:000debe0* _X509v3_addr_subset
0001:000ded40  _X509v3_addr_validate_path
0001:000deda0* _X509v3_addr_validate_resource_set
0001:000dee80  _v3_addr
Module: U:\tmp\ldconv_libcrypto_a_99560c9c37f156ab8.lib(v3_asid.obj)
0001:000e0f54* _ASIdOrRange_it
0001:000dfc80* _d2i_ASRange
0001:000e0fb0* _ASRange_it
0001:000dfcb0* _i2d_ASRange
0001:000dfce0* _ASRange_new
0001:000dfd00* _ASRange_free
0001:000dfd20* _d2i_ASIdOrRange
0001:000dfd50* _i2d_ASIdOrRange
0001:000dfd80* _ASIdOrRange_new
0001:000dfda0* _ASIdOrRange_free
0001:000dfdc0* _d2i_ASIdentifierChoice
0001:000e0edc* _ASIdentifierChoice_it
0001:000dfdf0* _i2d_ASIdentifierChoice
0001:000dfe20* _ASIdentifierChoice_new
0001:000dfe40* _ASIdentifierChoice_free
0001:000dfe60* _d2i_ASIdentifiers
0001:000e0e68* _ASIdentifiers_it
0001:000dfe90* _i2d_ASIdentifiers
0001:000dfec0* _ASIdentifiers_new
0001:000dfee0  _ASIdentifiers_free
0001:000dff00* _X509v3_asid_add_inherit
0001:000dff80* _X509v3_asid_add_id_or_range
0001:000e00c0* _X509v3_asid_is_canonical
0001:000e06a0* _X509v3_asid_canonize
0001:000e0c60* _X509v3_asid_inherits
0001:000e0c90* _X509v3_asid_subset
0001:000e0d30  _X509v3_asid_validate_path
0001:000e0d90* _X509v3_asid_validate_resource_set
0001:000e0e20  _v3_asid
Module: U:\tmp\ldconv_libcrypto_a_99560c9c37f156ab8.lib(tasn_dec.obj)
0001:000e3670  _ASN1_tag2bit
0001:000e3690  _ASN1_item_d2i
0001:000e4170  _ASN1_item_ex_d2i
Module: U:\tmp\ldconv_libcrypto_a_99560c9c37f156ab8.lib(tasn_enc.obj)
0001:000e52f0  _ASN1_item_ex_i2d
0001:000e5e90  _ASN1_item_ndef_i2d
0001:000e6410  _ASN1_item_i2d
Module: U:\tmp\ldconv_libcrypto_a_99560c9c37f156ab8.lib(tasn_new.obj)
0001:000e70a0  _ASN1_item_new
0001:000e7460  _ASN1_item_ex_new
Module: U:\tmp\ldconv_libcrypto_a_99560c9c37f156ab8.lib(tasn_fre.obj)
0001:000e7810  _asn1_primitive_free
0001:000e7920  _asn1_item_embed_free
0001:000e7ea0  _ASN1_item_free
0001:000e7ed0  _ASN1_item_ex_free
0001:000e7f00  _asn1_template_free
Module: U:\tmp\ldconv_libcrypto_a_99560c9c37f156ab8.lib(a_dup.obj)
0001:000e7fd0  _ASN1_dup
0001:000e80a0  _ASN1_item_dup
Module: U:\tmp\ldconv_libcrypto_a_99560c9c37f156ab8.lib(x_algor.obj)
0001:000e8160  _d2i_X509_ALGOR
0001:000e8590  _X509_ALGOR_it
0001:000e8190  _i2d_X509_ALGOR
0001:000e81c0  _X509_ALGOR_new
0001:000e81e0  _X509_ALGOR_free
0001:000e8200* _d2i_X509_ALGORS
0001:000e8548  _X509_ALGORS_it
0001:000e8230  _i2d_X509_ALGORS
0001:000e8260* _X509_ALGOR_dup
0001:000e8280  _X509_ALGOR_set0
0001:000e8330  _X509_ALGOR_get0
0001:000e8380  _X509_ALGOR_set_md
0001:000e8440  _X509_ALGOR_cmp
0001:000e8490  _X509_ALGOR_copy
Module: U:\tmp\ldconv_libcrypto_a_99560c9c37f156ab8.lib(x_val.obj)
0001:000e8600* _d2i_X509_VAL
0001:000e86a4  _X509_VAL_it
0001:000e8630* _i2d_X509_VAL
0001:000e8660* _X509_VAL_new
0001:000e8680* _X509_VAL_free
Module: U:\tmp\ldconv_libcrypto_a_99560c9c37f156ab8.lib(mem_dbg.obj)
0001:000e8720  _CRYPTO_mem_ctrl
Module: U:\tmp\ldconv_libssl_a_99560c9c37e1aece0.lib(s3_lib.obj)
0001:000e8760  _ssl3_handshake_write
0001:000e87c0  _ssl3_set_handshake_header
0001:000e8820  _ssl_sort_cipher_list
0001:000e88a0* _ssl3_default_timeout
0001:000e88b0  _ssl3_num_ciphers
0001:000e88c0  _ssl3_get_cipher
0001:000e88e0  _ssl3_new
0001:000e8940  _ssl3_free
0001:000e8af0  _ssl3_clear
0001:000e8cb0  _ssl3_ctrl
0001:000e97c0  _ssl3_callback_ctrl
0001:000e9830  _ssl3_ctx_ctrl
0001:000ea360  _ssl3_ctx_callback_ctrl
0001:000ea490  _ssl3_get_cipher_by_id
0001:000ea500  _ssl3_get_cipher_by_std_name
0001:000ea5a0  _ssl3_get_cipher_by_char
0001:000ea620  _ssl3_put_cipher_by_char
0001:000ea690  _ssl3_choose_cipher
0001:000eabc0  _ssl3_get_req_cert_type
0001:000eada0  _ssl3_shutdown
0001:000eaec0  _ssl3_write
0001:000eaf60  _ssl3_read
0001:000eb0b0  _ssl3_peek
0001:000eb200  _ssl3_renegotiate
0001:000eb220  _ssl3_renegotiate_check
0001:000eb2a0  _ssl_get_algorithm2
0001:000eb300  _ssl_fill_hello_random
0001:000eb3d0  _ssl_generate_master_secret
0001:000eb690  _ssl_generate_pkey
0001:000eb720  _ssl_generate_pkey_group
0001:000eb900  _ssl_generate_param_group
0001:000eba10  _ssl_derive
0001:000ebcd0  _ssl_dh_to_pkey
0001:000ebd30* _SSLv3_enc_data
0001:000ee2a4  _tls12downgrade
0001:000ee2ac  _tls11downgrade
Module: U:\tmp\ldconv_libcrypto_a_99560c9c37f156ab8.lib(ameth_lib.obj)
0001:000ee310  _EVP_PKEY_asn1_get_count
0001:000ee340  _EVP_PKEY_asn1_get0
0001:000ee390  _EVP_PKEY_asn1_find
0001:000ee4a0  _EVP_PKEY_asn1_find_str
0001:000ee620* _EVP_PKEY_asn1_add0
0001:000ee750* _EVP_PKEY_asn1_add_alias
0001:000ee910  _EVP_PKEY_asn1_get0_info
0001:000ee980  _EVP_PKEY_get0_asn1
0001:000ee990* _EVP_PKEY_asn1_new
0001:000eea90* _EVP_PKEY_asn1_copy
0001:000eeb40  _EVP_PKEY_asn1_free
0001:000eebc0* _EVP_PKEY_asn1_set_public
0001:000eebf0* _EVP_PKEY_asn1_set_private
0001:000eec10* _EVP_PKEY_asn1_set_param
0001:000eec40* _EVP_PKEY_asn1_set_free
0001:000eec50* _EVP_PKEY_asn1_set_ctrl
0001:000eec60* _EVP_PKEY_asn1_set_security_bits
0001:000eec70* _EVP_PKEY_asn1_set_item
0001:000eec90* _EVP_PKEY_asn1_set_siginf
0001:000eeca0* _EVP_PKEY_asn1_set_check
0001:000eecb0* _EVP_PKEY_asn1_set_public_check
0001:000eecc0* _EVP_PKEY_asn1_set_param_check
0001:000eecd0* _EVP_PKEY_asn1_set_set_priv_key
0001:000eece0* _EVP_PKEY_asn1_set_set_pub_key
0001:000eecf0* _EVP_PKEY_asn1_set_get_priv_key
0001:000eed00* _EVP_PKEY_asn1_set_get_pub_key
Module: U:\tmp\ldconv_libcrypto_a_99560c9c37f156ab8.lib(e_null.obj)
0001:000eed50  _EVP_enc_null
Module: U:\tmp\ldconv_libcrypto_a_99560c9c37f156ab8.lib(conf_mod.obj)
0001:000eee20* _CONF_modules_load
0001:000ef4b0* _CONF_modules_finish
0001:000ef560* _CONF_modules_unload
0001:000ef6b0  _CONF_module_add
0001:000ef7f0  _conf_modules_free_int
0001:000ef810* _CONF_imodule_get_name
0001:000ef820  _CONF_imodule_get_value
0001:000ef830* _CONF_imodule_get_usr_data
0001:000ef840* _CONF_imodule_set_usr_data
0001:000ef850* _CONF_imodule_get_module
0001:000ef860* _CONF_imodule_get_flags
0001:000ef870* _CONF_imodule_set_flags
0001:000ef880* _CONF_module_get_usr_data
0001:000ef890* _CONF_module_set_usr_data
0001:000ef8c0* _CONF_get1_default_config_file
0001:000ef970  _CONF_modules_load_file
0001:000efa60  _CONF_parse_list
Module: U:\tmp\ldconv_libcrypto_a_99560c9c37f156ab8.lib(b_print.obj)
0001:000f2480* _BIO_vprintf
0001:000f2570  _BIO_printf
0001:000f25a0  _BIO_snprintf
0001:000f2610* _BIO_vsnprintf
Module: U:\tmp\ldconv_libcrypto_a_99560c9c37f156ab8.lib(tb_pkmeth.obj)
0001:000f26d0* _ENGINE_unregister_pkey_meths
0001:000f26f0  _ENGINE_register_pkey_meths
0001:000f2770* _ENGINE_register_all_pkey_meths
0001:000f2810  _ENGINE_set_default_pkey_meths
0001:000f2890  _ENGINE_get_pkey_meth_engine
0001:000f28d0  _ENGINE_get_pkey_meth
0001:000f2950* _ENGINE_get_pkey_meths
0001:000f2960* _ENGINE_set_pkey_meths
0001:000f2980  _engine_pkey_meths_free
Module: U:\tmp\ldconv_libcrypto_a_99560c9c37f156ab8.lib(rsa_lib.obj)
0001:000f2a10* _RSA_get_method
0001:000f2a20* _RSA_set_method
0001:000f2a80  _RSA_free
0001:000f2bb0* _RSA_new_method
0001:000f2db0  _RSA_new
0001:000f2dd0  _RSA_up_ref
0001:000f2df0* _RSA_set_ex_data
0001:000f2e00* _RSA_get_ex_data
0001:000f2e10  _RSA_security_bits
0001:000f2e70* _RSA_set0_key
0001:000f2f20* _RSA_set0_factors
0001:000f2fd0* _RSA_set0_crt_params
0001:000f3090* _RSA_set0_multi_prime_params
0001:000f3240* _RSA_get0_key
0001:000f3270* _RSA_get0_factors
0001:000f32a0* _RSA_get_multi_prime_extra_count
0001:000f32c0* _RSA_get0_multi_prime_factors
0001:000f3320* _RSA_get0_crt_params
0001:000f3350* _RSA_get0_multi_prime_crt_params
0001:000f3420* _RSA_get0_n
0001:000f3430* _RSA_get0_e
0001:000f3440* _RSA_get0_d
0001:000f3450* _RSA_get0_p
0001:000f3460* _RSA_get0_q
0001:000f3470* _RSA_get0_dmp1
0001:000f3480* _RSA_get0_dmq1
0001:000f3490* _RSA_get0_iqmp
0001:000f34a0* _RSA_get0_pss_params
0001:000f34b0* _RSA_clear_flags
0001:000f34c0* _RSA_test_flags
0001:000f34d0* _RSA_set_flags
0001:000f34e0* _RSA_get_version
0001:000f34f0* _RSA_get0_engine
0001:000f3500  _RSA_pkey_ctx_ctrl
Module: U:\tmp\ldconv_libcrypto_a_99560c9c37f156ab8.lib(dsa_lib.obj)
0001:000f3560* _DSA_set_method
0001:000f35b0* _DSA_get_method
0001:000f35d0  _DSA_free
0001:000f3690* _DSA_new_method
0001:000f3890  _DSA_new
0001:000f38b0  _DSA_up_ref
0001:000f38d0  _DSA_size
0001:000f3940* _DSA_set_ex_data
0001:000f3950* _DSA_get_ex_data
0001:000f3960  _DSA_security_bits
0001:000f39b0  _DSA_dup_DH
0001:000f3ba0* _DSA_get0_pqg
0001:000f3bd0* _DSA_set0_pqg
0001:000f3c50* _DSA_get0_key
0001:000f3c80* _DSA_set0_key
0001:000f3ce0* _DSA_get0_p
0001:000f3cf0* _DSA_get0_q
0001:000f3d00* _DSA_get0_g
0001:000f3d10* _DSA_get0_pub_key
0001:000f3d20* _DSA_get0_priv_key
0001:000f3d30* _DSA_clear_flags
0001:000f3d40* _DSA_test_flags
0001:000f3d50* _DSA_set_flags
0001:000f3d60* _DSA_get0_engine
0001:000f3d70  _DSA_bits
Module: U:\tmp\ldconv_libcrypto_a_99560c9c37f156ab8.lib(x_attrib.obj)
0001:000f3d80* _d2i_X509_ATTRIBUTE
0001:000f3ee4  _X509_ATTRIBUTE_it
0001:000f3db0* _i2d_X509_ATTRIBUTE
0001:000f3de0  _X509_ATTRIBUTE_new
0001:000f3e00  _X509_ATTRIBUTE_free
0001:000f3e20  _X509_ATTRIBUTE_dup
0001:000f3e40  _X509_ATTRIBUTE_create
Module: U:\tmp\ldconv_libcrypto_a_99560c9c37f156ab8.lib(cmac.obj)
0001:000f3f80  _CMAC_CTX_new
0001:000f4020* _CMAC_CTX_cleanup
0001:000f4090* _CMAC_CTX_get0_cipher_ctx
0001:000f40a0  _CMAC_CTX_free
0001:000f4140  _CMAC_CTX_copy
0001:000f4200  _CMAC_Init
0001:000f44f0  _CMAC_Update
0001:000f4610  _CMAC_Final
0001:000f4910* _CMAC_resume
Module: U:\tmp\ldconv_libcrypto_a_99560c9c37f156ab8.lib(a_object.obj)
0001:000f49a0* _i2d_ASN1_OBJECT
0001:000f4af0  _a2d_ASN1_OBJECT
0001:000f50a0  _i2t_ASN1_OBJECT
0001:000f50e0  _i2a_ASN1_OBJECT
0001:000f52a0  _ASN1_OBJECT_new
0001:000f5310  _ASN1_OBJECT_free
0001:000f53d0  _c2i_ASN1_OBJECT
0001:000f5600  _d2i_ASN1_OBJECT
0001:000f56b0* _ASN1_OBJECT_create
Module: U:\tmp\ldconv_libcrypto_a_99560c9c37f156ab8.lib(obj_lib.obj)
0001:000f5720  _OBJ_dup
0001:000f5870  _OBJ_cmp
Module: U:\tmp\ldconv_libcrypto_a_99560c9c37f156ab8.lib(bn_shift.obj)
0001:000f58b0  _BN_lshift1
0001:000f5970  _BN_rshift1
0001:000f5a60  _BN_lshift
0001:000f5c10  _bn_lshift_fixed_top
0001:000f5d80  _bn_rshift_fixed_top
0001:000f5ec0  _BN_rshift
Module: U:\tmp\ldconv_libcrypto_a_99560c9c37f156ab8.lib(bn_word.obj)
0001:000f5f40  _BN_mod_word
0001:000f5fb0  _BN_div_word
0001:000f60a0  _BN_sub_word
0001:000f6190  _BN_add_word
0001:000f6260  _BN_mul_word
Module: U:\tmp\ldconv_libcrypto_a_99560c9c37f156ab8.lib(bn_print.obj)
0001:000f6310  _BN_bn2hex
0001:000f6500  _BN_bn2dec
0001:000f67c0  _BN_hex2bn
0001:000f69c0  _BN_dec2bn
0001:000f6ba0  _BN_asc2bn
0001:000f6c30  _BN_print
0001:000f6eb0* _BN_print_fp
0001:000f6f20* _BN_options
Module: U:\tmp\ldconv_libcrypto_a_99560c9c37f156ab8.lib(asn1_lib.obj)
0001:000f6f90* _ASN1_check_infinite_end
0001:000f6fd0* _ASN1_const_check_infinite_end
0001:000f7030  _ASN1_get_object
0001:000f7240  _ASN1_put_object
0001:000f7350  _ASN1_put_eoc
0001:000f7370  _ASN1_object_size
0001:000f73f0  _ASN1_STRING_copy
0001:000f7530  _ASN1_STRING_dup
0001:000f7730  _ASN1_STRING_set
0001:000f7850  _ASN1_STRING_set0
0001:000f7890  _ASN1_STRING_new
0001:000f7900  _ASN1_STRING_type_new
0001:000f7970  _asn1_string_embed_free
0001:000f79d0  _ASN1_STRING_free
0001:000f7a40  _ASN1_STRING_clear_free
0001:000f7af0  _ASN1_STRING_cmp
0001:000f7b30  _ASN1_STRING_length
0001:000f7b40* _ASN1_STRING_length_set
0001:000f7b50* _ASN1_STRING_type
0001:000f7b60  _ASN1_STRING_get0_data
0001:000f7b70* _ASN1_STRING_data
Module: U:\tmp\ldconv_libcrypto_a_99560c9c37f156ab8.lib(ctype.obj)
0001:000f7b80  _ossl_ctype_check
0001:000f7ba0  _ossl_tolower
0001:000f7bc0* _ossl_toupper
0001:000f7be0  _ascii_isdigit
Module: U:\tmp\ldconv_libcrypto_a_99560c9c37f156ab8.lib(ec_kmeth.obj)
0001:000f7d00  _EC_KEY_OpenSSL
0001:000f7d10* _EC_KEY_get_default_method
0001:000f7d20* _EC_KEY_set_default_method
0001:000f7d40* _EC_KEY_get_method
0001:000f7d50* _EC_KEY_set_method
0001:000f7dc0  _EC_KEY_new_method
0001:000f7fb0  _ECDH_compute_key
0001:000f80f0* _EC_KEY_METHOD_new
0001:000f8180* _EC_KEY_METHOD_free
0001:000f81c0* _EC_KEY_METHOD_set_init
0001:000f81f0* _EC_KEY_METHOD_set_keygen
0001:000f8200* _EC_KEY_METHOD_set_compute_key
0001:000f8210* _EC_KEY_METHOD_set_sign
0001:000f8230* _EC_KEY_METHOD_set_verify
0001:000f8250* _EC_KEY_METHOD_get_init
0001:000f82c0* _EC_KEY_METHOD_get_keygen
0001:000f82e0* _EC_KEY_METHOD_get_compute_key
0001:000f8300* _EC_KEY_METHOD_get_sign
0001:000f8330* _EC_KEY_METHOD_get_verify
Module: U:\tmp\ldconv_libcrypto_a_99560c9c37f156ab8.lib(bn_ctx.obj)
0001:000f83e0  _BN_CTX_new
0001:000f8480  _BN_CTX_secure_new
0001:000f8520  _BN_CTX_free
0001:000f85d0  _BN_CTX_start
0001:000f8710  _BN_CTX_end
0001:000f87a0  _BN_CTX_get
Module: U:\tmp\ldconv_libcrypto_a_99560c9c37f156ab8.lib(bn_rand.obj)
0001:000f8d90  _BN_rand
0001:000f8f60* _BN_bntest_rand
0001:000f9000  _BN_priv_rand
0001:000f91d0* _BN_rand_range
0001:000f9240  _BN_priv_rand_range
0001:000f92b0* _BN_pseudo_rand
0001:000f9480* _BN_pseudo_rand_range
0001:000f94f0  _BN_generate_dsa_nonce
Module: U:\tmp\ldconv_libcrypto_a_99560c9c37f156ab8.lib(bn_intern.obj)
0001:000f97e0  _bn_compute_wNAF
0001:000f9ae0  _bn_get_top
0001:000f9af0* _bn_get_dmax
0001:000f9b00  _bn_set_all_zero
0001:000f9b20  _bn_copy_words
0001:000f9b90  _bn_get_words
0001:000f9ba0* _bn_set_static_words
0001:000f9bd0  _bn_set_words
Module: U:\tmp\ldconv_libcrypto_a_99560c9c37f156ab8.lib(ec_oct.obj)
0001:000f9c80  _EC_POINT_set_compressed_coordinates
0001:000f9dc0* _EC_POINT_set_compressed_coordinates_GFp
0001:000f9f00* _EC_POINT_set_compressed_coordinates_GF2m
0001:000fa040  _EC_POINT_point2oct
0001:000fa190  _EC_POINT_oct2point
0001:000fa2d0  _EC_POINT_point2buf
Module: U:\tmp\ldconv_libcrypto_a_99560c9c37f156ab8.lib(ec_mult.obj)
0001:000fae60  _EC_ec_pre_comp_dup
0001:000fae70  _EC_ec_pre_comp_free
0001:000faf10  _ec_scalar_mul_ladder
0001:000fafd0  _ec_wNAF_mul
0001:000fc260  _ec_wNAF_precompute_mult
0001:000fc8c0  _ec_wNAF_have_precompute_mult
Module: U:\tmp\ldconv_libcrypto_a_99560c9c37f156ab8.lib(ecp_nistz256.obj)
0001:000fe9f0  _EC_nistz256_pre_comp_dup
0001:000fea00  _EC_nistz256_pre_comp_free
0001:000fea70  _EC_GFp_nistz256_method
Module: U:\tmp\ldconv_libcrypto_a_99560c9c37f156ab8.lib(bn_mont.obj)
0001:000fed60  _BN_mod_mul_montgomery
0001:000feec0  _bn_mul_mont_fixed_top
0001:000ff020  _BN_from_montgomery
0001:000ff090  _bn_from_mont_fixed_top
0001:000ff100  _bn_to_mont_fixed_top
0001:000ff270  _BN_MONT_CTX_new
0001:000ff310* _BN_MONT_CTX_init
0001:000ff360  _BN_MONT_CTX_free
0001:000ff3c0  _BN_MONT_CTX_set
0001:000ff760  _BN_MONT_CTX_copy
0001:000ff7e0  _BN_MONT_CTX_set_locked
Module: U:\tmp\ldconv_libcrypto_a_99560c9c37f156ab8.lib(bn_add.obj)
0001:000ff9b0  _BN_uadd
0001:000ffa90  _BN_usub
0001:000ffbb0  _BN_add
0001:000ffc60  _BN_sub
Module: U:\tmp\ldconv_libcrypto_a_99560c9c37f156ab8.lib(bn_div.obj)
0001:000ffd10* _bn_div_fixed_top
0001:001001c0  _BN_div
Module: U:\tmp\ldconv_libcrypto_a_99560c9c37f156ab8.lib(bn_exp.obj)
0001:00101410* _BN_exp
0001:00101600* _BN_mod_exp_recp
0001:001016c0  _BN_mod_exp_mont_consttime
0001:00101ea0  _BN_mod_exp_mont
0001:00101f60  _BN_mod_exp
0001:00102210* _BN_mod_exp_mont_word
0001:00102300* _BN_mod_exp_simple
Module: U:\tmp\ldconv_libcrypto_a_99560c9c37f156ab8.lib(ec_cvt.obj)
0001:001027e0  _EC_GROUP_new_curve_GFp
0001:00102840  _EC_GROUP_new_curve_GF2m
Module: U:\usr\lib\libc_dll.lib(highmemsocket.obj)
0001:001028cc* ___libsocket_safe_copy
0001:00102940  ___libsocket_safe_addr_pre
0001:00102a44  ___libsocket_safe_addr_post
0001:00102af5  ___libsocket_safe_addr_free
Module: U:\tmp\ldconv_libcrypto_a_99560c9c37f156ab8.lib(tb_asnmth.obj)
0001:00102bf0* _ENGINE_unregister_pkey_asn1_meths
0001:00102c10  _ENGINE_register_pkey_asn1_meths
0001:00102c90* _ENGINE_register_all_pkey_asn1_meths
0001:00102d30  _ENGINE_set_default_pkey_asn1_meths
0001:00102db0  _ENGINE_get_pkey_asn1_meth_engine
0001:00102df0  _ENGINE_get_pkey_asn1_meth
0001:00102e70  _ENGINE_get_pkey_asn1_meths
0001:00102e80* _ENGINE_set_pkey_asn1_meths
0001:00102ea0  _engine_pkey_asn1_meths_free
0001:00102f30* _ENGINE_get_pkey_asn1_meth_str
0001:00103010  _ENGINE_pkey_asn1_find_str
Module: U:\tmp\ldconv_libcrypto_a_99560c9c37f156ab8.lib(tb_dsa.obj)
0001:00103110* _ENGINE_unregister_DSA
0001:00103130  _ENGINE_register_DSA
0001:00103190* _ENGINE_register_all_DSA
0001:001031f0  _ENGINE_set_default_DSA
0001:00103250  _ENGINE_get_default_DSA
0001:00103270  _ENGINE_get_DSA
0001:00103280  _ENGINE_set_DSA
Module: U:\tmp\ldconv_libcrypto_a_99560c9c37f156ab8.lib(tb_dh.obj)
0001:001032c0* _ENGINE_unregister_DH
0001:001032e0  _ENGINE_register_DH
0001:00103340* _ENGINE_register_all_DH
0001:001033a0  _ENGINE_set_default_DH
0001:00103400  _ENGINE_get_default_DH
0001:00103420  _ENGINE_get_DH
0001:00103430  _ENGINE_set_DH
Module: U:\tmp\ldconv_libcrypto_a_99560c9c37f156ab8.lib(tb_cipher.obj)
0001:00103470* _ENGINE_unregister_ciphers
0001:00103490  _ENGINE_register_ciphers
0001:00103510* _ENGINE_register_all_ciphers
0001:001035b0  _ENGINE_set_default_ciphers
0001:00103630  _ENGINE_get_cipher_engine
0001:00103670  _ENGINE_get_cipher
0001:001036f0* _ENGINE_get_ciphers
0001:00103700  _ENGINE_set_ciphers
Module: U:\tmp\ldconv_libcrypto_a_99560c9c37f156ab8.lib(tb_digest.obj)
0001:00103740* _ENGINE_unregister_digests
0001:00103760  _ENGINE_register_digests
0001:001037e0* _ENGINE_register_all_digests
0001:00103880  _ENGINE_set_default_digests
0001:00103900  _ENGINE_get_digest_engine
0001:00103940  _ENGINE_get_digest
0001:001039c0* _ENGINE_get_digests
0001:001039d0  _ENGINE_set_digests
Module: U:\tmp\ldconv_libcrypto_a_99560c9c37f156ab8.lib(tb_rsa.obj)
0001:00103a10* _ENGINE_unregister_RSA
0001:00103a30  _ENGINE_register_RSA
0001:00103a90* _ENGINE_register_all_RSA
0001:00103af0  _ENGINE_set_default_RSA
0001:00103b50  _ENGINE_get_default_RSA
0001:00103b70  _ENGINE_get_RSA
0001:00103b80  _ENGINE_set_RSA
Module: U:\tmp\ldconv_libcrypto_a_99560c9c37f156ab8.lib(tb_eckey.obj)
0001:00103bc0* _ENGINE_unregister_EC
0001:00103be0  _ENGINE_register_EC
0001:00103c40* _ENGINE_register_all_EC
0001:00103ca0  _ENGINE_set_default_EC
0001:00103d00  _ENGINE_get_default_EC
0001:00103d20  _ENGINE_get_EC
0001:00103d30  _ENGINE_set_EC
Module: U:\tmp\ldconv_libcrypto_a_99560c9c37f156ab8.lib(getenv.obj)
0001:00103d50  _ossl_safe_getenv
Module: U:\tmp\ldconv_libcrypto_a_99560c9c37f156ab8.lib(encode.obj)
0001:00104090  _EVP_ENCODE_CTX_new
0001:001040c0  _EVP_ENCODE_CTX_free
0001:001040f0* _EVP_ENCODE_CTX_copy
0001:00104120  _EVP_ENCODE_CTX_num
0001:00104130  _evp_encode_ctx_set_flags
0001:00104140  _EVP_EncodeInit
0001:001041a0  _EVP_EncodeUpdate
0001:00104380  _EVP_EncodeFinal
0001:001043e0  _EVP_EncodeBlock
0001:00104400  _EVP_DecodeInit
0001:00104420  _EVP_DecodeUpdate
0001:00104820  _EVP_DecodeBlock
0001:00104840  _EVP_DecodeFinal
Module: U:\tmp\ldconv_libcrypto_a_99560c9c37f156ab8.lib(cryptlib.obj)
0002:0000d820  _OPENSSL_ia32cap_P
0001:00104a60  _OPENSSL_cpuid_setup
0001:00104a70* _OPENSSL_showfatal
0001:00104aa0* _OPENSSL_isservice
0001:00104ad0  _OPENSSL_die
0001:00104b00  _CRYPTO_memcmp
0001:00104b50  _OPENSSL_rdtsc
0001:00104b60* _OPENSSL_instrument_bus
0001:00104b70* _OPENSSL_instrument_bus2
Module: U:\tmp\ldconv_libcrypto_a_99560c9c37f156ab8.lib(bio_meth.obj)
0001:00104b80  _bwrite_conv
0001:00104bc0  _bread_conv
0001:00104c40* _BIO_get_new_index
0001:00104cc0* _BIO_meth_new
0001:00104d70* _BIO_meth_free
0001:00104dc0* _BIO_meth_get_write
0001:00104dd0* _BIO_meth_get_write_ex
0001:00104de0* _BIO_meth_set_write
0001:00104e00* _BIO_meth_set_write_ex
0001:00104e20* _BIO_meth_get_read
0001:00104e30* _BIO_meth_get_read_ex
0001:00104e40* _BIO_meth_set_read
0001:00104e60* _BIO_meth_set_read_ex
0001:00104e80* _BIO_meth_get_puts
0001:00104e90* _BIO_meth_set_puts
0001:00104eb0* _BIO_meth_get_gets
0001:00104ec0* _BIO_meth_set_gets
0001:00104ee0* _BIO_meth_get_ctrl
0001:00104ef0* _BIO_meth_set_ctrl
0001:00104f10* _BIO_meth_get_create
0001:00104f20* _BIO_meth_set_create
0001:00104f40* _BIO_meth_get_destroy
0001:00104f50* _BIO_meth_set_destroy
0001:00104f70* _BIO_meth_get_callback_ctrl
0001:00104f80* _BIO_meth_set_callback_ctrl
0002:0000d160  _bio_type_lock
Module: U:\tmp\ldconv_libcrypto_a_99560c9c37f156ab8.lib(b_sock.obj)
0001:00104fc0* _BIO_get_host_ip
0001:001050f0* _BIO_get_port
0001:00105230* _BIO_sock_error
0001:00105290* _BIO_gethostbyname
0001:001052a0  _BIO_sock_init
0001:001052b0  _bio_sock_cleanup_int
0001:001052c0* _BIO_socket_ioctl
0001:00105330* _BIO_get_accept_socket
0001:001054a0* _BIO_accept
0001:00105690* _BIO_set_tcp_ndelay
0001:001056d0  _BIO_socket_nbio
0001:00105750* _BIO_sock_info
Module: U:\tmp\ldconv_libcrypto_a_99560c9c37f156ab8.lib(des-586.obj)
0001:00106e30* _DES_SPtrans
0001:001066b0  _DES_encrypt1
0001:001067a0* _DES_encrypt2
0001:001067f0  _DES_encrypt3
0001:00106920  _DES_decrypt3
0001:00106a50  _DES_ncbc_encrypt
0001:00106c30  _DES_ede3_cbc_encrypt
Module: U:\tmp\ldconv_libcrypto_a_99560c9c37f156ab8.lib(o_fopen.obj)
0001:00107630  _openssl_fopen
Module: U:\tmp\ldconv_libcrypto_a_99560c9c37f156ab8.lib(conf_def.obj)
0001:00109290  _NCONF_default
0001:001092a0* _NCONF_WIN32
Module: U:\tmp\ldconv_libcrypto_a_99560c9c37f156ab8.lib(conf_api.obj)
0001:00109690  __CONF_get_section
0001:001096e0  __CONF_get_section_values
0001:00109730  __CONF_add_string
0001:001097f0  __CONF_get_string
0001:001098b0  __CONF_new_data
0001:00109910  __CONF_free_data
0001:00109980  __CONF_new_section
Module: U:\tmp\ldconv_libcrypto_a_99560c9c37f156ab8.lib(e_padlock.obj)
0001:00109aa0  _engine_load_padlock_int
Module: U:\tmp\ldconv_libcrypto_a_99560c9c37f156ab8.lib(eng_dyn.obj)
0001:0010a5f0  _engine_load_dynamic_int
Module: U:\tmp\ldconv_libcrypto_a_99560c9c37f156ab8.lib(eng_rdrand.obj)
0001:0010a930  _engine_load_rdrand_int
Module: U:\tmp\ldconv_libcrypto_a_99560c9c37f156ab8.lib(eng_openssl.obj)
0001:0010b170  _engine_load_openssl_int
Module: U:\tmp\ldconv_libcrypto_a_99560c9c37f156ab8.lib(conf_sap.obj)
0001:0010b2a0* _OPENSSL_config
0001:0010b300  _openssl_config_int
0001:0010b370  _openssl_no_config_int
Module: U:\tmp\ldconv_libcrypto_a_99560c9c37f156ab8.lib(c_alld.obj)
0001:0010b3d0  _openssl_add_all_digests_int
Module: U:\tmp\ldconv_libcrypto_a_99560c9c37f156ab8.lib(c_allc.obj)
0001:0010b850  _openssl_add_all_ciphers_int
Module: U:\tmp\ldconv_libcrypto_a_99560c9c37f156ab8.lib(err_all.obj)
0001:0010c4f0  _err_load_crypto_strings_int
Module: U:\tmp\ldconv_libcrypto_a_99560c9c37f156ab8.lib(store_init.obj)
0001:0010c6c0  _ossl_store_init_once
0001:0010c730  _ossl_store_cleanup_int
Module: U:\tmp\ldconv_libssl_a_99560c9c37e1aece0.lib(ssl_err.obj)
0001:0010c740  _ERR_load_SSL_strings
Module: U:\tmp\ldconv_libcrypto_a_99560c9c37f156ab8.lib(e_des.obj)
0001:00112870  _EVP_des_cbc
0001:00112880  _EVP_des_cfb64
0001:00112890  _EVP_des_ofb
0001:001128a0  _EVP_des_ecb
0001:001128b0  _EVP_des_cfb1
0001:001128c0  _EVP_des_cfb8
Module: U:\tmp\ldconv_libcrypto_a_99560c9c37f156ab8.lib(e_des3.obj)
0001:00113930  _EVP_des_ede_cbc
0001:00113940  _EVP_des_ede_cfb64
0001:00113950  _EVP_des_ede_ofb
0001:00113960* _EVP_des_ede_ecb
0001:00113970  _EVP_des_ede3_cbc
0001:00113980  _EVP_des_ede3_cfb64
0001:00113990  _EVP_des_ede3_ofb
0001:001139a0* _EVP_des_ede3_ecb
0001:001139b0  _EVP_des_ede3_cfb1
0001:001139c0  _EVP_des_ede3_cfb8
0001:001139d0  _EVP_des_ede
0001:001139e0  _EVP_des_ede3
0001:001139f0  _EVP_des_ede3_wrap
Module: U:\tmp\ldconv_libcrypto_a_99560c9c37f156ab8.lib(e_idea.obj)
0001:00114110  _EVP_idea_cbc
0001:00114120  _EVP_idea_cfb64
0001:00114130  _EVP_idea_ofb
0001:00114140  _EVP_idea_ecb
Module: U:\tmp\ldconv_libcrypto_a_99560c9c37f156ab8.lib(e_rc4.obj)
0001:001142e0  _EVP_rc4
0001:001142f0  _EVP_rc4_40
Module: U:\tmp\ldconv_libcrypto_a_99560c9c37f156ab8.lib(e_rc4_hmac_md5.obj)
0001:001148d0  _EVP_rc4_hmac_md5
Module: U:\tmp\ldconv_libcrypto_a_99560c9c37f156ab8.lib(e_rc2.obj)
0001:00115010  _EVP_rc2_cbc
0001:00115020  _EVP_rc2_cfb64
0001:00115030  _EVP_rc2_ofb
0001:00115040  _EVP_rc2_ecb
0001:00115050  _EVP_rc2_64_cbc
0001:00115060  _EVP_rc2_40_cbc
Module: U:\tmp\ldconv_libcrypto_a_99560c9c37f156ab8.lib(e_aes_cbc_hmac_sha1.obj)
0001:00115200  _EVP_aes_128_cbc_hmac_sha1
0001:00115210  _EVP_aes_256_cbc_hmac_sha1
Module: U:\tmp\ldconv_libcrypto_a_99560c9c37f156ab8.lib(e_aes_cbc_hmac_sha256.obj)
0001:00115220  _EVP_aes_128_cbc_hmac_sha256
0001:00115230  _EVP_aes_256_cbc_hmac_sha256
Module: U:\tmp\ldconv_libcrypto_a_99560c9c37f156ab8.lib(e_aria.obj)
0001:001171b0  _EVP_aria_128_cbc
0001:001171c0  _EVP_aria_128_cfb128
0001:001171d0  _EVP_aria_128_ofb
0001:001171e0  _EVP_aria_128_ecb
0001:001171f0  _EVP_aria_192_cbc
0001:00117200  _EVP_aria_192_cfb128
0001:00117210  _EVP_aria_192_ofb
0001:00117220  _EVP_aria_192_ecb
0001:00117230  _EVP_aria_256_cbc
0001:00117240  _EVP_aria_256_cfb128
0001:00117250  _EVP_aria_256_ofb
0001:00117260  _EVP_aria_256_ecb
0001:00117270  _EVP_aria_128_cfb1
0001:00117280  _EVP_aria_192_cfb1
0001:00117290  _EVP_aria_256_cfb1
0001:001172a0  _EVP_aria_128_cfb8
0001:001172b0  _EVP_aria_192_cfb8
0001:001172c0  _EVP_aria_256_cfb8
0001:001172d0  _EVP_aria_128_ctr
0001:001172e0  _EVP_aria_192_ctr
0001:001172f0  _EVP_aria_256_ctr
0001:00117300  _EVP_aria_128_gcm
0001:00117310  _EVP_aria_192_gcm
0001:00117320  _EVP_aria_256_gcm
0001:00117330  _EVP_aria_128_ccm
0001:00117340  _EVP_aria_192_ccm
0001:00117350  _EVP_aria_256_ccm
Module: U:\tmp\ldconv_libcrypto_a_99560c9c37f156ab8.lib(e_camellia.obj)
0001:001180f0  _EVP_camellia_128_cbc
0001:00118100  _EVP_camellia_128_ecb
0001:00118110  _EVP_camellia_128_ofb
0001:00118120  _EVP_camellia_128_cfb128
0001:00118130  _EVP_camellia_128_cfb1
0001:00118140  _EVP_camellia_128_cfb8
0001:00118150  _EVP_camellia_128_ctr
0001:00118160  _EVP_camellia_192_cbc
0001:00118170  _EVP_camellia_192_ecb
0001:00118180  _EVP_camellia_192_ofb
0001:00118190  _EVP_camellia_192_cfb128
0001:001181a0  _EVP_camellia_192_cfb1
0001:001181b0  _EVP_camellia_192_cfb8
0001:001181c0  _EVP_camellia_192_ctr
0001:001181d0  _EVP_camellia_256_cbc
0001:001181e0  _EVP_camellia_256_ecb
0001:001181f0  _EVP_camellia_256_ofb
0001:00118200  _EVP_camellia_256_cfb128
0001:00118210  _EVP_camellia_256_cfb1
0001:00118220  _EVP_camellia_256_cfb8
0001:00118230  _EVP_camellia_256_ctr
Module: U:\tmp\ldconv_libcrypto_a_99560c9c37f156ab8.lib(e_chacha20_poly1305.obj)
0001:0011a2e0  _EVP_chacha20
0001:0011a2f0  _EVP_chacha20_poly1305
Module: U:\tmp\ldconv_libcrypto_a_99560c9c37f156ab8.lib(e_seed.obj)
0001:0011a800  _EVP_seed_cbc
0001:0011a810  _EVP_seed_cfb128
0001:0011a820  _EVP_seed_ofb
0001:0011a830  _EVP_seed_ecb
Module: U:\tmp\ldconv_libcrypto_a_99560c9c37f156ab8.lib(o_names.obj)
0001:0011ac30* _OBJ_NAME_init
0001:0011ac60* _OBJ_NAME_new_index
0001:0011ae90  _OBJ_NAME_get
0001:0011af70  _OBJ_NAME_add
0001:0011b0d0* _OBJ_NAME_remove
0001:0011b1c0  _OBJ_NAME_do_all
0001:0011b200  _OBJ_NAME_do_all_sorted
0001:0011b300  _OBJ_NAME_cleanup
Module: U:\tmp\ldconv_libcrypto_a_99560c9c37f156ab8.lib(m_md5_sha1.obj)
0001:0011b7d0  _EVP_md5_sha1
Module: U:\tmp\ldconv_libssl_a_99560c9c37e1aece0.lib(s3_msg.obj)
0001:0011b840  _ssl3_do_change_cipher_spec
0001:0011b8f0  _ssl3_send_alert
0001:0011ba00  _ssl3_dispatch_alert
Module: U:\tmp\ldconv_libssl_a_99560c9c37e1aece0.lib(statem_clnt.obj)
0001:0011bb90* _tls_construct_client_hello
0001:0011cdb0* _tls_construct_client_key_exchange
0001:0011d6f0* _tls_construct_client_certificate
0001:0011d8a0* _tls_construct_end_of_early_data
0001:0011d900* _tls_construct_next_proto
0001:0011db40  _ossl_statem_client_read_transition
0001:0011e1d0  _ossl_statem_client_write_transition
0001:0011e690  _ossl_statem_client_pre_work
0001:0011e780  _ossl_statem_client_construct_message
0001:0011e9d0  _ossl_statem_client_max_message_size
0001:0011eb20* _dtls_process_hello_verify
0001:0011ec30* _tls_process_server_hello
0001:0011f870* _tls_process_server_certificate
0001:0011ff30* _tls_process_certificate_request
0001:001204f0* _tls_process_new_session_ticket
0001:00120ba0  _tls_process_cert_status_body
0001:00120c20* _tls_process_cert_status
0001:00120ca0  _tls_process_initial_server_flight
0001:00120f20* _tls_process_server_done
0001:00121250* _tls_client_key_exchange_post_work
0001:00121340  _ossl_statem_client_post_work
0001:00121650* _tls_prepare_client_certificate
0001:00121a60  _ossl_statem_client_post_process_message
0001:00121ac0* _ssl3_check_cert_and_algorithm
0001:00121c50* _tls_process_key_exchange
0001:00122bd0  _ossl_statem_client_process_message
0001:00123040* _tls_process_hello_req
0001:00123100* _ssl_do_client_cert_cb
Module: U:\tmp\ldconv_libssl_a_99560c9c37e1aece0.lib(statem_dtls.obj)
0001:001240d0  _dtls1_hm_fragment_free
0001:00124160  _dtls1_do_write
0001:00124650  _dtls_get_message
0001:00124880  _dtls_construct_change_cipher_spec
0001:00124910  _dtls1_read_failed
0001:001249c0* _dtls1_get_queue_priority
0001:001249d0* _dtls1_buffer_message
0001:00124c80* _dtls1_retransmit_message
0001:00124e90  _dtls1_retransmit_buffered_messages
0001:00124f20* _dtls1_set_message_header
0001:00124f90  _dtls1_get_message_header
0001:00125020  _dtls1_set_handshake_header
0001:00125120  _dtls1_close_construct_packet
Module: U:\tmp\ldconv_libssl_a_99560c9c37e1aece0.lib(d1_lib.obj)
0001:001254a0  _dtls1_default_timeout
0001:001254c0  _dtls1_new
0001:001255c0  _dtls1_clear_received_buffer
0001:00125610  _dtls1_clear_sent_buffer
0001:00125660  _dtls1_free
0001:00125750  _dtls1_clear
0001:00125910  _dtls1_start_timer
0001:00125a20* _dtls1_get_timeout
0001:00125af0  _dtls1_is_timer_expired
0001:00125ba0* _dtls1_double_timeout
0001:00125cc0  _dtls1_stop_timer
0001:00125d80  _dtls1_check_timeout_num
0001:00125e60  _dtls1_handle_timeout
0001:00125fd0  _dtls1_ctrl
0001:001260a0* _DTLSv1_listen
0001:00126b90  _dtls1_shutdown
0001:00126ba0  _dtls1_query_mtu
0001:00126d40  _dtls1_min_mtu
0001:00126d80* _DTLS_get_data_mtu
0001:00126e30* _DTLS_set_timer_cb
0001:00126e80  _DTLSv1_2_enc_data
0001:00126ec0  _DTLSv1_enc_data
Module: U:\tmp\ldconv_libssl_a_99560c9c37e1aece0.lib(packet.obj)
0001:00126ff0  _WPACKET_allocate_bytes
0001:001270c0  _WPACKET_sub_allocate_bytes__
0001:00127330  _WPACKET_reserve_bytes
0001:001273f0  _WPACKET_sub_reserve_bytes__
0001:001274d0  _WPACKET_init_static_len
0001:00127680* _WPACKET_init_len
0001:00127870  _WPACKET_init
0001:00127910  _WPACKET_set_flags
0001:00127940  _WPACKET_fill_lengths
0001:001279c0  _WPACKET_close
0001:00127aa0  _WPACKET_finish
0001:00127ba0  _WPACKET_start_sub_packet_len__
0001:00127cd0  _WPACKET_start_sub_packet
0001:00127d60  _WPACKET_put_bytes__
0001:00127e50* _WPACKET_set_max_size
0001:00127ec0  _WPACKET_memset
0001:00127fa0  _WPACKET_memcpy
0001:00128080  _WPACKET_sub_memcpy__
0001:001282c0  _WPACKET_get_total_written
0001:001282f0  _WPACKET_get_length
0001:00128320  _WPACKET_get_curr
0001:00128340  _WPACKET_cleanup
Module: U:\tmp\ldconv_libcrypto_a_99560c9c37f156ab8.lib(o_dir.obj)
0001:00128380  _OPENSSL_DIR_read
0001:00128470  _OPENSSL_DIR_end
Module: U:\tmp\ldconv_libcrypto_a_99560c9c37f156ab8.lib(x_int64.obj)
0001:00128b14  _ZUINT64_it
0001:00128b38  _ZINT64_it
0001:00128b5c  _ZUINT32_it
0001:00128b80  _ZINT32_it
0001:00128ba4* _UINT64_it
0001:00128bc8* _INT64_it
0001:00128bec  _UINT32_it
0001:00128c10  _INT32_it
Module: U:\tmp\ldconv_libcrypto_a_99560c9c37f156ab8.lib(sha1dgst.obj)
0001:00128c30  _SHA1_Update
0001:00128d90  _SHA1_Transform
0001:00128dc0  _SHA1_Final
0001:00128f10  _SHA1_Init
Module: U:\tmp\ldconv_libcrypto_a_99560c9c37f156ab8.lib(sha256.obj)
0001:001290b0  _SHA224_Init
0001:00129120  _SHA256_Init
0001:00129190  _SHA224_Update
0001:001292f0  _SHA256_Update
0001:00129450  _SHA256_Transform
0001:00129480  _SHA256_Final
0001:001296d0* _SHA224
0001:00129790  _SHA256
0001:00129850  _SHA224_Final
Module: U:\tmp\ldconv_libcrypto_a_99560c9c37f156ab8.lib(sha512.obj)
0001:00129860  _sha512_224_init
0001:00129910  _sha512_256_init
0001:001299c0  _SHA384_Init
0001:00129a70  _SHA512_Init
0001:00129b20  _SHA512_Final
0001:00129fa0  _SHA384_Final
0001:0012a420  _SHA512_Update
0001:0012a5d0  _SHA384_Update
0001:0012a780  _SHA512_Transform
0001:0012a7b0* _SHA384
0001:0012aef0  _SHA512
Module: U:\tmp\ldconv_libcrypto_a_99560c9c37f156ab8.lib(cbc128.obj)
0001:0012b630  _CRYPTO_cbc128_encrypt
0001:0012b9d0  _CRYPTO_cbc128_decrypt
Module: U:\tmp\ldconv_libcrypto_a_99560c9c37f156ab8.lib(aes_core.obj)
0001:0012c010  _AES_set_encrypt_key
0001:0012cb70  _AES_set_decrypt_key
0001:0012cdb0  _AES_encrypt
0001:0012d1f0  _AES_decrypt
Module: U:\tmp\ldconv_libcrypto_a_99560c9c37f156ab8.lib(aes_cbc.obj)
0001:0012f750  _AES_cbc_encrypt
Module: U:\tmp\ldconv_libcrypto_a_99560c9c37f156ab8.lib(ofb128.obj)
0001:0012f780  _CRYPTO_ofb128_encrypt
Module: U:\tmp\ldconv_libcrypto_a_99560c9c37f156ab8.lib(cfb128.obj)
0001:0012fb30  _CRYPTO_cfb128_encrypt
0001:001303e0  _CRYPTO_cfb128_1_encrypt
0001:001305e0  _CRYPTO_cfb128_8_encrypt
Module: U:\tmp\ldconv_libcrypto_a_99560c9c37f156ab8.lib(ctr128.obj)
0001:00130720  _CRYPTO_ctr128_encrypt
0001:00130c10  _CRYPTO_ctr128_encrypt_ctr32
Module: U:\tmp\ldconv_libcrypto_a_99560c9c37f156ab8.lib(gcm128.obj)
0001:00131160  _CRYPTO_gcm128_init
0001:00131630  _CRYPTO_gcm128_setiv
0001:00131b30  _CRYPTO_gcm128_aad
0001:00131dc0  _CRYPTO_gcm128_encrypt
0001:00132560  _CRYPTO_gcm128_decrypt
0001:00132d00  _CRYPTO_gcm128_encrypt_ctr32
0001:00133420  _CRYPTO_gcm128_decrypt_ctr32
0001:00133b40  _CRYPTO_gcm128_finish
0001:00133d00  _CRYPTO_gcm128_tag
0001:00133f20* _CRYPTO_gcm128_new
0001:00133f70* _CRYPTO_gcm128_release
Module: U:\tmp\ldconv_libcrypto_a_99560c9c37f156ab8.lib(xts128.obj)
0001:00133fa0  _CRYPTO_xts128_encrypt
Module: U:\tmp\ldconv_libcrypto_a_99560c9c37f156ab8.lib(ccm128.obj)
0001:001349b0  _CRYPTO_ccm128_init
0001:00134a10  _CRYPTO_ccm128_setiv
0001:00134a90  _CRYPTO_ccm128_aad
0001:00134b90  _CRYPTO_ccm128_encrypt
0001:00135290  _CRYPTO_ccm128_decrypt
0001:00135800  _CRYPTO_ccm128_encrypt_ccm64
0001:00136010  _CRYPTO_ccm128_decrypt_ccm64
0001:00136630  _CRYPTO_ccm128_tag
Module: U:\tmp\ldconv_libcrypto_a_99560c9c37f156ab8.lib(wrap128.obj)
0001:00136950  _CRYPTO_128_wrap
0001:001369a0  _CRYPTO_128_unwrap
0001:00136a30  _CRYPTO_128_wrap_pad
0001:00136b30  _CRYPTO_128_unwrap_pad
Module: U:\tmp\ldconv_libcrypto_a_99560c9c37f156ab8.lib(ocb128.obj)
0001:00136ea0  _CRYPTO_ocb128_init
0001:001375b0* _CRYPTO_ocb128_new
0001:00137640  _CRYPTO_ocb128_copy_ctx
0001:00137720  _CRYPTO_ocb128_setiv
0001:00137a70  _CRYPTO_ocb128_aad
0001:00137cd0  _CRYPTO_ocb128_encrypt
0001:00138200  _CRYPTO_ocb128_decrypt
0001:00138750  _CRYPTO_ocb128_finish
0001:00138800  _CRYPTO_ocb128_tag
0001:001388c0  _CRYPTO_ocb128_cleanup
Module: U:\tmp\ldconv_libcrypto_a_99560c9c37f156ab8.lib(evp_asn1.obj)
0001:00138910  _ASN1_TYPE_set_octetstring
0001:00138990  _ASN1_TYPE_get_octetstring
0001:00138a20  _ASN1_TYPE_set_int_octetstring
0001:00138a80  _ASN1_TYPE_get_int_octetstring
Module: U:\tmp\ldconv_libcrypto_a_99560c9c37f156ab8.lib(a_type.obj)
0001:00138bd0  _ASN1_TYPE_get
0001:00138bf0  _ASN1_TYPE_set
0001:00138c60  _ASN1_TYPE_set1
0001:00138db0  _ASN1_TYPE_cmp
0001:00138e20  _ASN1_TYPE_pack_sequence
0001:00138ee0  _ASN1_TYPE_unpack_sequence
Module: U:\tmp\ldconv_libcrypto_a_99560c9c37f156ab8.lib(pmeth_lib.obj)
0001:00138f60  _EVP_PKEY_meth_free
0001:00138fa0* _EVP_PKEY_meth_find
0001:00139030* _EVP_PKEY_meth_new
0001:001390b0* _EVP_PKEY_meth_get0_info
0001:001390d0* _EVP_PKEY_meth_copy
0001:00139230  _EVP_PKEY_CTX_new
0001:001394a0  _EVP_PKEY_CTX_new_id
0001:001396e0  _EVP_PKEY_CTX_dup
0001:00139870* _EVP_PKEY_meth_add0
0001:00139940  _evp_app_cleanup_int
0001:00139970* _EVP_PKEY_meth_remove
0001:001399a0* _EVP_PKEY_meth_get_count
0001:001399d0* _EVP_PKEY_meth_get0
0001:00139a30  _EVP_PKEY_CTX_free
0001:00139a90  _EVP_PKEY_CTX_ctrl
0001:00139c10* _EVP_PKEY_CTX_ctrl_uint64
0001:00139db0* _EVP_PKEY_CTX_ctrl_str
0001:00139ee0  _EVP_PKEY_CTX_str2ctrl
0001:00139f20  _EVP_PKEY_CTX_hex2ctrl
0001:00139fa0  _EVP_PKEY_CTX_md
0001:0013a150* _EVP_PKEY_CTX_get_operation
0001:0013a160  _EVP_PKEY_CTX_set0_keygen_info
0001:0013a180  _EVP_PKEY_CTX_set_data
0001:0013a190  _EVP_PKEY_CTX_get_data
0001:0013a1a0  _EVP_PKEY_CTX_get0_pkey
0001:0013a1b0  _EVP_PKEY_CTX_get0_peerkey
0001:0013a1c0* _EVP_PKEY_CTX_set_app_data
0001:0013a1d0* _EVP_PKEY_CTX_get_app_data
0001:0013a1e0* _EVP_PKEY_meth_set_init
0001:0013a1f0* _EVP_PKEY_meth_set_copy
0001:0013a200* _EVP_PKEY_meth_set_cleanup
0001:0013a210* _EVP_PKEY_meth_set_paramgen
0001:0013a230* _EVP_PKEY_meth_set_keygen
0001:0013a250* _EVP_PKEY_meth_set_sign
0001:0013a270* _EVP_PKEY_meth_set_verify
0001:0013a290* _EVP_PKEY_meth_set_verify_recover
0001:0013a2b0* _EVP_PKEY_meth_set_signctx
0001:0013a2d0* _EVP_PKEY_meth_set_verifyctx
0001:0013a2f0* _EVP_PKEY_meth_set_encrypt
0001:0013a310* _EVP_PKEY_meth_set_decrypt
0001:0013a330* _EVP_PKEY_meth_set_derive
0001:0013a350* _EVP_PKEY_meth_set_ctrl
0001:0013a370* _EVP_PKEY_meth_set_digestsign
0001:0013a380* _EVP_PKEY_meth_set_digestverify
0001:0013a390* _EVP_PKEY_meth_set_check
0001:0013a3a0* _EVP_PKEY_meth_set_public_check
0001:0013a3b0* _EVP_PKEY_meth_set_param_check
0001:0013a3c0* _EVP_PKEY_meth_set_digest_custom
0001:0013a3d0* _EVP_PKEY_meth_get_init
0001:0013a3e0* _EVP_PKEY_meth_get_copy
0001:0013a3f0* _EVP_PKEY_meth_get_cleanup
0001:0013a400* _EVP_PKEY_meth_get_paramgen
0001:0013a430* _EVP_PKEY_meth_get_keygen
0001:0013a460* _EVP_PKEY_meth_get_sign
0001:0013a490* _EVP_PKEY_meth_get_verify
0001:0013a4c0* _EVP_PKEY_meth_get_verify_recover
0001:0013a4f0* _EVP_PKEY_meth_get_signctx
0001:0013a520* _EVP_PKEY_meth_get_verifyctx
0001:0013a550* _EVP_PKEY_meth_get_encrypt
0001:0013a580* _EVP_PKEY_meth_get_decrypt
0001:0013a5b0* _EVP_PKEY_meth_get_derive
0001:0013a5e0* _EVP_PKEY_meth_get_ctrl
0001:0013a610* _EVP_PKEY_meth_get_digestsign
0001:0013a630* _EVP_PKEY_meth_get_digestverify
0001:0013a650* _EVP_PKEY_meth_get_check
0001:0013a670* _EVP_PKEY_meth_get_public_check
0001:0013a690* _EVP_PKEY_meth_get_param_check
0001:0013a6b0* _EVP_PKEY_meth_get_digest_custom
Module: U:\tmp\ldconv_libcrypto_a_99560c9c37f156ab8.lib(a_utf8.obj)
0001:0013a6d0  _UTF8_getc
0001:0013a9d0  _UTF8_putc
Module: U:\tmp\ldconv_libcrypto_a_99560c9c37f156ab8.lib(a_i2d_fp.obj)
0001:0013abe0  _ASN1_i2d_bio
0001:0013acd0  _ASN1_i2d_fp
0001:0013ad70  _ASN1_item_i2d_fp
0001:0013aec0  _ASN1_item_i2d_bio
Module: U:\tmp\ldconv_libcrypto_a_99560c9c37f156ab8.lib(a_d2i_fp.obj)
0001:0013afb0  _asn1_d2i_read_bio
0001:0013b340  _ASN1_d2i_bio
0001:0013b3b0  _ASN1_item_d2i_bio
0001:0013b420  _ASN1_d2i_fp
0001:0013b500  _ASN1_item_d2i_fp
Module: U:\tmp\ldconv_libcrypto_a_99560c9c37f156ab8.lib(p12_sbag.obj)
0001:0013b5e0* _PKCS12_get_attr
0001:0013b5f0  _PKCS12_SAFEBAG_get0_attr
0001:0013b600* _PKCS8_get_attr
0001:0013b630  _PKCS12_SAFEBAG_get0_p8inf
0001:0013b660* _PKCS12_SAFEBAG_get0_pkcs8
0001:0013b690  _PKCS12_SAFEBAG_get0_safes
0001:0013b6c0* _PKCS12_SAFEBAG_get0_type
0001:0013b6d0  _PKCS12_SAFEBAG_get_nid
0001:0013b6e0  _PKCS12_SAFEBAG_get_bag_nid
0001:0013b720  _PKCS12_SAFEBAG_get1_cert
0001:0013b780* _PKCS12_SAFEBAG_get1_crl
0001:0013b7e0* _PKCS12_SAFEBAG_create_cert
0001:0013b810* _PKCS12_SAFEBAG_create_crl
0001:0013b860* _PKCS12_SAFEBAG_create0_p8inf
0001:0013b8c0* _PKCS12_SAFEBAG_create0_pkcs8
0001:0013b920* _PKCS12_SAFEBAG_create_pkcs8_encrypt
Module: U:\tmp\ldconv_libcrypto_a_99560c9c37f156ab8.lib(evp_pkey.obj)
0001:0013ba20  _EVP_PKCS82PKEY
0001:0013bbe0  _EVP_PKEY2PKCS8
0001:0013bd00* _EVP_PKEY_get_attr_count
0001:0013bd10* _EVP_PKEY_get_attr_by_NID
0001:0013bd20* _EVP_PKEY_get_attr_by_OBJ
0001:0013bd30* _EVP_PKEY_get_attr
0001:0013bd40* _EVP_PKEY_delete_attr
0001:0013bd50* _EVP_PKEY_add1_attr
0001:0013bd80* _EVP_PKEY_add1_attr_by_OBJ
0001:0013bdc0* _EVP_PKEY_add1_attr_by_NID
0001:0013be00* _EVP_PKEY_add1_attr_by_txt
Module: U:\tmp\ldconv_libcrypto_a_99560c9c37f156ab8.lib(p12_add.obj)
0001:0013be60  _PKCS12_item_pack_safebag
0001:0013bf50* _PKCS12_pack_p7data
0001:0013c040  _PKCS12_unpack_p7data
0001:0013c0b0* _PKCS12_pack_p7encdata
0001:0013c2c0  _PKCS12_unpack_p7encdata
0001:0013c320  _PKCS12_decrypt_skey
0001:0013c330* _PKCS12_pack_authsafes
0001:0013c370  _PKCS12_unpack_authsafes
Module: U:\tmp\ldconv_libcrypto_a_99560c9c37f156ab8.lib(p8_pkey.obj)
0001:0013c430  _d2i_PKCS8_PRIV_KEY_INFO
0001:0013c624  _PKCS8_PRIV_KEY_INFO_it
0001:0013c460  _i2d_PKCS8_PRIV_KEY_INFO
0001:0013c490  _PKCS8_PRIV_KEY_INFO_new
0001:0013c4b0  _PKCS8_PRIV_KEY_INFO_free
0001:0013c4d0  _PKCS8_pkey_set0
0001:0013c560  _PKCS8_pkey_get0
0001:0013c5c0  _PKCS8_pkey_get0_attrs
0001:0013c5d0  _PKCS8_pkey_add1_attr_by_NID
Module: U:\tmp\ldconv_libcrypto_a_99560c9c37f156ab8.lib(p12_mutl.obj)
0001:0013cb30* _PKCS12_mac_present
0001:0013cb40* _PKCS12_get0_mac
0001:0013cbd0* _PKCS12_gen_mac
0001:0013cc10  _PKCS12_verify_mac
0001:0013cd50* _PKCS12_setup_mac
0001:0013cf60* _PKCS12_set_mac
Module: U:\tmp\ldconv_libcrypto_a_99560c9c37f156ab8.lib(pk7_asn1.obj)
0001:0013d230  _d2i_PKCS7
0001:0013dfd0  _PKCS7_it
0001:0013d260  _i2d_PKCS7
0001:0013d290  _PKCS7_new
0001:0013d2b0  _PKCS7_free
0001:0013d2d0* _i2d_PKCS7_NDEF
0001:0013d300* _PKCS7_dup
0001:0013d320* _d2i_PKCS7_SIGNED
0001:0013df24* _PKCS7_SIGNED_it
0001:0013d350* _i2d_PKCS7_SIGNED
0001:0013d380  _PKCS7_SIGNED_new
0001:0013d3a0  _PKCS7_SIGNED_free
0001:0013d3c0* _d2i_PKCS7_SIGNER_INFO
0001:0013de0c* _PKCS7_SIGNER_INFO_it
0001:0013d3f0* _i2d_PKCS7_SIGNER_INFO
0001:0013d420  _PKCS7_SIGNER_INFO_new
0001:0013d440  _PKCS7_SIGNER_INFO_free
0001:0013d460* _d2i_PKCS7_ISSUER_AND_SERIAL
0001:0013dda4  _PKCS7_ISSUER_AND_SERIAL_it
0001:0013d490* _i2d_PKCS7_ISSUER_AND_SERIAL
0001:0013d4c0* _PKCS7_ISSUER_AND_SERIAL_new
0001:0013d4e0* _PKCS7_ISSUER_AND_SERIAL_free
0001:0013d500* _d2i_PKCS7_ENVELOPE
0001:0013dd28* _PKCS7_ENVELOPE_it
0001:0013d530* _i2d_PKCS7_ENVELOPE
0001:0013d560  _PKCS7_ENVELOPE_new
0001:0013d580* _PKCS7_ENVELOPE_free
0001:0013d5a0* _d2i_PKCS7_RECIP_INFO
0001:0013dc60* _PKCS7_RECIP_INFO_it
0001:0013d5d0* _i2d_PKCS7_RECIP_INFO
0001:0013d600  _PKCS7_RECIP_INFO_new
0001:0013d620  _PKCS7_RECIP_INFO_free
0001:0013d640* _d2i_PKCS7_ENC_CONTENT
0001:0013dbd0* _PKCS7_ENC_CONTENT_it
0001:0013d670* _i2d_PKCS7_ENC_CONTENT
0001:0013d6a0* _PKCS7_ENC_CONTENT_new
0001:0013d6c0* _PKCS7_ENC_CONTENT_free
0001:0013d6e0* _d2i_PKCS7_SIGN_ENVELOPE
0001:0013dacc* _PKCS7_SIGN_ENVELOPE_it
0001:0013d710* _i2d_PKCS7_SIGN_ENVELOPE
0001:0013d740  _PKCS7_SIGN_ENVELOPE_new
0001:0013d760* _PKCS7_SIGN_ENVELOPE_free
0001:0013d780* _d2i_PKCS7_ENCRYPT
0001:0013da50* _PKCS7_ENCRYPT_it
0001:0013d7b0* _i2d_PKCS7_ENCRYPT
0001:0013d7e0  _PKCS7_ENCRYPT_new
0001:0013d800* _PKCS7_ENCRYPT_free
0001:0013d820* _d2i_PKCS7_DIGEST
0001:0013d99c* _PKCS7_DIGEST_it
0001:0013d850* _i2d_PKCS7_DIGEST
0001:0013d880  _PKCS7_DIGEST_new
0001:0013d8a0* _PKCS7_DIGEST_free
0001:0013d8c0* _PKCS7_print_ctx
0001:0013d908  _PKCS7_ATTR_VERIFY_it
0001:0013d95c  _PKCS7_ATTR_SIGN_it
Module: U:\tmp\ldconv_libcrypto_a_99560c9c37f156ab8.lib(x_sig.obj)
0001:0013e190  _d2i_X509_SIG
0001:0013e27c  _X509_SIG_it
0001:0013e1c0  _i2d_X509_SIG
0001:0013e1f0  _X509_SIG_new
0001:0013e210  _X509_SIG_free
0001:0013e230  _X509_SIG_get0
0001:0013e250  _X509_SIG_getm
Module: U:\tmp\ldconv_libcrypto_a_99560c9c37f156ab8.lib(pem_xaux.obj)
0001:0013e310  _PEM_read_bio_X509_AUX
0001:0013e350* _PEM_read_X509_AUX
0001:0013e390* _PEM_write_bio_X509_AUX
0001:0013e3f0* _PEM_write_X509_AUX
Module: U:\tmp\ldconv_libcrypto_a_99560c9c37f156ab8.lib(x_all.obj)
0001:0013e450  _X509_verify
0001:0013e4a0* _X509_REQ_verify
0001:0013e4e0* _NETSCAPE_SPKI_verify
0001:0013e520* _X509_sign
0001:0013e570* _X509_sign_ctx
0001:0013e5b0* _X509_http_nbio
0001:0013e5e0  _X509_REQ_sign
0001:0013e630* _X509_REQ_sign_ctx
0001:0013e670  _X509_CRL_sign
0001:0013e6c0* _X509_CRL_sign_ctx
0001:0013e700* _X509_CRL_http_nbio
0001:0013e730* _NETSCAPE_SPKI_sign
0001:0013e780* _d2i_X509_fp
0001:0013e7b0* _i2d_X509_fp
0001:0013e7e0  _d2i_X509_bio
0001:0013e810* _i2d_X509_bio
0001:0013e840* _d2i_X509_CRL_fp
0001:0013e870* _i2d_X509_CRL_fp
0001:0013e8a0  _d2i_X509_CRL_bio
0001:0013e8d0* _i2d_X509_CRL_bio
0001:0013e900* _d2i_PKCS7_fp
0001:0013e930* _i2d_PKCS7_fp
0001:0013e960* _d2i_PKCS7_bio
0001:0013e990* _i2d_PKCS7_bio
0001:0013e9c0* _d2i_X509_REQ_fp
0001:0013e9f0* _i2d_X509_REQ_fp
0001:0013ea20* _d2i_X509_REQ_bio
0001:0013ea50* _i2d_X509_REQ_bio
0001:0013ea80* _d2i_RSAPrivateKey_fp
0001:0013eab0* _i2d_RSAPrivateKey_fp
0001:0013eae0* _d2i_RSAPublicKey_fp
0001:0013eb10* _d2i_RSA_PUBKEY_fp
0001:0013eb40* _i2d_RSAPublicKey_fp
0001:0013eb70* _i2d_RSA_PUBKEY_fp
0001:0013eba0  _d2i_RSAPrivateKey_bio
0001:0013ebd0* _i2d_RSAPrivateKey_bio
0001:0013ec00* _d2i_RSAPublicKey_bio
0001:0013ec30* _d2i_RSA_PUBKEY_bio
0001:0013ec60* _i2d_RSAPublicKey_bio
0001:0013ec90* _i2d_RSA_PUBKEY_bio
0001:0013ecc0* _d2i_DSAPrivateKey_fp
0001:0013ecf0* _i2d_DSAPrivateKey_fp
0001:0013ed20* _d2i_DSA_PUBKEY_fp
0001:0013ed50* _i2d_DSA_PUBKEY_fp
0001:0013ed80* _d2i_DSAPrivateKey_bio
0001:0013edb0* _i2d_DSAPrivateKey_bio
0001:0013ede0* _d2i_DSA_PUBKEY_bio
0001:0013ee10* _i2d_DSA_PUBKEY_bio
0001:0013ee40* _d2i_EC_PUBKEY_fp
0001:0013ee70* _i2d_EC_PUBKEY_fp
0001:0013eea0* _d2i_ECPrivateKey_fp
0001:0013eed0* _i2d_ECPrivateKey_fp
0001:0013ef00* _d2i_EC_PUBKEY_bio
0001:0013ef30* _i2d_EC_PUBKEY_bio
0001:0013ef60* _d2i_ECPrivateKey_bio
0001:0013ef90* _i2d_ECPrivateKey_bio
0001:0013efc0  _X509_pubkey_digest
0001:0013f010  _X509_digest
0001:0013f0b0  _X509_CRL_digest
0001:0013f140* _X509_REQ_digest
0001:0013f180  _X509_NAME_digest
0001:0013f1c0* _PKCS7_ISSUER_AND_SERIAL_digest
0001:0013f200* _d2i_PKCS8_fp
0001:0013f230* _i2d_PKCS8_fp
0001:0013f260  _d2i_PKCS8_bio
0001:0013f290  _i2d_PKCS8_bio
0001:0013f2c0* _d2i_PKCS8_PRIV_KEY_INFO_fp
0001:0013f2f0* _i2d_PKCS8_PRIV_KEY_INFO_fp
0001:0013f320* _i2d_PKCS8PrivateKeyInfo_fp
0001:0013f370* _i2d_PrivateKey_fp
0001:0013f3a0* _d2i_PrivateKey_fp
0001:0013f3d0* _i2d_PUBKEY_fp
0001:0013f400* _d2i_PUBKEY_fp
0001:0013f430* _d2i_PKCS8_PRIV_KEY_INFO_bio
0001:0013f460  _i2d_PKCS8_PRIV_KEY_INFO_bio
0001:0013f490* _i2d_PKCS8PrivateKeyInfo_bio
0001:0013f4e0* _i2d_PrivateKey_bio
0001:0013f510  _d2i_PrivateKey_bio
0001:0013f540* _i2d_PUBKEY_bio
0001:0013f570* _d2i_PUBKEY_bio
Module: U:\tmp\ldconv_libcrypto_a_99560c9c37f156ab8.lib(pem_all.obj)
0001:0013f5c0* _PEM_read_bio_X509_REQ
0001:0013f600* _PEM_read_X509_REQ
0001:0013f640* _PEM_write_bio_X509_REQ
0001:0013f6a0* _PEM_write_X509_REQ
0001:0013f710* _PEM_write_bio_X509_REQ_NEW
0001:0013f770* _PEM_write_X509_REQ_NEW
0001:0013f7d0  _PEM_read_bio_X509_CRL
0001:0013f810* _PEM_read_X509_CRL
0001:0013f850* _PEM_write_bio_X509_CRL
0001:0013f8b0* _PEM_write_X509_CRL
0001:0013f910* _PEM_read_bio_PKCS7
0001:0013f950* _PEM_read_PKCS7
0001:0013f990* _PEM_write_bio_PKCS7
0001:0013f9f0* _PEM_write_PKCS7
0001:0013fa50* _PEM_read_bio_NETSCAPE_CERT_SEQUENCE
0001:0013fa90* _PEM_read_NETSCAPE_CERT_SEQUENCE
0001:0013fad0* _PEM_write_bio_NETSCAPE_CERT_SEQUENCE
0001:0013fb30* _PEM_write_NETSCAPE_CERT_SEQUENCE
0001:0013fb90  _PEM_read_bio_RSAPrivateKey
0001:0013fc10* _PEM_read_RSAPrivateKey
0001:0013fca0  _PEM_write_bio_RSAPrivateKey
0001:0013fd00* _PEM_write_RSAPrivateKey
0001:0013fd70* _PEM_read_bio_RSAPublicKey
0001:0013fdb0* _PEM_read_RSAPublicKey
0001:0013fdf0* _PEM_write_bio_RSAPublicKey
0001:0013fe50* _PEM_write_RSAPublicKey
0001:0013feb0* _PEM_read_bio_RSA_PUBKEY
0001:0013fef0* _PEM_read_RSA_PUBKEY
0001:0013ff30* _PEM_write_bio_RSA_PUBKEY
0001:0013ff90* _PEM_write_RSA_PUBKEY
0001:0013fff0* _PEM_read_bio_DSAPrivateKey
0001:00140080* _PEM_write_bio_DSAPrivateKey
0001:001400e0* _PEM_write_DSAPrivateKey
0001:00140140* _PEM_read_bio_DSA_PUBKEY
0001:00140180* _PEM_read_DSA_PUBKEY
0001:001401c0* _PEM_write_bio_DSA_PUBKEY
0001:00140220* _PEM_write_DSA_PUBKEY
0001:00140280* _PEM_read_DSAPrivateKey
0001:00140310* _PEM_read_bio_DSAparams
0001:00140350* _PEM_read_DSAparams
0001:00140390* _PEM_write_bio_DSAparams
0001:001403f0* _PEM_write_DSAparams
0001:00140450* _PEM_read_bio_ECPrivateKey
0001:001404e0* _PEM_read_bio_ECPKParameters
0001:00140520* _PEM_read_ECPKParameters
0001:00140560* _PEM_write_bio_ECPKParameters
0001:001405c0* _PEM_write_ECPKParameters
0001:00140630* _PEM_write_bio_ECPrivateKey
0001:00140690* _PEM_write_ECPrivateKey
0001:001406f0* _PEM_read_bio_EC_PUBKEY
0001:00140730* _PEM_read_EC_PUBKEY
0001:00140770* _PEM_write_bio_EC_PUBKEY
0001:001407d0* _PEM_write_EC_PUBKEY
0001:00140830* _PEM_read_ECPrivateKey
0001:001408c0* _PEM_write_bio_DHparams
0001:00140920* _PEM_write_DHparams
0001:00140990* _PEM_write_bio_DHxparams
0001:001409f0* _PEM_write_DHxparams
0001:00140a50* _PEM_read_bio_PUBKEY
0001:00140a90* _PEM_read_PUBKEY
0001:00140ad0* _PEM_write_bio_PUBKEY
0001:00140b30* _PEM_write_PUBKEY
Module: U:\tmp\ldconv_libcrypto_a_99560c9c37f156ab8.lib(rsa_asn1.obj)
0001:00140ca0* _d2i_RSA_PSS_PARAMS
0001:00140f94  _RSA_PSS_PARAMS_it
0001:00140cd0* _i2d_RSA_PSS_PARAMS
0001:00140d00  _RSA_PSS_PARAMS_new
0001:00140d20  _RSA_PSS_PARAMS_free
0001:00140d40* _d2i_RSA_OAEP_PARAMS
0001:00140eec  _RSA_OAEP_PARAMS_it
0001:00140d70* _i2d_RSA_OAEP_PARAMS
0001:00140da0  _RSA_OAEP_PARAMS_new
0001:00140dc0  _RSA_OAEP_PARAMS_free
0001:00140de0  _d2i_RSAPrivateKey
0001:001410e0  _RSAPrivateKey_it
0001:00140e10  _i2d_RSAPrivateKey
0001:00140e40  _d2i_RSAPublicKey
0001:00141068  _RSAPublicKey_it
0001:00140e70  _i2d_RSAPublicKey
0001:00140ea0* _RSAPublicKey_dup
0001:00140ec0* _RSAPrivateKey_dup
0001:00141220* _RSA_PRIME_INFO_it
Module: U:\tmp\ldconv_libcrypto_a_99560c9c37f156ab8.lib(d2i_pr.obj)
0001:001412b0  _d2i_PrivateKey
0001:001414a0  _d2i_AutoPrivateKey
Module: U:\tmp\ldconv_libcrypto_a_99560c9c37f156ab8.lib(ui_null.obj)
0001:001415f0  _UI_null
Module: U:\tmp\ldconv_libcrypto_a_99560c9c37f156ab8.lib(err_prn.obj)
0001:001417f0  _ERR_print_errors_cb
0001:00141970  _ERR_print_errors
0001:00141980* _ERR_print_errors_fp
Module: U:\tmp\ldconv_libssl_a_99560c9c37e1aece0.lib(rec_layer_d1.obj)
0001:00141ef0  _DTLS_RECORD_LAYER_new
0001:00141ff0  _DTLS_RECORD_LAYER_clear
0001:00142150  _DTLS_RECORD_LAYER_free
0001:001421d0  _DTLS_RECORD_LAYER_set_saved_w_epoch
0001:00142270  _DTLS_RECORD_LAYER_set_write_sequence
0001:00142290  _dtls1_buffer_record
0001:00142580  _dtls1_retrieve_buffered_record
0001:001426b0  _dtls1_process_buffered_records
0001:00142980  _dtls1_read_bytes
0001:001432f0  _dtls1_write_bytes
0001:00143410  _do_dtls1_write
0001:001434e0  _dtls1_get_bitmap
0001:00143540  _dtls1_reset_seq_numbers
Module: U:\tmp\ldconv_libssl_a_99560c9c37e1aece0.lib(d1_msg.obj)
0001:001435f0  _dtls1_write_app_data_bytes
0001:001436e0  _dtls1_dispatch_alert
Module: U:\tmp\ldconv_libcrypto_a_99560c9c37f156ab8.lib(p12_p8d.obj)
0001:00143810  _PKCS8_decrypt
Module: U:\tmp\ldconv_libcrypto_a_99560c9c37f156ab8.lib(pem_pk8.obj)
0001:00143b80* _PEM_write_bio_PKCS8PrivateKey_nid
0001:00143bd0  _PEM_write_bio_PKCS8PrivateKey
0001:00143c20* _i2d_PKCS8PrivateKey_bio
0001:00143c70* _i2d_PKCS8PrivateKey_nid_bio
0001:00143cc0* _d2i_PKCS8PrivateKey_bio
0001:00143e00* _i2d_PKCS8PrivateKey_fp
0001:00143eb0* _i2d_PKCS8PrivateKey_nid_fp
0001:00143f60* _PEM_write_PKCS8PrivateKey_nid
0001:00144010* _PEM_write_PKCS8PrivateKey
0001:001440c0* _d2i_PKCS8PrivateKey_fp
0001:00144150* _PEM_read_bio_PKCS8
0001:00144190* _PEM_read_PKCS8
0001:001441d0* _PEM_write_bio_PKCS8
0001:00144230* _PEM_write_PKCS8
0001:00144290* _PEM_read_bio_PKCS8_PRIV_KEY_INFO
0001:001442d0* _PEM_read_PKCS8_PRIV_KEY_INFO
0001:00144310* _PEM_write_bio_PKCS8_PRIV_KEY_INFO
0001:00144370* _PEM_write_PKCS8_PRIV_KEY_INFO
Module: U:\tmp\ldconv_libcrypto_a_99560c9c37f156ab8.lib(i2d_pr.obj)
0001:001443f0  _i2d_PrivateKey
Module: U:\tmp\ldconv_libcrypto_a_99560c9c37f156ab8.lib(dh_asn1.obj)
0001:001444f0  _d2i_DHparams
0001:00144844* _DHparams_it
0001:00144520  _i2d_DHparams
0001:00144550* _d2i_int_dhx
0001:00144580* _i2d_int_dhx
0001:001445c0  _d2i_DHxparams
0001:001446b0  _i2d_DHxparams
Module: U:\tmp\ldconv_libcrypto_a_99560c9c37f156ab8.lib(dh_key.obj)
0001:00144e90  _DH_generate_key
0001:00144ea0  _DH_compute_key
0001:00144f50  _DH_compute_key_padded
0001:00144fe0* _DH_OpenSSL
0001:00144ff0* _DH_set_default_method
0001:00145000  _DH_get_default_method
Module: U:\tmp\ldconv_libcrypto_a_99560c9c37f156ab8.lib(o_time.obj)
0001:00145020  _OPENSSL_gmtime
0001:00145050  _OPENSSL_gmtime_adj
0001:001452b0  _OPENSSL_gmtime_diff
Module: U:\tmp\ldconv_libcrypto_a_99560c9c37f156ab8.lib(a_gentm.obj)
0001:00145510* _asn1_generalizedtime_to_tm
0001:00145530  _ASN1_GENERALIZEDTIME_check
0001:00145560  _ASN1_GENERALIZEDTIME_set_string
0001:001455d0* _ASN1_GENERALIZEDTIME_set
0001:00145610  _ASN1_GENERALIZEDTIME_adj
0001:00145680  _ASN1_GENERALIZEDTIME_print
Module: U:\tmp\ldconv_libcrypto_a_99560c9c37f156ab8.lib(a_utctm.obj)
0001:001456a0* _asn1_utctime_to_tm
0001:001456c0  _ASN1_UTCTIME_check
0001:001456f0  _ASN1_UTCTIME_set_string
0001:00145760* _ASN1_UTCTIME_set
0001:001457a0  _ASN1_UTCTIME_adj
0001:00145810* _ASN1_UTCTIME_cmp_time_t
0001:001458a0  _ASN1_UTCTIME_print
Module: U:\tmp\ldconv_libcrypto_a_99560c9c37f156ab8.lib(v3_info.obj)
0001:00145f0c  _ACCESS_DESCRIPTION_it
0001:00145d40  _ACCESS_DESCRIPTION_free
0001:00145d60* _d2i_ACCESS_DESCRIPTION
0001:00145d90* _i2d_ACCESS_DESCRIPTION
0001:00145dc0  _ACCESS_DESCRIPTION_new
0001:00145de0* _d2i_AUTHORITY_INFO_ACCESS
0001:00145eb8* _AUTHORITY_INFO_ACCESS_it
0001:00145e10* _i2d_AUTHORITY_INFO_ACCESS
0001:00145e40* _AUTHORITY_INFO_ACCESS_new
0001:00145e60  _AUTHORITY_INFO_ACCESS_free
0001:00145e80* _i2a_ACCESS_DESCRIPTION
0001:00145f80  _v3_sinfo
0001:00145fc0  _v3_info
Module: U:\tmp\ldconv_libcrypto_a_99560c9c37f156ab8.lib(a_octet.obj)
0001:00146000  _ASN1_OCTET_STRING_dup
0001:00146010  _ASN1_OCTET_STRING_cmp
0001:00146020  _ASN1_OCTET_STRING_set
Module: U:\tmp\ldconv_libcrypto_a_99560c9c37f156ab8.lib(a_sign.obj)
0001:00146050* _ASN1_sign
0001:00146510  _ASN1_item_sign_ctx
0001:00146930  _ASN1_item_sign
Module: U:\tmp\ldconv_libcrypto_a_99560c9c37f156ab8.lib(asn_pack.obj)
0001:00146a10  _ASN1_item_pack
0001:00146b60  _ASN1_item_unpack
Module: U:\tmp\ldconv_libcrypto_a_99560c9c37f156ab8.lib(b_sock2.obj)
0001:00146c00  _BIO_socket
0001:00146cb0* _BIO_connect
0001:00146f20* _BIO_bind
0001:001470b0  _BIO_listen
0001:00147460  _BIO_accept_ex
0001:00147550  _BIO_closesocket
Module: U:\tmp\ldconv_libcrypto_a_99560c9c37f156ab8.lib(x509_v3.obj)
0001:00147570  _X509v3_get_ext_count
0001:00147590  _X509v3_get_ext_by_NID
0001:00147620  _X509v3_get_ext_by_OBJ
0001:001476a0  _X509v3_get_ext_by_critical
0001:00147730  _X509v3_get_ext
0001:00147770  _X509v3_delete_ext
0001:001477d0  _X509v3_add_ext
0001:001478f0  _X509_EXTENSION_create_by_NID
0001:00147a60  _X509_EXTENSION_create_by_OBJ
0001:00147b60* _X509_EXTENSION_set_object
0001:00147bb0* _X509_EXTENSION_set_critical
0001:00147be0  _X509_EXTENSION_set_data
0001:00147c20  _X509_EXTENSION_get_object
0001:00147c40  _X509_EXTENSION_get_data
0001:00147c60  _X509_EXTENSION_get_critical
Module: U:\tmp\ldconv_libcrypto_a_99560c9c37f156ab8.lib(v3_lib.obj)
0001:00147d10* _X509V3_EXT_add
0001:00147dc0  _X509V3_EXT_get_nid
0001:00147e50  _X509V3_EXT_get
0001:00147f00* _X509V3_EXT_add_list
0001:00147fe0* _X509V3_EXT_add_alias
0001:00148220* _X509V3_EXT_cleanup
0001:00148250* _X509V3_add_standard_extensions
0001:00148260  _X509V3_EXT_d2i
0001:00148370  _X509V3_get_d2i
0001:001484d0  _X509V3_add1_i2d
Module: U:\tmp\ldconv_libcrypto_a_99560c9c37f156ab8.lib(v3_conf.obj)
0001:00148d70* _X509V3_EXT_nconf
0001:00148f60* _X509V3_EXT_nconf_nid
0001:001490e0  _X509V3_EXT_i2d
0001:00149160* _X509V3_EXT_add_nconf_sk
0001:001492c0* _X509V3_EXT_add_nconf
0001:001492e0* _X509V3_EXT_CRL_add_nconf
0001:00149300* _X509V3_EXT_REQ_add_nconf
0001:00149390* _X509V3_get_string
0001:001493f0  _X509V3_get_section
0001:00149450* _X509V3_string_free
0001:00149480  _X509V3_section_free
0001:001494b0  _X509V3_set_nconf
0001:001494d0* _X509V3_set_ctx
0001:00149500* _X509V3_EXT_conf
0001:00149540* _X509V3_EXT_conf_nid
0001:00149580* _X509V3_set_conf_lhash
0001:001495a0* _X509V3_EXT_add_conf
0001:001495f0* _X509V3_EXT_CRL_add_conf
0001:00149640* _X509V3_EXT_REQ_add_conf
Module: U:\tmp\ldconv_libcrypto_a_99560c9c37f156ab8.lib(x_crl.obj)
0001:0014a474  _X509_CRL_INFO_it
0001:00149f60* _d2i_X509_REVOKED
0001:0014a584* _X509_REVOKED_it
0001:00149f90* _i2d_X509_REVOKED
0001:00149fc0* _X509_REVOKED_new
0001:00149fe0  _X509_REVOKED_free
0001:0014a000  _X509_REVOKED_dup
0001:0014a020* _d2i_X509_CRL_INFO
0001:0014a050  _i2d_X509_CRL_INFO
0001:0014a080* _X509_CRL_INFO_new
0001:0014a0a0* _X509_CRL_INFO_free
0001:0014a0c0  _d2i_X509_CRL
0001:0014a3d4  _X509_CRL_it
0001:0014a0f0  _i2d_X509_CRL
0001:0014a120  _X509_CRL_new
0001:0014a140  _X509_CRL_free
0001:0014a160* _X509_CRL_dup
0001:0014a190  _X509_CRL_add0_revoked
0001:0014a210  _X509_CRL_verify
0001:0014a230  _X509_CRL_get0_by_serial
0001:0014a270  _X509_CRL_get0_by_cert
0001:0014a2c0* _X509_CRL_set_default_method
0001:0014a2e0* _X509_CRL_METHOD_new
0001:0014a370* _X509_CRL_METHOD_free
0001:0014a3b0* _X509_CRL_set_meth_data
0001:0014a3c0* _X509_CRL_get_meth_data
Module: U:\tmp\ldconv_libcrypto_a_99560c9c37f156ab8.lib(pcy_tree.obj)
0001:0014a730  _X509_policy_tree_free
0001:0014a750  _X509_policy_check
Module: U:\tmp\ldconv_libcrypto_a_99560c9c37f156ab8.lib(x509_trs.obj)
0001:0014b750* _X509_TRUST_set_default
0001:0014b760  _X509_check_trust
0001:0014b830* _X509_TRUST_get_count
0001:0014b860* _X509_TRUST_get0
0001:0014b8b0  _X509_TRUST_get_by_id
0001:0014b900  _X509_TRUST_set
0001:0014b980* _X509_TRUST_add
0001:0014bc00* _X509_TRUST_cleanup
0001:0014bc30* _X509_TRUST_get_flags
0001:0014bc40* _X509_TRUST_get0_name
0001:0014bc50* _X509_TRUST_get_trust
Module: U:\tmp\ldconv_libcrypto_a_99560c9c37f156ab8.lib(x509cset.obj)
0001:0014bcc0  _X509_CRL_set_version
0001:0014bd10  _X509_CRL_set_issuer_name
0001:0014bd30  _X509_CRL_set1_lastUpdate
0001:0014bd50  _X509_CRL_set1_nextUpdate
0001:0014bd70* _X509_CRL_sort
0001:0014bdd0  _X509_CRL_up_ref
0001:0014bdf0* _X509_CRL_get_version
0001:0014be00  _X509_CRL_get0_lastUpdate
0001:0014be10  _X509_CRL_get0_nextUpdate
0001:0014be20* _X509_CRL_get_lastUpdate
0001:0014be30* _X509_CRL_get_nextUpdate
0001:0014be40  _X509_CRL_get_issuer
0001:0014be50* _X509_CRL_get0_extensions
0001:0014be60  _X509_CRL_get_REVOKED
0001:0014be70* _X509_CRL_get0_signature
0001:0014bea0* _X509_CRL_get_signature_nid
0001:0014beb0* _X509_REVOKED_get0_revocationDate
0001:0014bec0* _X509_REVOKED_set_revocationDate
0001:0014bf10* _X509_REVOKED_get0_serialNumber
0001:0014bf20* _X509_REVOKED_set_serialNumber
0001:0014bf50* _X509_REVOKED_get0_extensions
0001:0014bf60* _i2d_re_X509_CRL_tbs
Module: U:\tmp\ldconv_libcrypto_a_99560c9c37f156ab8.lib(x509name.obj)
0001:0014c110* _X509_NAME_get_text_by_OBJ
0001:0014c210* _X509_NAME_get_text_by_NID
0001:0014c260  _X509_NAME_entry_count
0001:0014c280  _X509_NAME_get_index_by_NID
0001:0014c320* _X509_NAME_get_index_by_OBJ
0001:0014c3a0  _X509_NAME_get_entry
0001:0014c3f0  _X509_NAME_delete_entry
0001:0014c4b0  _X509_NAME_add_entry
0001:0014c650* _X509_NAME_ENTRY_set_object
0001:0014c6d0* _X509_NAME_ENTRY_set_data
0001:0014c7b0* _X509_NAME_ENTRY_create_by_OBJ
0001:0014c890* _X509_NAME_add_entry_by_OBJ
0001:0014c970  _X509_NAME_add_entry_by_txt
0001:0014caa0* _X509_NAME_add_entry_by_NID
0001:0014cbb0* _X509_NAME_ENTRY_create_by_NID
0001:0014cce0* _X509_NAME_ENTRY_create_by_txt
0001:0014ce40  _X509_NAME_ENTRY_get_object
0001:0014ce60  _X509_NAME_ENTRY_get_data
0001:0014ce80  _X509_NAME_ENTRY_set
Module: U:\tmp\ldconv_libcrypto_a_99560c9c37f156ab8.lib(a_verify.obj)
0001:0014ceb0* _ASN1_verify
0001:0014d160  _ASN1_item_verify
Module: U:\tmp\ldconv_libcrypto_a_99560c9c37f156ab8.lib(f_string.obj)
0001:0014d520  _i2a_ASN1_STRING
0001:0014d650* _a2i_ASN1_STRING
Module: U:\tmp\ldconv_libcrypto_a_99560c9c37f156ab8.lib(f_int.obj)
0001:0014d9e0  _i2a_ASN1_INTEGER
0001:0014db50* _a2i_ASN1_INTEGER
0001:0014dee0* _i2a_ASN1_ENUMERATED
0001:0014def0* _a2i_ASN1_ENUMERATED
Module: U:\tmp\ldconv_libcrypto_a_99560c9c37f156ab8.lib(v3_alt.obj)
0001:0014ebb0  _i2v_GENERAL_NAME
0001:0014ef30  _i2v_GENERAL_NAMES
0001:0014f070  _GENERAL_NAME_print
0001:0014f2a0  _v2i_GENERAL_NAMES
0001:0014f8d0  _v2i_GENERAL_NAME
0001:0014fdf0* _a2i_GENERAL_NAME
0001:001502a0  _v2i_GENERAL_NAME_ex
0001:001508c0  _v3_alt
Module: U:\tmp\ldconv_libcrypto_a_99560c9c37f156ab8.lib(v3_prn.obj)
0001:001509a0* _X509V3_EXT_val_prn
0001:00150ba0* _X509V3_EXT_print
0001:00150ee0  _X509V3_extensions_print
0001:00151080* _X509V3_EXT_print_fp
Module: U:\tmp\ldconv_libcrypto_a_99560c9c37f156ab8.lib(t_x509.obj)
0001:001514b0* _X509_ocspid_print
0001:001516b0  _X509_signature_dump
0001:001517b0  _X509_signature_print
0001:00151a60* _X509_print_ex
0001:001521c0* _X509_print_ex_fp
0001:00152270  _X509_print
0001:001522a0* _X509_print_fp
0001:00152350* _X509_aux_print
Module: U:\tmp\ldconv_libcrypto_a_99560c9c37f156ab8.lib(asn1_par.obj)
0001:00153100* _ASN1_parse
0001:00153140  _ASN1_parse_dump
0001:00153180  _ASN1_tag2str
Module: U:\tmp\ldconv_libcrypto_a_99560c9c37f156ab8.lib(a_mbstr.obj)
0001:00153580  _ASN1_mbstring_ncopy
0001:00154180  _ASN1_mbstring_copy
Module: U:\tmp\ldconv_libcrypto_a_99560c9c37f156ab8.lib(x509_req.obj)
0001:001541f0* _X509_to_X509_REQ
0001:001542f0* _X509_REQ_get_pubkey
0001:00154310* _X509_REQ_get0_pubkey
0001:00154330* _X509_REQ_get_X509_PUBKEY
0001:00154340* _X509_REQ_check_private_key
0001:001544d0* _X509_REQ_extension_nid
0001:00154510* _X509_REQ_get_extension_nids
0001:00154520* _X509_REQ_set_extension_nids
0001:00154530  _X509_REQ_get_extensions
0001:001545f0* _X509_REQ_add_extensions_nid
0001:00154680  _X509_REQ_add_extensions
0001:00154710* _X509_REQ_get_attr_count
0001:00154720* _X509_REQ_get_attr_by_NID
0001:00154730* _X509_REQ_get_attr_by_OBJ
0001:00154740* _X509_REQ_get_attr
0001:00154750* _X509_REQ_delete_attr
0001:00154760* _X509_REQ_add1_attr
0001:00154790* _X509_REQ_add1_attr_by_OBJ
0001:001547d0* _X509_REQ_add1_attr_by_NID
0001:00154810* _X509_REQ_add1_attr_by_txt
0001:00154850* _X509_REQ_get_version
0001:00154860  _X509_REQ_get_subject_name
0001:00154870* _X509_REQ_get0_signature
0001:001548a0* _X509_REQ_set0_signature
0001:001548d0* _X509_REQ_set1_signature_algo
0001:001548e0* _X509_REQ_get_signature_nid
0001:001548f0* _i2d_re_X509_REQ_tbs
Module: U:\tmp\ldconv_libcrypto_a_99560c9c37f156ab8.lib(pem_info.obj)
0001:00154980  _PEM_X509_INFO_read_bio
0001:00154fa0* _PEM_X509_INFO_read
0001:00155040* _PEM_X509_INFO_write_bio
Module: U:\tmp\ldconv_libcrypto_a_99560c9c37f156ab8.lib(x_info.obj)
0001:001552a0  _X509_INFO_new
0001:00155310  _X509_INFO_free
Module: U:\tmp\ldconv_libcrypto_a_99560c9c37f156ab8.lib(x509_def.obj)
0001:001553a0* _X509_get_default_private_dir
0001:001553c0  _X509_get_default_cert_area
0001:001553e0  _X509_get_default_cert_dir
0001:00155400  _X509_get_default_cert_file
0001:00155420  _X509_get_default_cert_dir_env
0001:00155440  _X509_get_default_cert_file_env
Module: U:\tmp\ldconv_libcrypto_a_99560c9c37f156ab8.lib(bn_prime.obj)
0001:001559c0  _BN_GENCB_call
0001:00155a50  _BN_generate_prime_ex
0001:00156540  _BN_is_prime_ex
0001:001565e0  _BN_is_prime_fasttest_ex
Module: U:\tmp\ldconv_libgcc_eh_a_99560c9c382174360.lib(emx-ctordtor.obj)
0001:00157690  ___ctordtorInit
0001:001576c4  ___ctordtorTerm
Module: U:\tmp\ldconv_libcrypto_a_99560c9c37f156ab8.lib(drbg_ctr.obj)
0001:001596b0  _drbg_ctr_init
Module: U:\tmp\ldconv_libcrypto_a_99560c9c37f156ab8.lib(eng_table.obj)
0001:00159a60* _ENGINE_get_table_flags
0001:00159a70* _ENGINE_set_table_flags
0001:00159a80  _engine_table_register
0001:00159cd0  _engine_table_unregister
0001:00159d20  _engine_table_cleanup
0001:00159d70  _engine_table_select
0001:00159e90  _engine_table_doall
Module: U:\tmp\ldconv_libcrypto_a_99560c9c37f156ab8.lib(obj_xref.obj)
0001:00159f90  _OBJ_find_sigid_algs
0001:0015a030  _OBJ_find_sigid_by_algs
0001:0015a0e0* _OBJ_add_sigid
0001:0015a240  _OBJ_sigid_free
Module: U:\tmp\ldconv_libcrypto_a_99560c9c37f156ab8.lib(rsa_crpt.obj)
0001:0015a590  _RSA_bits
0001:0015a5a0  _RSA_size
0001:0015a5d0  _RSA_public_encrypt
0001:0015a5e0  _RSA_private_encrypt
0001:0015a5f0  _RSA_private_decrypt
0001:0015a600  _RSA_public_decrypt
0001:0015a610  _RSA_flags
0001:0015a630* _RSA_blinding_off
0001:0015a670  _RSA_setup_blinding
0001:0015a930* _RSA_blinding_on
Module: U:\tmp\ldconv_libcrypto_a_99560c9c37f156ab8.lib(bn_const.obj)
0001:0015a990* _BN_get_rfc2409_prime_768
0001:0015a9c0  _BN_get_rfc2409_prime_1024
0001:0015a9f0* _BN_get_rfc3526_prime_1536
0001:0015aa20  _BN_get_rfc3526_prime_2048
0001:0015aa50  _BN_get_rfc3526_prime_3072
0001:0015aa80  _BN_get_rfc3526_prime_4096
0001:0015aab0* _BN_get_rfc3526_prime_6144
0001:0015aae0  _BN_get_rfc3526_prime_8192
Module: U:\tmp\ldconv_libssl_a_99560c9c37e1aece0.lib(ssl3_record_tls13.obj)
0001:0015b850  _tls13_enc
Module: U:\tmp\ldconv_libssl_a_99560c9c37e1aece0.lib(ssl3_record.obj)
0001:0015be70  _SSL3_RECORD_clear
0001:0015bee0  _SSL3_RECORD_release
0001:0015bf30  _SSL3_RECORD_set_seq_num
0001:0015bf50  _early_data_count_ok
0001:0015c080* _ssl3_do_uncompress
0001:0015c110  _ssl3_do_compress
0001:0015c170  _ssl3_enc
0001:0015c3d0  _n_ssl3_mac
0001:0015c770  _tls1_mac
0001:0015ca80* _ssl3_cbc_remove_padding
0001:0015caf0* _tls1_cbc_remove_padding
0001:0015cc60  _tls1_enc
0001:0015d5d0* _ssl3_cbc_copy_mac
0001:0015d780  _ssl3_get_record
0001:0015e8b0  _dtls1_process_record
0001:0015eed0  _dtls1_get_record
0001:0015f230  _dtls_buffer_listen_record
Module: U:\tmp\ldconv_libssl_a_99560c9c37e1aece0.lib(t1_enc.obj)
0001:0015f680  _tls1_change_cipher_state
0001:0015fed0  _tls1_setup_key_block
0001:00160120  _tls1_final_finish_mac
0001:00160230  _tls1_generate_master_secret
0001:001603f0  _tls1_export_keying_material
0001:00160790  _tls1_alert_code
Module: U:\tmp\ldconv_libcrypto_a_99560c9c37f156ab8.lib(m_sigver.obj)
0001:00160890  _EVP_DigestSignInit
0001:00160a80  _EVP_DigestVerifyInit
0001:00160c70  _EVP_DigestSignFinal
0001:00160f70  _EVP_DigestSign
0001:00160fe0  _EVP_DigestVerifyFinal
0001:00161160  _EVP_DigestVerify
Module: U:\tmp\ldconv_libssl_a_99560c9c37e1aece0.lib(extensions_srvr.obj)
0001:001611f0  _tls_parse_ctos_renegotiate
0001:00161310  _tls_parse_ctos_server_name
0001:00161560  _tls_parse_ctos_maxfragmentlen
0001:00161650  _tls_parse_ctos_srp
0001:00161770  _tls_parse_ctos_ec_pt_formats
0001:001618b0  _tls_parse_ctos_session_ticket
0001:00161930  _tls_parse_ctos_sig_algs_cert
0001:00161a20  _tls_parse_ctos_sig_algs
0001:00161b10  _tls_parse_ctos_status_request
0001:00161e30  _tls_parse_ctos_npn
0001:00161e60  _tls_parse_ctos_alpn
0001:00162010  _tls_parse_ctos_use_srtp
0001:001621d0  _tls_parse_ctos_etm
0001:001621f0  _tls_parse_ctos_psk_kex_modes
0001:001622c0  _tls_parse_ctos_key_share
0001:001626a0  _tls_parse_ctos_cookie
0001:00162e80  _tls_parse_ctos_supported_groups
0001:00162fe0  _tls_parse_ctos_ems
0001:00163050  _tls_parse_ctos_early_data
0001:001630f0  _tls_parse_ctos_psk
0001:00163950  _tls_parse_ctos_post_handshake_auth
0001:001639c0  _tls_construct_stoc_renegotiate
0001:00163ad0  _tls_construct_stoc_server_name
0001:00163bb0  _tls_construct_stoc_maxfragmentlen
0001:00163c90  _tls_construct_stoc_ec_pt_formats
0001:00163da0  _tls_construct_stoc_supported_groups
0001:00163fa0  _tls_construct_stoc_session_ticket
0001:00164060  _tls_construct_stoc_status_request
0001:00164190  _tls_construct_stoc_next_proto_neg
0001:001642a0  _tls_construct_stoc_alpn
0001:001643b0  _tls_construct_stoc_use_srtp
0001:001644c0  _tls_construct_stoc_etm
0001:001645a0  _tls_construct_stoc_ems
0001:00164640  _tls_construct_stoc_supported_versions
0001:00164760  _tls_construct_stoc_key_share
0001:00164a90  _tls_construct_stoc_cookie
0001:00164fd0  _tls_construct_stoc_cryptopro_bug
0001:001650b0  _tls_construct_stoc_early_data
0001:001651f0  _tls_construct_stoc_psk
Module: U:\tmp\ldconv_libssl_a_99560c9c37e1aece0.lib(extensions_clnt.obj)
0001:001652e0  _tls_construct_ctos_renegotiate
0001:001653c0  _tls_construct_ctos_server_name
0001:001654e0  _tls_construct_ctos_maxfragmentlen
0001:001655b0  _tls_construct_ctos_srp
0001:001656c0  _tls_construct_ctos_ec_pt_formats
0001:00165830  _tls_construct_ctos_supported_groups
0001:00165a20  _tls_construct_ctos_session_ticket
0001:00165bd0  _tls_construct_ctos_sig_algs
0001:00165d20  _tls_construct_ctos_status_request
0001:00165f90  _tls_construct_ctos_npn
0001:00166060  _tls_construct_ctos_alpn
0001:00166170  _tls_construct_ctos_use_srtp
0001:001662d0  _tls_construct_ctos_etm
0001:00166390  _tls_construct_ctos_sct
0001:00166440  _tls_construct_ctos_ems
0001:001664d0  _tls_construct_ctos_supported_versions
0001:00166630  _tls_construct_ctos_psk_kex_modes
0001:00166760  _tls_construct_ctos_key_share
0001:00166ab0  _tls_construct_ctos_cookie
0001:00166bc0  _tls_construct_ctos_early_data
0001:00167120  _tls_construct_ctos_padding
0001:001672c0  _tls_construct_ctos_psk
0001:001678b0  _tls_construct_ctos_post_handshake_auth
0001:00167960  _tls_parse_stoc_renegotiate
0001:00167b80  _tls_parse_stoc_maxfragmentlen
0001:00167c60  _tls_parse_stoc_server_name
0001:00167db0  _tls_parse_stoc_ec_pt_formats
0001:00167f40  _tls_parse_stoc_session_ticket
0001:00168070  _tls_parse_stoc_status_request
0001:001681b0  _tls_parse_stoc_sct
0001:001683a0  _tls_parse_stoc_npn
0001:00168610  _tls_parse_stoc_alpn
0001:001688c0  _tls_parse_stoc_use_srtp
0001:00168a40  _tls_parse_stoc_etm
0001:00168a80  _tls_parse_stoc_ems
0001:00168ab0  _tls_parse_stoc_supported_versions
0001:00168b80  _tls_parse_stoc_key_share
0001:00168ef0  _tls_parse_stoc_cookie
0001:00168ff0  _tls_parse_stoc_early_data
0001:00169110  _tls_parse_stoc_psk
Module: U:\tmp\ldconv_libcrypto_a_99560c9c37f156ab8.lib(async_null.obj)
0001:00169350* _ASYNC_is_capable
0001:00169360  _async_local_cleanup
Module: U:\tmp\ldconv_libcrypto_a_99560c9c37f156ab8.lib(ct_sct_ctx.obj)
0001:00169390  _SCT_CTX_new
0001:00169400  _SCT_CTX_free
0001:001694b0  _SCT_CTX_set1_cert
0001:00169830* _SCT_CTX_set1_issuer
0001:00169970  _SCT_CTX_set1_issuer_pubkey
0001:00169aa0  _SCT_CTX_set1_pubkey
0001:00169c20  _SCT_CTX_set_time
Module: U:\tmp\ldconv_libcrypto_a_99560c9c37f156ab8.lib(ct_vfy.obj)
0001:00169c60  _SCT_CTX_verify
Module: U:\tmp\ldconv_libcrypto_a_99560c9c37f156ab8.lib(ct_b64.obj)
0001:0016a130* _SCT_new_from_base64
0001:0016a360  _CTLOG_new_from_base64
Module: U:\tmp\ldconv_libcrypto_a_99560c9c37f156ab8.lib(srp_lib.obj)
0001:0016a600  _SRP_Calc_u
0001:0016a740  _SRP_Calc_server_key
0001:0016a850  _SRP_Calc_B
0001:0016a9d0  _SRP_Calc_x
0001:0016abe0  _SRP_Calc_A
0001:0016ac70  _SRP_Calc_client_key
0001:0016af00  _SRP_Verify_B_mod_N
0001:0016afa0  _SRP_Verify_A_mod_N
0001:0016b040  _SRP_check_known_gN_param
0001:0016b0b0  _SRP_get_default_gN
Module: U:\tmp\ldconv_libcrypto_a_99560c9c37f156ab8.lib(srp_vfy.obj)
0001:0016b770* _SRP_user_pwd_free
0001:0016b7f0* _SRP_VBASE_new
0001:0016b8e0* _SRP_VBASE_free
0001:0016b950* _SRP_VBASE_init
0001:0016bea0* _SRP_VBASE_get_by_user
0001:0016bf00* _SRP_VBASE_get1_by_user
0001:0016c240  _SRP_create_verifier_BN
0001:0016c400* _SRP_create_verifier
Module: U:\tmp\ldconv_libcrypto_a_99560c9c37f156ab8.lib(evp_pbe.obj)
0001:0016c850  _EVP_PBE_CipherInit
0001:0016cb10* _EVP_PBE_alg_add_type
0001:0016cc00* _EVP_PBE_alg_add
0001:0016cd10  _EVP_PBE_find
0001:0016cde0  _EVP_PBE_cleanup
0001:0016ce10* _EVP_PBE_get
Module: U:\tmp\ldconv_libssl_a_99560c9c37e1aece0.lib(s3_enc.obj)
0001:0016d0c0  _ssl3_change_cipher_state
0001:0016d500  _ssl3_setup_key_block
0001:0016dae0  _ssl3_cleanup_key_block
0001:0016db30  _ssl3_init_finished_mac
0001:0016dc00  _ssl3_free_digest_list
0001:0016dc50  _ssl3_finish_mac
0001:0016dd60  _ssl3_digest_cached_records
0001:0016def0  _ssl3_final_finish_mac
0001:0016e1f0  _ssl3_generate_master_secret
0001:0016e470  _ssl3_alert_code
Module: U:\tmp\ldconv_libcrypto_a_99560c9c37f156ab8.lib(pmeth_fn.obj)
0001:0016e550  _EVP_PKEY_sign_init
0001:0016e5e0  _EVP_PKEY_sign
0001:0016e760  _EVP_PKEY_verify_init
0001:0016e7f0  _EVP_PKEY_verify
0001:0016e880* _EVP_PKEY_verify_recover_init
0001:0016e910* _EVP_PKEY_verify_recover
0001:0016ea90  _EVP_PKEY_encrypt_init
0001:0016eb20  _EVP_PKEY_encrypt
0001:0016ecb0  _EVP_PKEY_decrypt_init
0001:0016ed40  _EVP_PKEY_decrypt
0001:0016eed0  _EVP_PKEY_derive_init
0001:0016ef60  _EVP_PKEY_derive_set_peer
0001:0016f1a0  _EVP_PKEY_derive
Module: U:\tmp\ldconv_libcrypto_a_99560c9c37f156ab8.lib(conf_ssl.obj)
0001:0016f7a0  _conf_ssl_get
0001:0016f7d0  _conf_ssl_name_find
0001:0016f840  _conf_ssl_get_cmd
0001:0016f870  _conf_add_ssl_module
Module: U:\tmp\ldconv_libcrypto_a_99560c9c37f156ab8.lib(v3_bcons.obj)
0001:0016fb50* _BASIC_CONSTRAINTS_it
0001:0016faa0* _d2i_BASIC_CONSTRAINTS
0001:0016fad0* _i2d_BASIC_CONSTRAINTS
0001:0016fb00* _BASIC_CONSTRAINTS_new
0001:0016fb20  _BASIC_CONSTRAINTS_free
0001:0016fbc0  _v3_bcons
Module: U:\tmp\ldconv_libcrypto_a_99560c9c37f156ab8.lib(v3_pcia.obj)
0001:0016fc00* _d2i_PROXY_POLICY
0001:0016fdd8* _PROXY_POLICY_it
0001:0016fc30* _i2d_PROXY_POLICY
0001:0016fc60* _PROXY_POLICY_new
0001:0016fc80* _PROXY_POLICY_free
0001:0016fca0* _d2i_PROXY_CERT_INFO_EXTENSION
0001:0016fd58  _PROXY_CERT_INFO_EXTENSION_it
0001:0016fcd0* _i2d_PROXY_CERT_INFO_EXTENSION
0001:0016fd00  _PROXY_CERT_INFO_EXTENSION_new
0001:0016fd20  _PROXY_CERT_INFO_EXTENSION_free
Module: U:\tmp\ldconv_libcrypto_a_99560c9c37f156ab8.lib(md5_dgst.obj)
0001:0016fe60  _MD5_Update
0001:0016ffc0  _MD5_Transform
0001:0016fff0  _MD5_Final
0001:00170130  _MD5_Init
Module: U:\tmp\ldconv_libcrypto_a_99560c9c37f156ab8.lib(a_bitstr.obj)
0001:00170180  _ASN1_BIT_STRING_set
0001:00170190  _i2c_ASN1_BIT_STRING
0001:00170380  _c2i_ASN1_BIT_STRING
0001:00170540  _ASN1_BIT_STRING_set_bit
0001:00170680  _ASN1_BIT_STRING_get_bit
0001:001706d0* _ASN1_BIT_STRING_check
Module: U:\tmp\ldconv_libcrypto_a_99560c9c37f156ab8.lib(pcy_data.obj)
0001:00170760  _policy_data_free
0001:001707d0  _policy_data_new
Module: U:\tmp\ldconv_libcrypto_a_99560c9c37f156ab8.lib(v3_cpols.obj)
0001:00170910  _POLICYINFO_free
0001:00172068* _POLICYINFO_it
0001:00171f88* _POLICYQUALINFO_it
0001:00171f04* _USERNOTICE_it
0001:00171e90* _NOTICEREF_it
0001:00171a90* _d2i_CERTIFICATEPOLICIES
0001:001720ec* _CERTIFICATEPOLICIES_it
0001:00171ac0* _i2d_CERTIFICATEPOLICIES
0001:00171af0* _CERTIFICATEPOLICIES_new
0001:00171b10* _CERTIFICATEPOLICIES_free
0001:00171b30* _d2i_POLICYINFO
0001:00171b60* _i2d_POLICYINFO
0001:00171b90* _POLICYINFO_new
0001:00171bb0* _d2i_POLICYQUALINFO
0001:00171be0* _i2d_POLICYQUALINFO
0001:00171c10* _POLICYQUALINFO_new
0001:00171c30  _POLICYQUALINFO_free
0001:00171c50* _d2i_USERNOTICE
0001:00171c80* _i2d_USERNOTICE
0001:00171cb0* _USERNOTICE_new
0001:00171cd0* _USERNOTICE_free
0001:00171cf0* _d2i_NOTICEREF
0001:00171d20* _i2d_NOTICEREF
0001:00171d50* _NOTICEREF_new
0001:00171d70* _NOTICEREF_free
0001:00171dc0* _X509_POLICY_NODE_print
0001:00172130  _v3_cpols
Module: U:\tmp\ldconv_libcrypto_a_99560c9c37f156ab8.lib(v3_pcons.obj)
0001:00172450* _POLICY_CONSTRAINTS_it
0001:00172400* _POLICY_CONSTRAINTS_new
0001:00172420  _POLICY_CONSTRAINTS_free
0001:001724b0  _v3_policy_constraints
Module: U:\tmp\ldconv_libcrypto_a_99560c9c37f156ab8.lib(pcy_map.obj)
0001:001724f0  _policy_cache_set_mapping
Module: U:\tmp\ldconv_libcrypto_a_99560c9c37f156ab8.lib(tasn_utl.obj)
0001:00172660  _asn1_get_choice_selector
0001:00172680  _asn1_set_choice_selector
0001:001726b0  _asn1_do_lock
0001:001727a0  _asn1_enc_init
0001:001727e0  _asn1_enc_free
0001:00172840  _asn1_enc_save
0001:00172920  _asn1_enc_restore
0001:001729a0  _asn1_get_field_ptr
0001:001729b0  _asn1_do_adb
Module: U:\tmp\ldconv_libcrypto_a_99560c9c37f156ab8.lib(pmeth_gn.obj)
0001:00172b00  _EVP_PKEY_paramgen_init
0001:00172b90  _EVP_PKEY_paramgen
0001:00172cd0  _EVP_PKEY_keygen_init
0001:00172d60  _EVP_PKEY_keygen
0001:00172e60* _EVP_PKEY_CTX_set_cb
0001:00172e70* _EVP_PKEY_CTX_get_cb
0001:00172e80  _evp_pkey_set_cb_translate
0001:00172eb0* _EVP_PKEY_CTX_get_keygen_info
0001:00172ee0  _EVP_PKEY_new_mac_key
0001:00172fc0* _EVP_PKEY_check
0001:00173060* _EVP_PKEY_public_check
0001:00173100* _EVP_PKEY_param_check
Module: U:\tmp\ldconv_libcrypto_a_99560c9c37f156ab8.lib(rsa_ameth.obj)
0001:001746e0  _rsa_pss_params_create
0001:00174a30  _rsa_pss_get_param
0001:00175dc0  _rsa_pss_asn1_meth
0001:00175e80  _rsa_asn1_meths
Module: U:\tmp\ldconv_libcrypto_a_99560c9c37f156ab8.lib(dh_ameth.obj)
0001:00178760  _dhx_asn1_meth
0001:001776a0* _DHparams_dup
0001:001783f0* _DHparams_print
0001:00178820  _dh_asn1_meth
Module: U:\tmp\ldconv_libcrypto_a_99560c9c37f156ab8.lib(dsa_ameth.obj)
0001:00179a80  _dsa_asn1_meths
Module: U:\tmp\ldconv_libcrypto_a_99560c9c37f156ab8.lib(ec_ameth.obj)
0001:0017be70  _EC_KEY_print
0001:0017c150  _ECParameters_print
0001:0017c2a0  _sm2_asn1_meth
0001:0017c360  _eckey_asn1_meth
Module: U:\tmp\ldconv_libcrypto_a_99560c9c37f156ab8.lib(hm_ameth.obj)
0001:0017c600  _hmac_asn1_meth
Module: U:\tmp\ldconv_libcrypto_a_99560c9c37f156ab8.lib(cm_ameth.obj)
0001:0017c700  _cmac_asn1_meth
Module: U:\tmp\ldconv_libcrypto_a_99560c9c37f156ab8.lib(ecx_meth.obj)
0001:0017e840  _ed448_pkey_meth
0001:0017e8e0  _ed25519_pkey_meth
0001:0017e980  _ecx448_pkey_meth
0001:0017ea20  _ecx25519_pkey_meth
0001:0017eae0  _ed448_asn1_meth
0001:0017eba0  _ed25519_asn1_meth
0001:0017ec60  _ecx448_asn1_meth
0001:0017ed20  _ecx25519_asn1_meth
Module: U:\tmp\ldconv_libcrypto_a_99560c9c37f156ab8.lib(poly1305_ameth.obj)
0001:0017ef80  _poly1305_asn1_meth
Module: U:\tmp\ldconv_libcrypto_a_99560c9c37f156ab8.lib(siphash_ameth.obj)
0001:0017f1e0  _siphash_asn1_meth
Module: U:\tmp\ldconv_libcrypto_a_99560c9c37f156ab8.lib(dso_lib.obj)
0001:0017f2a0  _DSO_free
0001:0017f570  _DSO_new
0001:0017f580* _DSO_flags
0001:0017f590* _DSO_up_ref
0001:0017f5f0  _DSO_bind_func
0001:0017f6d0  _DSO_ctrl
0001:0017f7a0* _DSO_get_filename
0001:0017f7f0* _DSO_set_filename
0001:0017f910  _DSO_load
0001:0017fb00  _DSO_merge
0001:0017fb70  _DSO_convert_filename
0001:0017fca0* _DSO_pathbyaddr
0001:0017fd20* _DSO_dsobyaddr
0001:0017fe80* _DSO_global_lookup
Module: U:\tmp\ldconv_libgcc_a_99560c9c382191438.lib(_udivmoddi4.obj)
0001:0017fef0  ___udivmoddi4
Module: U:\tmp\ldconv_libcrypto_a_99560c9c37f156ab8.lib(rsa_mp.obj)
0001:001800d0  _rsa_multip_info_free_ex
0001:00180100  _rsa_multip_info_free
0001:00180150  _rsa_multip_info_new
0001:00180240  _rsa_multip_calc_product
0001:00180320  _rsa_multip_cap
Module: U:\tmp\ldconv_libcrypto_a_99560c9c37f156ab8.lib(bn_blind.obj)
0001:00180370* _BN_BLINDING_new
0001:00180520  _BN_BLINDING_free
0001:00180580* _BN_BLINDING_invert
0001:00180670  _BN_BLINDING_invert_ex
0001:00180780  _BN_BLINDING_is_current_thread
0001:001807b0  _BN_BLINDING_set_current_thread
0001:001807d0  _BN_BLINDING_lock
0001:001807e0  _BN_BLINDING_unlock
0001:001807f0* _BN_BLINDING_get_flags
0001:00180800* _BN_BLINDING_set_flags
0001:00180810  _BN_BLINDING_create_param
0001:00180a90* _BN_BLINDING_update
0001:00180c40  _BN_BLINDING_convert_ex
0001:00180d40* _BN_BLINDING_convert
Module: U:\tmp\ldconv_libcrypto_a_99560c9c37f156ab8.lib(rsa_ossl.obj)
0001:001830b0* _RSA_set_default_method
0001:001830c0  _RSA_get_default_method
0001:001830d0* _RSA_PKCS1_OpenSSL
0001:001830e0* _RSA_null_method
Module: U:\tmp\ldconv_libcrypto_a_99560c9c37f156ab8.lib(dsa_ossl.obj)
0001:001842d0* _DSA_set_default_method
0001:001842e0  _DSA_get_default_method
0001:001842f0* _DSA_OpenSSL
Module: U:\tmp\ldconv_libcrypto_a_99560c9c37f156ab8.lib(b_dump.obj)
0001:001845d0* _BIO_dump_cb
0001:001845f0* _BIO_dump_indent_cb
0001:001848f0* _BIO_dump_fp
0001:00184910* _BIO_dump_indent_fp
0001:00184950  _BIO_dump
0001:00184970  _BIO_dump_indent
0001:001849c0  _BIO_hex_string
Module: U:\tmp\ldconv_libgcc_a_99560c9c382191438.lib(_umoddi3.obj)
0001:00184ab0  ___umoddi3
Module: U:\tmp\ldconv_libcrypto_a_99560c9c37f156ab8.lib(bn-586.obj)
0001:00184bd0  _bn_mul_add_words
0001:00184d60  _bn_mul_words
0001:00184e90  _bn_sqr_words
0001:00184f80  _bn_div_words
0001:00184f90  _bn_add_words
0001:00185140  _bn_sub_words
0001:001852f0  _bn_sub_part_words
Module: U:\tmp\ldconv_libcrypto_a_99560c9c37f156ab8.lib(ecdh_ossl.obj)
0001:00185890  _ossl_ecdh_compute_key
0001:001858f0  _ecdh_simple_compute_key
Module: U:\tmp\ldconv_libcrypto_a_99560c9c37f156ab8.lib(ecdsa_ossl.obj)
0001:00185ce0  _ossl_ecdsa_sign
0001:00185d70  _ossl_ecdsa_sign_setup
0001:001861b0  _ossl_ecdsa_sign_sig
0001:00186c40  _ossl_ecdsa_verify
0001:00186d40  _ossl_ecdsa_verify_sig
Module: U:\tmp\ldconv_libcrypto_a_99560c9c37f156ab8.lib(ec2_oct.obj)
0001:001872f0  _ec_GF2m_simple_set_compressed_coordinates
0001:001875f0  _ec_GF2m_simple_point2oct
0001:00187a20  _ec_GF2m_simple_oct2point
Module: U:\tmp\ldconv_libcrypto_a_99560c9c37f156ab8.lib(ecp_oct.obj)
0001:00187e00  _ec_GFp_simple_set_compressed_coordinates
0001:001882d0  _ec_GFp_simple_point2oct
0001:001886a0  _ec_GFp_simple_oct2point
Module: U:\tmp\ldconv_libcrypto_a_99560c9c37f156ab8.lib(bn_mul.obj)
0001:00188a20* _bn_mul_normal
0001:00188b80* _bn_mul_recursive
0001:00189130* _bn_mul_part_recursive
0001:001897b0  _bn_mul_fixed_top
0001:00189aa0  _BN_mul
0001:00189da0* _bn_mul_low_normal
0001:00189ec0* _bn_mul_low_recursive
Module: U:\tmp\ldconv_libcrypto_a_99560c9c37f156ab8.lib(bn_mod.obj)
0001:0018a000  _BN_nnmod
0001:0018a080  _BN_mod_add
0001:0018a130  _bn_mod_add_fixed_top
0001:0018a340  _BN_mod_add_quick
0001:0018a390  _BN_mod_sub
0001:0018a430  _bn_mod_sub_fixed_top
0001:0018a5c0  _BN_mod_sub_quick
0001:0018a620  _BN_mod_mul
0001:0018a720  _BN_mod_sqr
0001:0018a770* _BN_mod_lshift1
0001:0018a800  _BN_mod_lshift1_quick
0001:0018a860  _BN_mod_lshift_quick
0001:0018a960* _BN_mod_lshift
Module: U:\tmp\ldconv_libcrypto_a_99560c9c37f156ab8.lib(ecp_nistz256-x86.obj)
0001:0018aa20  _ecp_nistz256_precomputed
0001:001afae0* _ecp_nistz256_mul_by_2
0001:001afb00* _ecp_nistz256_mul_by_3
0001:001afb30* _ecp_nistz256_div_by_2
0001:001afc20* _ecp_nistz256_add
0001:001afd10* _ecp_nistz256_sub
0001:001afdc0  _ecp_nistz256_neg
0001:001afe10* _ecp_nistz256_to_mont
0001:001afe40  _ecp_nistz256_from_mont
0001:001afe70  _ecp_nistz256_mul_mont
0001:001afe90  _ecp_nistz256_sqr_mont
0001:001b0600  _ecp_nistz256_scatter_w5
0001:001b0640  _ecp_nistz256_gather_w5
0001:001b0760  _ecp_nistz256_scatter_w7
0001:001b07a0  _ecp_nistz256_gather_w7
0001:001b0ac0  _ecp_nistz256_point_double
0001:001b0cb0  _ecp_nistz256_point_add
0001:001b1440  _ecp_nistz256_point_add_affine
Module: U:\tmp\ldconv_libcrypto_a_99560c9c37f156ab8.lib(ecp_mont.obj)
0001:001b2a20  _ec_GFp_mont_group_init
0001:001b2a50  _ec_GFp_mont_group_finish
0001:001b2a90  _ec_GFp_mont_group_clear_finish
0001:001b2ae0  _ec_GFp_mont_group_set_curve
0001:001b2c80  _ec_GFp_mont_field_inv
0001:001b2db0  _ec_GFp_mont_group_copy
0001:001b2e60  _ec_GFp_mont_field_encode
0001:001b2ed0  _ec_GFp_mont_field_mul
0001:001b2f40  _ec_GFp_mont_field_sqr
0001:001b2fc0  _ec_GFp_mont_field_decode
0001:001b3030  _ec_GFp_mont_field_set_to_one
0001:001b30a0  _EC_GFp_mont_method
Module: U:\tmp\ldconv_libcrypto_a_99560c9c37f156ab8.lib(ecp_smpl.obj)
0001:001b31a0  _ec_GFp_simple_group_init
0001:001b3210  _ec_GFp_simple_group_finish
0001:001b3240  _ec_GFp_simple_point_init
0001:001b32b0  _ec_GFp_simple_point_finish
0001:001b32e0  _ec_GFp_simple_group_clear_finish
0001:001b3310  _ec_GFp_simple_point_clear_finish
0001:001b3350  _ec_GFp_simple_group_get_degree
0001:001b3360  _ec_GFp_simple_group_get_curve
0001:001b34b0  _ec_GFp_simple_get_Jprojective_coordinates_GFp
0001:001b3630  _ec_GFp_simple_is_at_infinity
0001:001b3640* _ec_GFp_simple_field_sqr
0001:001b3660* _ec_GFp_simple_field_mul
0001:001b36a0  _ec_GFp_simple_group_check_discriminant
0001:001b3940  _ec_GFp_simple_point_set_to_infinity
0001:001b3970  _ec_GFp_simple_set_Jprojective_coordinates_GFp
0001:001b3b10  _ec_GFp_simple_point_get_affine_coordinates
0001:001b3ee0  _ec_GFp_simple_dbl
0001:001b44f0  _ec_GFp_simple_ladder_step
0001:001b4b10  _ec_GFp_simple_ladder_pre
0001:001b4e70* _ec_GFp_simple_field_inv
0001:001b4fc0  _ec_GFp_simple_blind_coordinates
0001:001b5180  _ec_GFp_simple_group_copy
0001:001b51f0  _ec_GFp_simple_point_copy
0001:001b5270  _ec_GFp_simple_group_set_curve
0001:001b5480  _ec_GFp_simple_point_set_affine_coordinates
0001:001b5510  _ec_GFp_simple_cmp
0001:001b5880  _ec_GFp_simple_add
0001:001b6020  _ec_GFp_simple_invert
0001:001b6080  _ec_GFp_simple_is_on_curve
0001:001b6400  _ec_GFp_simple_make_affine
0001:001b6550  _ec_GFp_simple_points_make_affine
0001:001b6af0  _ec_GFp_simple_ladder_post
0001:001b70e0* _EC_GFp_simple_method
Module: U:\tmp\ldconv_libcrypto_a_99560c9c37f156ab8.lib(x86-mont.obj)
0001:001b71e0  _bn_mul_mont
Module: U:\tmp\ldconv_libcrypto_a_99560c9c37f156ab8.lib(bn_sqr.obj)
0001:001b7630* _bn_sqr_normal
0001:001b7730* _bn_sqr_recursive
0001:001b7910  _bn_sqr_fixed_top
0001:001b7b20  _BN_sqr
Module: U:\tmp\ldconv_libcrypto_a_99560c9c37f156ab8.lib(bn_gcd.obj)
0001:001b8840  _int_bn_mod_inverse
0001:001b88d0  _BN_mod_inverse
0001:001b89d0  _BN_gcd
Module: U:\tmp\ldconv_libcrypto_a_99560c9c37f156ab8.lib(bn_recp.obj)
0001:001b8cf0  _BN_RECP_CTX_init
0001:001b8d50* _BN_RECP_CTX_new
0001:001b8dd0  _BN_RECP_CTX_free
0001:001b8e20  _BN_RECP_CTX_set
0001:001b8e80* _BN_div_recp
0001:001b91c0  _BN_mod_mul_reciprocal
0001:001b9270* _BN_reciprocal
Module: U:\tmp\ldconv_libcrypto_a_99560c9c37f156ab8.lib(ec2_smpl.obj)
0001:001b92f0* _ec_GF2m_simple_points_make_affine
0001:001b9350* _ec_GF2m_simple_group_init
0001:001b93c0* _ec_GF2m_simple_group_finish
0001:001b93f0* _ec_GF2m_simple_point_init
0001:001b9460* _ec_GF2m_simple_point_finish
0001:001b9490* _ec_GF2m_simple_group_clear_finish
0001:001b94f0* _ec_GF2m_simple_point_clear_finish
0001:001b9530* _ec_GF2m_simple_group_get_degree
0001:001b9550* _ec_GF2m_simple_is_at_infinity
0001:001b9580* _ec_GF2m_simple_group_check_discriminant
0001:001b9650* _ec_GF2m_simple_point_set_to_infinity
0001:001b98b0* _ec_GF2m_simple_field_mul
0001:001b98e0* _ec_GF2m_simple_field_sqr
0001:001b9900* _ec_GF2m_simple_field_div
0001:001b9930* _ec_GF2m_simple_group_get_curve
0001:001b99b0* _ec_GF2m_simple_point_copy
0001:001b9a30* _ec_GF2m_simple_group_copy
0001:001b9b20* _ec_GF2m_simple_group_set_curve
0001:001b9c50* _ec_GF2m_simple_point_set_affine_coordinates
0001:001b9d50* _ec_GF2m_simple_point_get_affine_coordinates
0001:001b9e90* _ec_GF2m_simple_cmp
0001:001ba080* _ec_GF2m_simple_make_affine
0001:001ba1a0* _ec_GF2m_simple_is_on_curve
0001:001ba7b0* _ec_GF2m_simple_add
0001:001ba830* _ec_GF2m_simple_invert
0001:001bb1f0* _ec_GF2m_simple_dbl
0001:001bb270  _EC_GF2m_simple_method
Module: U:\tmp\ldconv_libcrypto_a_99560c9c37f156ab8.lib(uid.obj)
0001:001bb370  _OPENSSL_issetugid
Module: U:\tmp\ldconv_libcrypto_a_99560c9c37f156ab8.lib(b_addr.obj)
0002:0000d830  _bio_lookup_lock
0001:001bb770  _BIO_ADDR_new
0001:001bb7e0  _BIO_ADDR_free
0001:001bb810  _BIO_ADDR_clear
0001:001bb840* _BIO_ADDR_make
0001:001bb8f0* _BIO_ADDR_rawmake
0001:001bba30  _BIO_ADDR_family
0001:001bba40  _BIO_ADDR_rawaddress
0001:001bbab0  _BIO_ADDR_rawport
0001:001bbad0  _BIO_ADDR_hostname_string
0001:001bbb20  _BIO_ADDR_service_string
0001:001bbb70* _BIO_ADDR_path_string
0001:001bbbb0  _BIO_ADDR_sockaddr
0001:001bbbc0  _BIO_ADDR_sockaddr_noconst
0001:001bbbd0  _BIO_ADDR_sockaddr_size
0001:001bbc00* _BIO_ADDRINFO_next
0001:001bbc10  _BIO_ADDRINFO_family
0001:001bbc20  _BIO_ADDRINFO_socktype
0001:001bbc30  _BIO_ADDRINFO_protocol
0001:001bbc70* _BIO_ADDRINFO_sockaddr_size
0001:001bbc80* _BIO_ADDRINFO_sockaddr
0001:001bbc90  _BIO_ADDRINFO_address
0001:001bbca0  _BIO_ADDRINFO_free
0001:001bbd10  _BIO_parse_hostserv
0001:001bbf70  _BIO_lookup
0001:001bc380* _BIO_lookup_ex
Module: U:\tmp\ldconv_libcrypto_a_99560c9c37f156ab8.lib(cmeth_lib.obj)
0001:001bc7b0  _EVP_CIPHER_meth_new
0001:001bc7f0* _EVP_CIPHER_meth_dup
0001:001bc890  _EVP_CIPHER_meth_free
0001:001bc8c0  _EVP_CIPHER_meth_set_iv_length
0001:001bc8e0  _EVP_CIPHER_meth_set_flags
0001:001bc900  _EVP_CIPHER_meth_set_impl_ctx_size
0001:001bc920  _EVP_CIPHER_meth_set_init
0001:001bc940  _EVP_CIPHER_meth_set_do_cipher
0001:001bc960* _EVP_CIPHER_meth_set_cleanup
0001:001bc980* _EVP_CIPHER_meth_set_set_asn1_params
0001:001bc9a0* _EVP_CIPHER_meth_set_get_asn1_params
0001:001bc9c0* _EVP_CIPHER_meth_set_ctrl
0001:001bc9e0* _EVP_CIPHER_meth_get_init
0001:001bc9f0* _EVP_CIPHER_meth_get_do_cipher
0001:001bca00* _EVP_CIPHER_meth_get_cleanup
0001:001bca10* _EVP_CIPHER_meth_get_set_asn1_params
0001:001bca20* _EVP_CIPHER_meth_get_get_asn1_params
0001:001bca30* _EVP_CIPHER_meth_get_ctrl
Module: U:\tmp\ldconv_libcrypto_a_99560c9c37f156ab8.lib(rc4-586.obj)
0001:001bca40  _RC4
0001:001bcbb0  _RC4_set_key
0001:001bcc60* _RC4_options
Module: U:\tmp\ldconv_libcrypto_a_99560c9c37f156ab8.lib(conf_mall.obj)
0001:001bcd40  _OPENSSL_load_builtin_modules
Module: U:\tmp\ldconv_libcrypto_a_99560c9c37f156ab8.lib(m_md4.obj)
0001:001bcde0  _EVP_md4
Module: U:\tmp\ldconv_libcrypto_a_99560c9c37f156ab8.lib(m_mdc2.obj)
0001:001bcec0  _EVP_mdc2
Module: U:\tmp\ldconv_libcrypto_a_99560c9c37f156ab8.lib(m_ripemd.obj)
0001:001bcfa0  _EVP_ripemd160
Module: U:\tmp\ldconv_libcrypto_a_99560c9c37f156ab8.lib(m_wp.obj)
0001:001bd080  _EVP_whirlpool
Module: U:\tmp\ldconv_libcrypto_a_99560c9c37f156ab8.lib(m_sm3.obj)
0001:001bd160  _EVP_sm3
Module: U:\tmp\ldconv_libcrypto_a_99560c9c37f156ab8.lib(m_blake2b.obj)
0001:001bd240  _EVP_blake2b512
Module: U:\tmp\ldconv_libcrypto_a_99560c9c37f156ab8.lib(m_blake2s.obj)
0001:001bd320  _EVP_blake2s256
Module: U:\tmp\ldconv_libcrypto_a_99560c9c37f156ab8.lib(m_sha3.obj)
0001:001bd690  _EVP_sha3_224
0001:001bd6a0  _EVP_sha3_256
0001:001bd6b0  _EVP_sha3_384
0001:001bd6c0  _EVP_sha3_512
0001:001bd6d0  _EVP_shake128
0001:001bd6e0  _EVP_shake256
Module: U:\tmp\ldconv_libcrypto_a_99560c9c37f156ab8.lib(e_xcbc_d.obj)
0001:001bda60  _EVP_desx_cbc
Module: U:\tmp\ldconv_libcrypto_a_99560c9c37f156ab8.lib(e_sm4.obj)
0001:001be050  _EVP_sm4_cbc
0001:001be060  _EVP_sm4_cfb128
0001:001be070  _EVP_sm4_ofb
0001:001be080  _EVP_sm4_ecb
0001:001be090  _EVP_sm4_ctr
Module: U:\tmp\ldconv_libcrypto_a_99560c9c37f156ab8.lib(e_bf.obj)
0001:001be5d0  _EVP_bf_cbc
0001:001be5e0  _EVP_bf_cfb64
0001:001be5f0  _EVP_bf_ofb
0001:001be600  _EVP_bf_ecb
Module: U:\tmp\ldconv_libcrypto_a_99560c9c37f156ab8.lib(e_cast.obj)
0001:001beb10  _EVP_cast5_cbc
0001:001beb20  _EVP_cast5_cfb64
0001:001beb30  _EVP_cast5_ofb
0001:001beb40  _EVP_cast5_ecb
Module: U:\tmp\ldconv_libcrypto_a_99560c9c37f156ab8.lib(bn_err.obj)
0001:001bec60  _ERR_load_BN_strings
Module: U:\tmp\ldconv_libcrypto_a_99560c9c37f156ab8.lib(rsa_err.obj)
0001:001bf340  _ERR_load_RSA_strings
Module: U:\tmp\ldconv_libcrypto_a_99560c9c37f156ab8.lib(dh_err.obj)
0001:001c02e0  _ERR_load_DH_strings
Module: U:\tmp\ldconv_libcrypto_a_99560c9c37f156ab8.lib(evp_err.obj)
0001:001c0880  _ERR_load_EVP_strings
Module: U:\tmp\ldconv_libcrypto_a_99560c9c37f156ab8.lib(buf_err.obj)
0001:001c1c00  _ERR_load_BUF_strings
Module: U:\tmp\ldconv_libcrypto_a_99560c9c37f156ab8.lib(obj_err.obj)
0001:001c1ca0  _ERR_load_OBJ_strings
Module: U:\tmp\ldconv_libcrypto_a_99560c9c37f156ab8.lib(pem_err.obj)
0001:001c1e00  _ERR_load_PEM_strings
Module: U:\tmp\ldconv_libcrypto_a_99560c9c37f156ab8.lib(dsa_err.obj)
0001:001c25a0  _ERR_load_DSA_strings
Module: U:\tmp\ldconv_libcrypto_a_99560c9c37f156ab8.lib(x509_err.obj)
0001:001c2980  _ERR_load_X509_strings
Module: U:\tmp\ldconv_libcrypto_a_99560c9c37f156ab8.lib(asn1_err.obj)
0001:001c34c0  _ERR_load_ASN1_strings
Module: U:\tmp\ldconv_libcrypto_a_99560c9c37f156ab8.lib(conf_err.obj)
0001:001c4c40  _ERR_load_CONF_strings
Module: U:\tmp\ldconv_libcrypto_a_99560c9c37f156ab8.lib(cpt_err.obj)
0001:001c5120  _ERR_load_CRYPTO_strings
Module: U:\tmp\ldconv_libcrypto_a_99560c9c37f156ab8.lib(comp_err.obj)
0001:001c5420  _ERR_load_COMP_strings
Module: U:\tmp\ldconv_libcrypto_a_99560c9c37f156ab8.lib(ec_err.obj)
0001:001c5560  _ERR_load_EC_strings
Module: U:\tmp\ldconv_libcrypto_a_99560c9c37f156ab8.lib(bio_err.obj)
0001:001c7260  _ERR_load_BIO_strings
Module: U:\tmp\ldconv_libcrypto_a_99560c9c37f156ab8.lib(pkcs7err.obj)
0001:001c7b80  _ERR_load_PKCS7_strings
Module: U:\tmp\ldconv_libcrypto_a_99560c9c37f156ab8.lib(v3err.obj)
0001:001c8440  _ERR_load_X509V3_strings
Module: U:\tmp\ldconv_libcrypto_a_99560c9c37f156ab8.lib(pk12err.obj)
0001:001c92e0  _ERR_load_PKCS12_strings
Module: U:\tmp\ldconv_libcrypto_a_99560c9c37f156ab8.lib(rand_err.obj)
0001:001c98e0  _ERR_load_RAND_strings
Module: U:\tmp\ldconv_libcrypto_a_99560c9c37f156ab8.lib(dso_err.obj)
0001:001ca0a0  _ERR_load_DSO_strings
Module: U:\tmp\ldconv_libcrypto_a_99560c9c37f156ab8.lib(ts_err.obj)
0001:001ca620  _ERR_load_TS_strings
Module: U:\tmp\ldconv_libcrypto_a_99560c9c37f156ab8.lib(eng_err.obj)
0001:001cb1c0  _ERR_load_ENGINE_strings
Module: U:\tmp\ldconv_libcrypto_a_99560c9c37f156ab8.lib(ocsp_err.obj)
0001:001cba20  _ERR_load_OCSP_strings
Module: U:\tmp\ldconv_libcrypto_a_99560c9c37f156ab8.lib(ui_err.obj)
0001:001cbf80  _ERR_load_UI_strings
Module: U:\tmp\ldconv_libcrypto_a_99560c9c37f156ab8.lib(cms_err.obj)
0001:001cc380  _ERR_load_CMS_strings
Module: U:\tmp\ldconv_libcrypto_a_99560c9c37f156ab8.lib(ct_err.obj)
0001:001cd7a0  _ERR_load_CT_strings
Module: U:\tmp\ldconv_libcrypto_a_99560c9c37f156ab8.lib(async_err.obj)
0001:001cdc80  _ERR_load_ASYNC_strings
Module: U:\tmp\ldconv_libcrypto_a_99560c9c37f156ab8.lib(kdf_err.obj)
0001:001cde20  _ERR_load_KDF_strings
Module: U:\tmp\ldconv_libcrypto_a_99560c9c37f156ab8.lib(store_err.obj)
0001:001ce120  _ERR_load_OSSL_STORE_strings
Module: U:\tmp\ldconv_libcrypto_a_99560c9c37f156ab8.lib(loader_file.obj)
0001:001d0b80  _ossl_store_file_attach_pem_bio_int
0001:001d0bf0  _ossl_store_file_detach_pem_bio_int
0001:001d0c60  _ossl_store_file_loader_init
Module: U:\tmp\ldconv_libcrypto_a_99560c9c37f156ab8.lib(store_register.obj)
0001:001d0d60* _OSSL_STORE_LOADER_new
0001:001d0e10* _OSSL_STORE_LOADER_get0_engine
0001:001d0e20* _OSSL_STORE_LOADER_get0_scheme
0001:001d0e30* _OSSL_STORE_LOADER_set_open
0001:001d0e50* _OSSL_STORE_LOADER_set_ctrl
0001:001d0e70* _OSSL_STORE_LOADER_set_expect
0001:001d0e90* _OSSL_STORE_LOADER_set_find
0001:001d0eb0* _OSSL_STORE_LOADER_set_load
0001:001d0ed0* _OSSL_STORE_LOADER_set_eof
0001:001d0ef0* _OSSL_STORE_LOADER_set_error
0001:001d0f10* _OSSL_STORE_LOADER_set_close
0001:001d0f30* _OSSL_STORE_LOADER_free
0001:001d0f60  _ossl_store_register_loader_int
0001:001d11a0* _OSSL_STORE_register_loader
0001:001d11d0  _ossl_store_get0_loader_int
0001:001d1300  _ossl_store_unregister_loader_int
0001:001d1420* _OSSL_STORE_unregister_loader
0001:001d1540  _ossl_store_destroy_loaders_int
0001:001d1580* _OSSL_STORE_do_all_loaders
Module: U:\tmp\ldconv_libcrypto_a_99560c9c37f156ab8.lib(cfb64enc.obj)
0001:001d15b0  _DES_cfb64_encrypt
Module: U:\tmp\ldconv_libcrypto_a_99560c9c37f156ab8.lib(ofb64enc.obj)
0001:001d1700  _DES_ofb64_encrypt
Module: U:\tmp\ldconv_libcrypto_a_99560c9c37f156ab8.lib(cfb_enc.obj)
0001:001d1810  _DES_cfb_encrypt
Module: U:\tmp\ldconv_libcrypto_a_99560c9c37f156ab8.lib(cfb64ede.obj)
0001:001d2020  _DES_ede3_cfb64_encrypt
0001:001d2190  _DES_ede3_cfb_encrypt
Module: U:\tmp\ldconv_libcrypto_a_99560c9c37f156ab8.lib(ofb64ede.obj)
0001:001d2a30  _DES_ede3_ofb64_encrypt
Module: U:\tmp\ldconv_libcrypto_a_99560c9c37f156ab8.lib(ecb3_enc.obj)
0001:001d2b30  _DES_ecb3_encrypt
Module: U:\tmp\ldconv_libcrypto_a_99560c9c37f156ab8.lib(sha1_one.obj)
0001:001d2ba0  _SHA1
Module: U:\tmp\ldconv_libcrypto_a_99560c9c37f156ab8.lib(i_cbc.obj)
0001:001d2c10  _IDEA_encrypt
0001:001d3500  _IDEA_cbc_encrypt
Module: U:\tmp\ldconv_libcrypto_a_99560c9c37f156ab8.lib(i_cfb64.obj)
0001:001d39a0  _IDEA_cfb64_encrypt
Module: U:\tmp\ldconv_libcrypto_a_99560c9c37f156ab8.lib(i_ofb64.obj)
0001:001d3b10  _IDEA_ofb64_encrypt
Module: U:\tmp\ldconv_libcrypto_a_99560c9c37f156ab8.lib(i_ecb.obj)
0001:001d3c20* _IDEA_options
0001:001d3c30  _IDEA_ecb_encrypt
Module: U:\tmp\ldconv_libcrypto_a_99560c9c37f156ab8.lib(i_skey.obj)
0001:001d3c80  _IDEA_set_encrypt_key
0001:001d41b0  _IDEA_set_decrypt_key
Module: U:\tmp\ldconv_libcrypto_a_99560c9c37f156ab8.lib(rc2_cbc.obj)
0001:001d4330  _RC2_encrypt
0001:001d4470  _RC2_decrypt
0001:001d45e0  _RC2_cbc_encrypt
Module: U:\tmp\ldconv_libcrypto_a_99560c9c37f156ab8.lib(rc2_skey.obj)
0001:001d4a70  _RC2_set_key
Module: U:\tmp\ldconv_libcrypto_a_99560c9c37f156ab8.lib(rc2cfb64.obj)
0001:001d4d70  _RC2_cfb64_encrypt
Module: U:\tmp\ldconv_libcrypto_a_99560c9c37f156ab8.lib(rc2ofb64.obj)
0001:001d4ec0  _RC2_ofb64_encrypt
Module: U:\tmp\ldconv_libcrypto_a_99560c9c37f156ab8.lib(rc2_ecb.obj)
0001:001d4fb0  _RC2_ecb_encrypt
Module: U:\tmp\ldconv_libcrypto_a_99560c9c37f156ab8.lib(aria.obj)
0001:001d5000  _aria_encrypt
0001:001d5610  _aria_set_encrypt_key
0001:001d6330  _aria_set_decrypt_key
Module: U:\tmp\ldconv_libcrypto_a_99560c9c37f156ab8.lib(cmll-x86.obj)
0001:001d76c0* _Camellia_EncryptBlock_Rounds
0001:001d7770* _Camellia_EncryptBlock
0001:001d7790  _Camellia_encrypt
0001:001d7b50* _Camellia_DecryptBlock_Rounds
0001:001d7c00* _Camellia_DecryptBlock
0001:001d7c20  _Camellia_decrypt
0001:001d7fe0* _Camellia_Ekeygen
0001:001d8980  _Camellia_set_key
0001:001d9a40  _Camellia_cbc_encrypt
Module: U:\tmp\ldconv_libcrypto_a_99560c9c37f156ab8.lib(chacha-x86.obj)
0001:001d9e40  _ChaCha20_ctr32
Module: U:\tmp\ldconv_libcrypto_a_99560c9c37f156ab8.lib(poly1305.obj)
0001:001da330  _Poly1305_ctx_size
0001:001da340  _Poly1305_Init
0001:001da3b0  _Poly1305_Update
0001:001da510  _Poly1305_Final
Module: U:\tmp\ldconv_libcrypto_a_99560c9c37f156ab8.lib(seed_cbc.obj)
0001:001da610  _SEED_cbc_encrypt
Module: U:\tmp\ldconv_libcrypto_a_99560c9c37f156ab8.lib(seed.obj)
0001:001da640  _SEED_set_key
0001:001daf80  _SEED_encrypt
0001:001dbab0  _SEED_decrypt
Module: U:\tmp\ldconv_libcrypto_a_99560c9c37f156ab8.lib(seed_cfb.obj)
0001:001dd5e0  _SEED_cfb128_encrypt
Module: U:\tmp\ldconv_libcrypto_a_99560c9c37f156ab8.lib(seed_ofb.obj)
0001:001dd630  _SEED_ofb128_encrypt
Module: U:\tmp\ldconv_libcrypto_a_99560c9c37f156ab8.lib(seed_ecb.obj)
0001:001dd680  _SEED_ecb_encrypt
Module: U:\tmp\ldconv_libcrypto_a_99560c9c37f156ab8.lib(dh_check.obj)
0001:001dd6a0  _DH_check_params
0001:001dd7a0* _DH_check_params_ex
0001:001dd850* _DH_check
0001:001dda80  _DH_check_ex
0001:001ddca0  _DH_check_pub_key
0001:001dddd0  _DH_check_pub_key_ex
Module: U:\tmp\ldconv_libssl_a_99560c9c37e1aece0.lib(pqueue.obj)
0001:001ddef0  _pitem_new
0001:001ddf70  _pitem_free
0001:001ddfa0  _pqueue_new
0001:001de010  _pqueue_free
0001:001de040  _pqueue_insert
0001:001de0e0  _pqueue_peek
0001:001de0f0  _pqueue_pop
0001:001de100  _pqueue_find
0001:001de160  _pqueue_iterator
0001:001de170  _pqueue_next
0001:001de1a0  _pqueue_size
Module: U:\tmp\ldconv_libcrypto_a_99560c9c37f156ab8.lib(sha1-586.obj)
0001:001de1c0  _sha1_block_data_order
Module: U:\tmp\ldconv_libcrypto_a_99560c9c37f156ab8.lib(sha256-586.obj)
0001:001df170  _sha256_block_data_order
Module: U:\tmp\ldconv_libcrypto_a_99560c9c37f156ab8.lib(sha512-586.obj)
0001:001df5f0  _sha512_block_data_order
Module: U:\tmp\ldconv_libcrypto_a_99560c9c37f156ab8.lib(ghash-x86.obj)
0001:001dfef0  _gcm_gmult_4bit
0001:001e0060  _gcm_ghash_4bit
Module: U:\tmp\ldconv_libcrypto_a_99560c9c37f156ab8.lib(rsa_pmeth.obj)
0001:001e20b0  _rsa_pss_pkey_meth
0001:001e2150  _rsa_pkey_meth
Module: U:\tmp\ldconv_libcrypto_a_99560c9c37f156ab8.lib(dh_pmeth.obj)
0001:001e2f90  _dhx_pkey_meth
0001:001e3030  _dh_pkey_meth
Module: U:\tmp\ldconv_libcrypto_a_99560c9c37f156ab8.lib(dsa_pmeth.obj)
0001:001e3930  _dsa_pkey_meth
Module: U:\tmp\ldconv_libcrypto_a_99560c9c37f156ab8.lib(ec_pmeth.obj)
0001:001e4870  _ec_pkey_meth
Module: U:\tmp\ldconv_libcrypto_a_99560c9c37f156ab8.lib(hm_pmeth.obj)
0001:001e4eb0  _hmac_pkey_meth
Module: U:\tmp\ldconv_libcrypto_a_99560c9c37f156ab8.lib(cm_pmeth.obj)
0001:001e52b0  _cmac_pkey_meth
Module: U:\tmp\ldconv_libcrypto_a_99560c9c37f156ab8.lib(scrypt.obj)
0001:001e5dd0  _scrypt_pkey_meth
Module: U:\tmp\ldconv_libcrypto_a_99560c9c37f156ab8.lib(tls1_prf.obj)
0001:001e68b0  _tls1_prf_pkey_meth
Module: U:\tmp\ldconv_libcrypto_a_99560c9c37f156ab8.lib(hkdf.obj)
0001:001e7430  _hkdf_pkey_meth
Module: U:\tmp\ldconv_libcrypto_a_99560c9c37f156ab8.lib(poly1305_pmeth.obj)
0001:001e7a10  _poly1305_pkey_meth
Module: U:\tmp\ldconv_libcrypto_a_99560c9c37f156ab8.lib(siphash_pmeth.obj)
0001:001e8110  _siphash_pkey_meth
Module: U:\tmp\ldconv_libcrypto_a_99560c9c37f156ab8.lib(sm2_pmeth.obj)
0001:001e8b50  _sm2_pkey_meth
Module: U:\tmp\ldconv_libcrypto_a_99560c9c37f156ab8.lib(p12_attr.obj)
0001:001e8bf0* _PKCS12_add_localkeyid
0001:001e8c30* _PKCS8_add_keyusage
0001:001e8c70* _PKCS12_add_friendlyname_asc
0001:001e8cb0* _PKCS12_add_friendlyname_utf8
0001:001e8cf0* _PKCS12_add_friendlyname_uni
0001:001e8d30* _PKCS12_add_CSPName_asc
0001:001e8d70  _PKCS12_get_attr_gen
0001:001e8dc0* _PKCS12_get_friendlyname
0001:001e8e10* _PKCS12_SAFEBAG_get0_attrs
Module: U:\tmp\ldconv_libcrypto_a_99560c9c37f156ab8.lib(p12_p8e.obj)
0001:001e8e40  _PKCS8_encrypt
0001:001e9030* _PKCS8_set0_pbe
Module: U:\tmp\ldconv_libcrypto_a_99560c9c37f156ab8.lib(x509_att.obj)
0001:001e9110  _X509at_get_attr_count
0001:001e9120  _X509at_get_attr_by_NID
0001:001e91b0  _X509at_get_attr_by_OBJ
0001:001e9230  _X509at_get_attr
0001:001e9270  _X509at_delete_attr
0001:001e92d0  _X509at_add1_attr
0001:001e93d0  _X509at_get0_data_by_OBJ
0001:001e9580* _X509_ATTRIBUTE_set1_object
0001:001e95d0* _X509_ATTRIBUTE_set1_data
0001:001e97c0* _X509_ATTRIBUTE_create_by_OBJ
0001:001e9900  _X509at_add1_attr_by_OBJ
0001:001e99d0  _X509at_add1_attr_by_txt
0001:001e9b20  _X509at_add1_attr_by_NID
0001:001e9c40* _X509_ATTRIBUTE_create_by_NID
0001:001e9dc0* _X509_ATTRIBUTE_create_by_txt
0001:001e9f60  _X509_ATTRIBUTE_count
0001:001e9f80  _X509_ATTRIBUTE_get0_object
0001:001e9fa0* _X509_ATTRIBUTE_get0_data
0001:001ea030  _X509_ATTRIBUTE_get0_type
Module: U:\tmp\ldconv_libcrypto_a_99560c9c37f156ab8.lib(pk7_lib.obj)
0001:001ea070  _PKCS7_ctrl
0001:001ea1b0* _PKCS7_set_content
0001:001ea250  _PKCS7_set_type
0001:001ea460* _PKCS7_content_new
0001:001ea530* _PKCS7_set0_type_other
0001:001ea560* _PKCS7_add_signer
0001:001ea6c0* _PKCS7_add_certificate
0001:001ea7d0* _PKCS7_add_crl
0001:001ea8e0* _PKCS7_SIGNER_INFO_set
0001:001eaa50* _PKCS7_add_signature
0001:001eab30* _PKCS7_set_digest
0001:001eac10* _PKCS7_get_signer_info
0001:001eac60  _PKCS7_SIGNER_INFO_get0_algs
0001:001eac90  _PKCS7_RECIP_INFO_get0_alg
0001:001eacb0* _PKCS7_add_recipient_info
0001:001ead40* _PKCS7_RECIP_INFO_set
0001:001eae90* _PKCS7_add_recipient
0001:001eaf40* _PKCS7_cert_from_signer_info
0001:001eaf90* _PKCS7_set_cipher
0001:001eb060  _PKCS7_stream
Module: U:\tmp\ldconv_libcrypto_a_99560c9c37f156ab8.lib(p5_pbev2.obj)
0001:001eb120* _d2i_PBE2PARAM
0001:001eb87c  _PBE2PARAM_it
0001:001eb150* _i2d_PBE2PARAM
0001:001eb180  _PBE2PARAM_new
0001:001eb1a0  _PBE2PARAM_free
0001:001eb1c0* _d2i_PBKDF2PARAM
0001:001eb7d8  _PBKDF2PARAM_it
0001:001eb1f0* _i2d_PBKDF2PARAM
0001:001eb220* _PBKDF2PARAM_new
0001:001eb240  _PBKDF2PARAM_free
0001:001eb280  _PKCS5_pbkdf2_set
0001:001eb4a0  _PKCS5_pbe2_set_iv
0001:001eb790  _PKCS5_pbe2_set
Module: U:\tmp\ldconv_libcrypto_a_99560c9c37f156ab8.lib(p12_decr.obj)
0001:001eb920  _PKCS12_pbe_crypt
0001:001ebb60  _PKCS12_item_decrypt_d2i
0001:001ebca0  _PKCS12_item_i2d_encrypt
Module: U:\tmp\ldconv_libcrypto_a_99560c9c37f156ab8.lib(p5_pbe.obj)
0001:001ebe30* _d2i_PBEPARAM
0001:001ec198  _PBEPARAM_it
0001:001ebe60* _i2d_PBEPARAM
0001:001ebe90* _PBEPARAM_new
0001:001ebeb0  _PBEPARAM_free
0001:001ebee0* _PKCS5_pbe_set0_algor
0001:001ec100  _PKCS5_pbe_set
Module: U:\tmp\ldconv_libcrypto_a_99560c9c37f156ab8.lib(p12_key.obj)
0001:001ec230* _PKCS12_key_gen_uni
0001:001ec6d0* _PKCS12_key_gen_asc
0001:001ec7f0  _PKCS12_key_gen_utf8
Module: U:\tmp\ldconv_libcrypto_a_99560c9c37f156ab8.lib(p5_crpt2.obj)
0001:001ec920  _PKCS5_PBKDF2_HMAC
0001:001ecdb0* _PKCS5_PBKDF2_HMAC_SHA1
0001:001ece20  _PKCS5_v2_PBE_keyivgen
0001:001ed070  _PKCS5_v2_PBKDF2_keyivgen
Module: U:\tmp\ldconv_libcrypto_a_99560c9c37f156ab8.lib(pk7_doit.obj)
0001:001ed8c0  _PKCS7_dataInit
0001:001ee1b0* _PKCS7_dataDecode
0001:001eebe0* _PKCS7_SIGNER_INFO_sign
0001:001eee70  _PKCS7_dataFinal
0001:001ef700* _PKCS7_signatureVerify
0001:001efb30* _PKCS7_dataVerify
0001:001efda0* _PKCS7_get_issuer_and_serial
0001:001efe00  _PKCS7_get_signed_attribute
0001:001efe50* _PKCS7_get_attribute
0001:001efea0* _PKCS7_digest_from_attributes
0001:001efef0* _PKCS7_set_signed_attributes
0001:001eff80* _PKCS7_set_attributes
0001:001f0010  _PKCS7_add_signed_attribute
0001:001f0030* _PKCS7_add_attribute
Module: U:\tmp\ldconv_libcrypto_a_99560c9c37f156ab8.lib(tasn_prn.obj)
0001:001f1120* _ASN1_PCTX_new
0001:001f1190* _ASN1_PCTX_free
0001:001f11c0* _ASN1_PCTX_get_flags
0001:001f11d0* _ASN1_PCTX_set_flags
0001:001f11e0* _ASN1_PCTX_get_nm_flags
0001:001f11f0* _ASN1_PCTX_set_nm_flags
0001:001f1200* _ASN1_PCTX_get_cert_flags
0001:001f1210* _ASN1_PCTX_set_cert_flags
0001:001f1220* _ASN1_PCTX_get_oid_flags
0001:001f1230* _ASN1_PCTX_set_oid_flags
0001:001f1240* _ASN1_PCTX_get_str_flags
0001:001f1250* _ASN1_PCTX_set_str_flags
0001:001f1260  _ASN1_item_print
Module: U:\tmp\ldconv_libcrypto_a_99560c9c37f156ab8.lib(x_req.obj)
0001:001f16d0* _d2i_X509_REQ_INFO
0001:001f18d4  _X509_REQ_INFO_it
0001:001f1700  _i2d_X509_REQ_INFO
0001:001f1730* _X509_REQ_INFO_new
0001:001f1750* _X509_REQ_INFO_free
0001:001f1770  _d2i_X509_REQ
0001:001f1834  _X509_REQ_it
0001:001f17a0  _i2d_X509_REQ
0001:001f17d0  _X509_REQ_new
0001:001f17f0  _X509_REQ_free
0001:001f1810* _X509_REQ_dup
Module: U:\tmp\ldconv_libcrypto_a_99560c9c37f156ab8.lib(x_spki.obj)
0001:001f19b0* _d2i_NETSCAPE_SPKAC
0001:001f1b9c  _NETSCAPE_SPKAC_it
0001:001f19e0* _i2d_NETSCAPE_SPKAC
0001:001f1a10* _NETSCAPE_SPKAC_new
0001:001f1a30* _NETSCAPE_SPKAC_free
0001:001f1a50* _d2i_NETSCAPE_SPKI
0001:001f1afc* _NETSCAPE_SPKI_it
0001:001f1a80* _i2d_NETSCAPE_SPKI
0001:001f1ab0* _NETSCAPE_SPKI_new
0001:001f1ad0* _NETSCAPE_SPKI_free
Module: U:\tmp\ldconv_libcrypto_a_99560c9c37f156ab8.lib(dsa_asn1.obj)
0001:001f1c70  _d2i_DSA_SIG
0001:001f1ca0* _i2d_DSA_SIG
0001:001f1ce0  _DSA_SIG_new
0001:001f1d50  _DSA_SIG_free
0001:001f1d90  _DSA_SIG_get0
0001:001f1db0* _DSA_SIG_set0
0001:001f1e00  _d2i_DSAPrivateKey
0001:001f1e30  _i2d_DSAPrivateKey
0001:001f1e60  _d2i_DSAparams
0001:001f1e90  _i2d_DSAparams
0001:001f1ec0* _d2i_DSAPublicKey
0001:001f1ef0* _i2d_DSAPublicKey
0001:001f1f20* _DSAparams_dup
0001:001f1f40  _DSA_sign
0001:001f1fe0  _DSA_verify
Module: U:\tmp\ldconv_libcrypto_a_99560c9c37f156ab8.lib(ec_asn1.obj)
0001:001f23f0  _EC_GROUP_get_basis_type
0001:001f2460* _EC_GROUP_get_trinomial_basis
0001:001f24f0* _EC_GROUP_get_pentanomial_basis
0001:001f25b0* _X9_62_PENTANOMIAL_new
0001:001f25d0* _X9_62_PENTANOMIAL_free
0001:001f25f0* _X9_62_CHARACTERISTIC_TWO_new
0001:001f2610* _X9_62_CHARACTERISTIC_TWO_free
0001:001f2630* _ECPARAMETERS_new
0001:001f557c* _ECPARAMETERS_it
0001:001f2650* _ECPARAMETERS_free
0001:001f2670* _d2i_ECPKPARAMETERS
0001:001f54d0* _ECPKPARAMETERS_it
0001:001f26a0* _i2d_ECPKPARAMETERS
0001:001f26d0* _ECPKPARAMETERS_new
0001:001f26f0* _ECPKPARAMETERS_free
0001:001f2710* _d2i_EC_PRIVATEKEY
0001:001f2740* _i2d_EC_PRIVATEKEY
0001:001f2770* _EC_PRIVATEKEY_new
0001:001f2790* _EC_PRIVATEKEY_free
0001:001f27b0* _EC_GROUP_get_ecparameters
0001:001f3280* _EC_GROUP_get_ecpkparameters
0001:001f3410* _EC_GROUP_new_from_ecparameters
0001:001f3f50* _EC_GROUP_new_from_ecpkparameters
0001:001f40d0  _d2i_ECPKParameters
0001:001f4300  _i2d_ECPKParameters
0001:001f44d0  _d2i_ECPrivateKey
0001:001f4780  _i2d_ECPrivateKey
0001:001f4a90  _i2d_ECParameters
0001:001f4ca0  _d2i_ECParameters
0001:001f4ed0  _o2i_ECPublicKey
0001:001f4f90  _i2o_ECPublicKey
0001:001f5180  _d2i_ECDSA_SIG
0001:001f51b0  _i2d_ECDSA_SIG
0001:001f51e0  _ECDSA_SIG_new
0001:001f5250  _ECDSA_SIG_free
0001:001f5290  _ECDSA_SIG_get0
0001:001f52b0* _ECDSA_SIG_get0_r
0001:001f52c0* _ECDSA_SIG_get0_s
0001:001f52d0  _ECDSA_SIG_set0
0001:001f5320  _ECDSA_size
Module: U:\tmp\ldconv_libcrypto_a_99560c9c37f156ab8.lib(a_digest.obj)
0001:001f5990* _ASN1_digest
0001:001f5af0  _ASN1_item_digest
Module: U:\tmp\ldconv_libcrypto_a_99560c9c37f156ab8.lib(nsseq.obj)
0001:001f5bf0  _d2i_NETSCAPE_CERT_SEQUENCE
0001:001f5ca4* _NETSCAPE_CERT_SEQUENCE_it
0001:001f5c20  _i2d_NETSCAPE_CERT_SEQUENCE
0001:001f5c50* _NETSCAPE_CERT_SEQUENCE_new
0001:001f5c70* _NETSCAPE_CERT_SEQUENCE_free
Module: U:\tmp\ldconv_libcrypto_a_99560c9c37f156ab8.lib(x_bignum.obj)
0001:001f5f70  _CBIGNUM_it
0001:001f5f94  _BIGNUM_it
Module: U:\tmp\ldconv_libssl_a_99560c9c37e1aece0.lib(dtls1_bitmap.obj)
0001:001f5fb0  _dtls1_record_replay_check
0001:001f60a0  _dtls1_record_bitmap_update
Module: U:\tmp\ldconv_libcrypto_a_99560c9c37f156ab8.lib(p_sign.obj)
0001:001f61c0  _EVP_SignFinal
Module: U:\tmp\ldconv_libcrypto_a_99560c9c37f156ab8.lib(v3_bitst.obj)
0001:001f6390* _i2v_ASN1_BIT_STRING
0001:001f6440* _v2i_ASN1_BIT_STRING
0001:001f6610  _v3_key_usage
0001:001f6650  _v3_nscert
Module: U:\tmp\ldconv_libcrypto_a_99560c9c37f156ab8.lib(v3_ia5.obj)
0001:001f6850* _i2s_ASN1_IA5STRING
0001:001f68f0* _s2i_ASN1_IA5STRING
0001:001f69b0  _v3_ns_ia5_list
Module: U:\tmp\ldconv_libcrypto_a_99560c9c37f156ab8.lib(v3_skey.obj)
0001:001f6b70* _i2s_ASN1_OCTET_STRING
0001:001f6de0* _s2i_ASN1_OCTET_STRING
0001:001f6e70  _v3_skey_id
Module: U:\tmp\ldconv_libcrypto_a_99560c9c37f156ab8.lib(v3_pku.obj)
0001:001f6fa0* _d2i_PKEY_USAGE_PERIOD
0001:001f7050* _PKEY_USAGE_PERIOD_it
0001:001f6fd0* _i2d_PKEY_USAGE_PERIOD
0001:001f7000* _PKEY_USAGE_PERIOD_new
0001:001f7020* _PKEY_USAGE_PERIOD_free
0001:001f70d0  _v3_pkey_usage_period
Module: U:\tmp\ldconv_libcrypto_a_99560c9c37f156ab8.lib(v3_int.obj)
0001:001f7130  _v3_inhibit_anyp
0001:001f7170  _v3_delta_crl
0001:001f71b0  _v3_crl_num
Module: U:\tmp\ldconv_libcrypto_a_99560c9c37f156ab8.lib(v3_akey.obj)
0001:001f76f0  _v3_akey_id
Module: U:\tmp\ldconv_libcrypto_a_99560c9c37f156ab8.lib(v3_extku.obj)
0001:001f7950* _d2i_EXTENDED_KEY_USAGE
0001:001f7a00* _EXTENDED_KEY_USAGE_it
0001:001f7980* _i2d_EXTENDED_KEY_USAGE
0001:001f79b0* _EXTENDED_KEY_USAGE_new
0001:001f79d0* _EXTENDED_KEY_USAGE_free
0001:001f7a30  _v3_ocsp_accresp
0001:001f7a70  _v3_ext_ku
Module: U:\tmp\ldconv_libcrypto_a_99560c9c37f156ab8.lib(v3_enum.obj)
0001:001f7ad0* _i2s_ASN1_ENUMERATED_TABLE
0001:001f7b50  _v3_crl_reason
Module: U:\tmp\ldconv_libcrypto_a_99560c9c37f156ab8.lib(v3_ocsp.obj)
0001:001f81d0  _v3_ocsp_serviceloc
0001:001f8210  _v3_ocsp_nocheck
0001:001f8250  _v3_ocsp_nonce
0001:001f8290  _v3_crl_hold
0001:001f82d0  _v3_crl_invdate
0001:001f8310  _v3_ocsp_acutoff
0001:001f8350  _v3_ocsp_crlid
Module: U:\tmp\ldconv_libcrypto_a_99560c9c37f156ab8.lib(v3_sxnet.obj)
0001:001f8fc0* _SXNETID_it
0001:001f8f54* _SXNET_it
0001:001f87e0* _d2i_SXNETID
0001:001f8810* _i2d_SXNETID
0001:001f8840* _SXNETID_new
0001:001f8860* _SXNETID_free
0001:001f8880* _d2i_SXNET
0001:001f88b0* _i2d_SXNET
0001:001f88e0* _SXNET_new
0001:001f8900* _SXNET_free
0001:001f8920* _SXNET_add_id_asc
0001:001f89e0* _SXNET_add_id_ulong
0001:001f8ac0* _SXNET_add_id_INTEGER
0001:001f8d50* _SXNET_get_id_asc
0001:001f8e10* _SXNET_get_id_ulong
0001:001f8ee0* _SXNET_get_id_INTEGER
0001:001f9030  _v3_sxnet
Module: U:\tmp\ldconv_libcrypto_a_99560c9c37f156ab8.lib(v3_pci.obj)
0001:001f9c50  _v3_pci
Module: U:\tmp\ldconv_libcrypto_a_99560c9c37f156ab8.lib(v3_pmaps.obj)
0001:001fa034* _POLICY_MAPPING_it
0001:001f9fb0  _POLICY_MAPPING_free
0001:001f9fd0* _POLICY_MAPPING_new
0001:001f9ff4* _POLICY_MAPPINGS_it
0001:001fa0d0  _v3_policy_mappings
Module: U:\tmp\ldconv_libcrypto_a_99560c9c37f156ab8.lib(ct_x509v3.obj)
0001:001fa2d0  _v3_ct_scts
Module: U:\tmp\ldconv_libcrypto_a_99560c9c37f156ab8.lib(v3_tlsf.obj)
0001:001fa6a0* _TLS_FEATURE_new
0001:001fa6c0* _TLS_FEATURE_free
0001:001fa6f0  _v3_tls_feature
Module: U:\tmp\ldconv_libcrypto_a_99560c9c37f156ab8.lib(v3_admis.obj)
0001:001fa770* _PROFESSION_INFO_free
0001:001fb65c* _PROFESSION_INFO_it
0001:001fa790* _ADMISSIONS_free
0001:001fb5c4* _ADMISSIONS_it
0001:001fafd0* _d2i_NAMING_AUTHORITY
0001:001fb748* _NAMING_AUTHORITY_it
0001:001fb000* _i2d_NAMING_AUTHORITY
0001:001fb030* _NAMING_AUTHORITY_new
0001:001fb050* _NAMING_AUTHORITY_free
0001:001fb070* _d2i_PROFESSION_INFO
0001:001fb0a0* _i2d_PROFESSION_INFO
0001:001fb0d0* _PROFESSION_INFO_new
0001:001fb0f0* _d2i_ADMISSIONS
0001:001fb120* _i2d_ADMISSIONS
0001:001fb150* _ADMISSIONS_new
0001:001fb170* _d2i_ADMISSION_SYNTAX
0001:001fb53c* _ADMISSION_SYNTAX_it
0001:001fb1a0* _i2d_ADMISSION_SYNTAX
0001:001fb1d0* _ADMISSION_SYNTAX_new
0001:001fb1f0* _ADMISSION_SYNTAX_free
0001:001fb210* _NAMING_AUTHORITY_get0_authorityId
0001:001fb220* _NAMING_AUTHORITY_set0_authorityId
0001:001fb240* _NAMING_AUTHORITY_get0_authorityURL
0001:001fb250* _NAMING_AUTHORITY_set0_authorityURL
0001:001fb270* _NAMING_AUTHORITY_get0_authorityText
0001:001fb280* _NAMING_AUTHORITY_set0_authorityText
0001:001fb2a0* _ADMISSION_SYNTAX_get0_admissionAuthority
0001:001fb2b0* _ADMISSION_SYNTAX_set0_admissionAuthority
0001:001fb2d0* _ADMISSION_SYNTAX_get0_contentsOfAdmissions
0001:001fb2e0* _ADMISSION_SYNTAX_set0_contentsOfAdmissions
0001:001fb310* _ADMISSIONS_get0_admissionAuthority
0001:001fb320* _ADMISSIONS_set0_admissionAuthority
0001:001fb340* _ADMISSIONS_get0_namingAuthority
0001:001fb350* _ADMISSIONS_set0_namingAuthority
0001:001fb380* _ADMISSIONS_get0_professionInfos
0001:001fb390* _ADMISSIONS_set0_professionInfos
0001:001fb3c0* _PROFESSION_INFO_get0_addProfessionInfo
0001:001fb3d0* _PROFESSION_INFO_set0_addProfessionInfo
0001:001fb3f0* _PROFESSION_INFO_get0_namingAuthority
0001:001fb400* _PROFESSION_INFO_set0_namingAuthority
0001:001fb430* _PROFESSION_INFO_get0_professionItems
0001:001fb440* _PROFESSION_INFO_set0_professionItems
0001:001fb470* _PROFESSION_INFO_get0_professionOIDs
0001:001fb480* _PROFESSION_INFO_set0_professionOIDs
0001:001fb4b0* _PROFESSION_INFO_get0_registrationNumber
0001:001fb4c0* _PROFESSION_INFO_set0_registrationNumber
0001:001fb4f0  _v3_ext_admission
Module: U:\tmp\ldconv_libcrypto_a_99560c9c37f156ab8.lib(asn1_gen.obj)
0001:001fcd90* _ASN1_generate_nconf
0001:001fce40  _ASN1_generate_v3
0001:001fceb0  _ASN1_str2mask
Module: U:\tmp\ldconv_libcrypto_a_99560c9c37f156ab8.lib(pcy_node.obj)
0001:001fd320  _policy_node_cmp_new
0001:001fd340  _tree_find_sk
0001:001fd380  _level_find_node
0001:001fd410  _level_add_node
0001:001fd5b0  _policy_node_free
0001:001fd5e0  _policy_node_match
Module: U:\tmp\ldconv_libcrypto_a_99560c9c37f156ab8.lib(pcy_lib.obj)
0001:001fd680* _X509_policy_tree_level_count
0001:001fd6a0* _X509_policy_tree_get0_level
0001:001fd6d0* _X509_policy_tree_get0_policies
0001:001fd6f0  _X509_policy_tree_get0_user_policies
0001:001fd720* _X509_policy_level_node_count
0001:001fd760* _X509_policy_level_get0_node
0001:001fd7a0* _X509_policy_node_get0_policy
0001:001fd7c0* _X509_policy_node_get0_qualifiers
0001:001fd7e0* _X509_policy_node_get0_parent
Module: U:\tmp\ldconv_libcrypto_a_99560c9c37f156ab8.lib(a_strnid.obj)
0001:001fd890* _ASN1_STRING_set_default_mask
0001:001fd8a0* _ASN1_STRING_get_default_mask
0001:001fd8d0* _ASN1_STRING_set_default_mask_asc
0001:001fd9e0  _ASN1_STRING_set_by_NID
0001:001fdb00* _ASN1_STRING_TABLE_get
0001:001fdb80  _ASN1_STRING_TABLE_add
0001:001fdda0  _ASN1_STRING_TABLE_cleanup
Module: U:\tmp\ldconv_libcrypto_a_99560c9c37f156ab8.lib(a_print.obj)
0001:001fe000  _ASN1_PRINTABLE_type
0001:001fe0e0* _ASN1_UNIVERSALSTRING_to_string
0001:001fe260  _ASN1_STRING_print
Module: U:\tmp\ldconv_libcrypto_a_99560c9c37f156ab8.lib(p_verify.obj)
0001:001fe3a0  _EVP_VerifyFinal
Module: U:\tmp\ldconv_libcrypto_a_99560c9c37f156ab8.lib(x509rset.obj)
0001:001fe540* _X509_REQ_set_version
0001:001fe570  _X509_REQ_set_subject_name
0001:001fe5a0  _X509_REQ_set_pubkey
Module: U:\tmp\ldconv_libcrypto_a_99560c9c37f156ab8.lib(x_pkey.obj)
0001:001fe5f0  _X509_PKEY_new
0001:001fe6e0  _X509_PKEY_free
Module: U:\tmp\ldconv_libgcc_eh_a_99560c9c382174360.lib(emx-eh.obj)
0001:001fe760  ___ehInit
0001:001fe79c* ___ehTerm
Module: U:\tmp\ldconv_libssl_a_99560c9c37e1aece0.lib(s3_cbc.obj)
0001:001febd0  _ssl3_cbc_record_digest_supported
0001:001fec20  _ssl3_cbc_digest_record
Module: U:\tmp\ldconv_libssl_a_99560c9c37e1aece0.lib(d1_srtp.obj)
0001:001ffbc0* _SSL_CTX_set_tlsext_use_srtp
0001:001ffbe0* _SSL_set_tlsext_use_srtp
0001:001ffc00  _SSL_get_srtp_profiles
0001:001ffc40* _SSL_get_selected_srtp_profile
Module: U:\tmp\ldconv_libcrypto_a_99560c9c37f156ab8.lib(bn_srp.obj)
0001:001ffcb0  _bn_generator_2
0001:001ffcc8  _bn_generator_5
0001:001ffce0  _bn_generator_19
0001:001ffcf8  _bn_group_8192
0001:00200110  _bn_group_6144
0001:00200430  _bn_group_4096
0001:00200650  _bn_group_3072
0001:002007f0  _bn_group_2048
0001:00200910  _bn_group_1536
0001:002009f0  _bn_group_1024
Module: U:\tmp\ldconv_libcrypto_a_99560c9c37f156ab8.lib(txt_db.obj)
0001:00200ab0  _TXT_DB_read
0001:00200ec0* _TXT_DB_get_by_index
0001:00200f20* _TXT_DB_create_index
0001:002010c0* _TXT_DB_write
0001:002012a0* _TXT_DB_insert
0001:00201450  _TXT_DB_free
Module: U:\tmp\ldconv_libcrypto_a_99560c9c37f156ab8.lib(p5_crpt.obj)
0001:002015f0* _PKCS5_PBE_add
0001:00201610  _PKCS5_PBE_keyivgen
Module: U:\tmp\ldconv_libcrypto_a_99560c9c37f156ab8.lib(p12_crpt.obj)
0001:00201a10* _PKCS12_PBE_add
0001:00201a30  _PKCS12_PBE_keyivgen
Module: U:\tmp\ldconv_libcrypto_a_99560c9c37f156ab8.lib(p5_scrypt.obj)
0001:00201c70* _d2i_SCRYPT_PARAMS
0001:002025b4* _SCRYPT_PARAMS_it
0001:00201ca0* _i2d_SCRYPT_PARAMS
0001:00201cd0* _SCRYPT_PARAMS_new
0001:00201cf0* _SCRYPT_PARAMS_free
0001:00201d30* _PKCS5_pbe2_set_scrypt
0001:002022a0  _PKCS5_v2_scrypt_keyivgen
Module: U:\tmp\ldconv_libcrypto_a_99560c9c37f156ab8.lib(md5-586.obj)
0001:00202690  _md5_block_asm_data_order
Module: U:\tmp\ldconv_libcrypto_a_99560c9c37f156ab8.lib(rsa_chk.obj)
0001:00203730* _RSA_check_key
0001:002037a0  _RSA_check_key_ex
Module: U:\tmp\ldconv_libcrypto_a_99560c9c37f156ab8.lib(t_pkey.obj)
0001:00203830  _ASN1_buf_print
0001:00203960  _ASN1_bn_print
Module: U:\tmp\ldconv_libcrypto_a_99560c9c37f156ab8.lib(cms_sd.obj)
0001:00203b60* _CMS_SignedData_init
0001:00203c60  _cms_set1_SignerIdentifier
0001:00203d00  _cms_SignerIdentifier_get0_signer_id
0001:00203d70  _cms_SignerIdentifier_cert_cmp
0001:00203db0  _CMS_SignerInfo_get0_pkey_ctx
0001:00203dc0* _CMS_SignerInfo_get0_md_ctx
0001:00203dd0* _CMS_get0_SignerInfos
0001:00203e40* _CMS_get0_signers
0001:00203f20* _CMS_SignerInfo_set1_signer_cert
0001:00203f70* _CMS_SignerInfo_get0_signer_id
0001:00203fe0* _CMS_SignerInfo_cert_cmp
0001:00204020* _CMS_set1_signers_certs
0001:002042a0  _CMS_SignerInfo_get0_algs
0001:002042e0* _CMS_SignerInfo_get0_signature
0001:002042f0* _CMS_SignerInfo_sign
0001:00204640  _cms_SignedData_final
0001:00204ba0* _CMS_SignerInfo_verify
0001:00204e20  _cms_SignedData_init_bio
0001:00205040* _CMS_SignerInfo_verify_content
0001:002053a0* _CMS_add_smimecap
0001:00205420* _CMS_add_simple_smimecap
0001:00205510* _CMS_add_standard_smimecap
0001:00205b30* _CMS_add1_signer
Module: U:\tmp\ldconv_libcrypto_a_99560c9c37f156ab8.lib(cms_env.obj)
0001:00206440  _cms_get0_enveloped
0001:002064a0  _cms_env_asn1_ctrl
0001:00206590* _CMS_get0_RecipientInfos
0001:00206600* _CMS_RecipientInfo_type
0001:00206610  _CMS_RecipientInfo_get0_pkey_ctx
0001:00206650* _CMS_EnvelopedData_create
0001:002067c0* _CMS_add1_recipient_cert
0001:00206a60  _CMS_RecipientInfo_ktri_get0_algs
0001:00206af0* _CMS_RecipientInfo_ktri_get0_signer_id
0001:00206b50* _CMS_RecipientInfo_ktri_cert_cmp
0001:00206bb0* _CMS_RecipientInfo_set0_pkey
0001:00206c20* _CMS_RecipientInfo_kekri_id_cmp
0001:00206cb0* _CMS_add0_recipient_key
0001:00206f50* _CMS_RecipientInfo_kekri_get0_id
0001:00207030* _CMS_RecipientInfo_set0_key
0001:002070a0* _CMS_RecipientInfo_decrypt
0001:002076c0* _CMS_RecipientInfo_encrypt
0001:00207b40  _cms_EnvelopedData_init_bio
0001:00207db0* _cms_pkey_get_ri_type
Module: U:\tmp\ldconv_libcrypto_a_99560c9c37f156ab8.lib(cms_kari.obj)
0001:00207fe0  _CMS_RecipientInfo_kari_get0_alg
0001:00208060* _CMS_RecipientInfo_kari_get0_reks
0001:002080c0  _CMS_RecipientInfo_kari_get0_orig_id
0001:002081f0* _CMS_RecipientInfo_kari_orig_id_cmp
0001:00208270* _CMS_RecipientEncryptedKey_get0_id
0001:00208340* _CMS_RecipientEncryptedKey_cert_cmp
0001:00208380* _CMS_RecipientInfo_kari_set0_pkey
0001:00208400  _CMS_RecipientInfo_kari_get0_ctx
0001:00208420* _CMS_RecipientInfo_kari_decrypt
0001:00208510  _cms_RecipientInfo_kari_init
0001:002086c0  _cms_RecipientInfo_kari_encrypt
Module: U:\tmp\ldconv_libcrypto_a_99560c9c37f156ab8.lib(cms_asn1.obj)
0001:00208b80  _CMS_SharedInfo_encode
0001:00208c98* _CMS_Receipt_it
0001:00208d74* _CMS_ReceiptRequest_it
0001:00208e90  _CMS_Attributes_Verify_it
0001:00208ee4  _CMS_Attributes_Sign_it
0001:00208f24  _CMS_ContentInfo_it
0001:00209e28  _CMS_SignedData_it
0001:00209434  _CMS_EnvelopedData_it
0001:002093a0  _CMS_DigestedData_it
0001:002092f8  _CMS_EncryptedData_it
0001:00209108* _CMS_CompressedData_it
0001:002094c8  _CMS_RecipientInfo_it
0001:00209c94  _CMS_KeyTransRecipientInfo_it
0001:00209828  _CMS_KeyAgreeRecipientInfo_it
0001:002096f8  _CMS_KEKRecipientInfo_it
0001:00209634  _CMS_PasswordRecipientInfo_it
0001:00209c04  _CMS_OtherKeyAttribute_it
0001:00209a54  _CMS_RecipientEncryptedKey_it
0001:0020a374  _CMS_IssuerAndSerialNumber_it
0001:002099c4  _CMS_OriginatorPublicKey_it
0001:00209b74  _CMS_RecipientKeyIdentifier_it
0001:0020a210  _CMS_CertificateChoices_it
0001:00209f04  _CMS_RevocationInfoChoice_it
0001:0020a008  _CMS_SignerInfo_it
Module: U:\tmp\ldconv_libcrypto_a_99560c9c37f156ab8.lib(ec_check.obj)
0001:0020a410  _EC_GROUP_check
Module: U:\tmp\ldconv_libcrypto_a_99560c9c37f156ab8.lib(eck_prn.obj)
0001:0020a6b0* _EC_KEY_print_fp
0001:0020a750* _ECParameters_print_fp
0001:0020a8b0  _ECPKParameters_print
0001:0020b040* _ECPKParameters_print_fp
Module: U:\tmp\ldconv_libcrypto_a_99560c9c37f156ab8.lib(curve25519.obj)
0001:00211420  _ED25519_sign
0001:00214b20  _ED25519_verify
0001:00217ae0  _ED25519_public_from_private
0001:00217bc0  _X25519
0001:00217c00  _X25519_public_from_private
Module: U:\tmp\ldconv_libcrypto_a_99560c9c37f156ab8.lib(eddsa.obj)
0001:0021fd70* _c448_ed448_convert_private_key_to_x448
0001:0021fe00* _c448_ed448_derive_public_key
0001:0021ff30* _c448_ed448_sign
0001:00220380* _c448_ed448_sign_prehash
0001:002203d0* _c448_ed448_verify
0001:00220460* _c448_ed448_verify_prehash
0001:002204d0  _ED448_sign
0001:00220530  _ED448_verify
0001:002205a0* _ED448ph_sign
0001:00220600* _ED448ph_verify
0001:00220670  _ED448_public_from_private
Module: U:\tmp\ldconv_libcrypto_a_99560c9c37f156ab8.lib(m_null.obj)
0001:00220710  _EVP_md_null
Module: U:\tmp\ldconv_libcrypto_a_99560c9c37f156ab8.lib(curve448.obj)
0001:00222cd0* _curve448_point_double
0001:00222ce0  _curve448_point_eq
0001:00222d40* _curve448_point_valid
0001:00222e60  _curve448_precomputed_scalarmul
0001:002235d0  _curve448_point_mul_by_ratio_and_encode_like_eddsa
0001:00223900  _curve448_point_decode_like_eddsa_and_mul_by_ratio
0001:00223e30* _x448_int
0001:00226010* _curve448_point_mul_by_ratio_and_encode_like_x448
0001:002261a0* _x448_derive_public_key
0001:00226420  _curve448_base_double_scalarmul_non_secret
0001:00227c80* _curve448_point_identity
0001:00227c10  _curve448_point_destroy
0001:00227c30  _X448
0001:00227c60  _X448_public_from_private
Module: U:\tmp\ldconv_libcrypto_a_99560c9c37f156ab8.lib(dso_openssl.obj)
0001:00227e40  _DSO_METHOD_openssl
Module: U:\tmp\ldconv_libcrypto_a_99560c9c37f156ab8.lib(rsa_pk1.obj)
0001:00227e90  _RSA_padding_add_PKCS1_type_1
0001:00227f40  _RSA_padding_check_PKCS1_type_1
0001:00228150  _RSA_padding_add_PKCS1_type_2
0001:00228250  _RSA_padding_check_PKCS1_type_2
Module: U:\tmp\ldconv_libcrypto_a_99560c9c37f156ab8.lib(rsa_x931.obj)
0001:00228590  _RSA_padding_add_X931
0001:00228640  _RSA_padding_check_X931
0001:002287a0  _RSA_X931_hash_id
Module: U:\tmp\ldconv_libcrypto_a_99560c9c37f156ab8.lib(rsa_ssl.obj)
0001:00228810  _RSA_padding_add_SSLv23
0001:00228920  _RSA_padding_check_SSLv23
Module: U:\tmp\ldconv_libcrypto_a_99560c9c37f156ab8.lib(rsa_oaep.obj)
0001:00228cf0  _PKCS1_MGF1
0001:00228e80  _RSA_padding_add_PKCS1_OAEP_mgf1
0001:002293c0  _RSA_padding_check_PKCS1_OAEP_mgf1
0001:00229cc0  _RSA_padding_check_PKCS1_OAEP
0001:00229d20  _RSA_padding_add_PKCS1_OAEP
Module: U:\tmp\ldconv_libcrypto_a_99560c9c37f156ab8.lib(rsa_none.obj)
0001:0022a240  _RSA_padding_add_none
0001:0022a2e0* _RSA_padding_check_none
Module: U:\tmp\ldconv_libcrypto_a_99560c9c37f156ab8.lib(bn_exp2.obj)
0001:0022a390  _BN_mod_exp2_mont
Module: U:\tmp\ldconv_libcrypto_a_99560c9c37f156ab8.lib(ecdsa_sign.obj)
0001:0022ac90* _ECDSA_do_sign
0001:0022ad10  _ECDSA_do_sign_ex
0001:0022ad60  _ECDSA_sign
0001:0022adf0* _ECDSA_sign_ex
0001:0022ae40* _ECDSA_sign_setup
Module: U:\tmp\ldconv_libcrypto_a_99560c9c37f156ab8.lib(ecdsa_vrf.obj)
0001:0022aeb0  _ECDSA_do_verify
0001:0022af00  _ECDSA_verify
Module: U:\tmp\ldconv_libcrypto_a_99560c9c37f156ab8.lib(bn_gf2m.obj)
0001:0022af50  _BN_GF2m_add
0001:0022b010  _BN_GF2m_mod_arr
0001:0022b2f0* _BN_GF2m_mod
0001:0022b400  _BN_GF2m_mod_sqr_arr
0001:0022b670  _BN_GF2m_mod_mul_arr
0001:0022bc50* _BN_GF2m_mod_exp_arr
0001:0022bde0  _BN_GF2m_mod_sqrt_arr
0001:0022be90  _BN_GF2m_mod_solve_quad_arr
0001:0022bee0  _BN_GF2m_poly2arr
0001:0022bfa0* _BN_GF2m_mod_mul
0001:0022c080  _BN_GF2m_mod_inv
0001:0022c680* _BN_GF2m_mod_inv_arr
0001:0022c710  _BN_GF2m_mod_div
0001:0022c7a0* _BN_GF2m_mod_div_arr
0001:0022c880* _BN_GF2m_mod_sqr
0001:0022c950* _BN_GF2m_mod_exp
0001:0022ca30* _BN_GF2m_mod_sqrt
0001:0022cb80* _BN_GF2m_mod_solve_quad
0001:0022cc70* _BN_GF2m_arr2poly
Module: U:\tmp\ldconv_libcrypto_a_99560c9c37f156ab8.lib(bn_sqrt.obj)
0001:0022ccf0  _BN_mod_sqrt
Module: U:\tmp\ldconv_libcrypto_a_99560c9c37f156ab8.lib(bn_kron.obj)
0001:0022d6b0  _BN_kronecker
Module: U:\tmp\ldconv_libcrypto_a_99560c9c37f156ab8.lib(co-586.obj)
0001:0022d930  _bn_mul_comba8
0001:0022dd80* _bn_mul_comba4
0001:0022dec0  _bn_sqr_comba8
0001:0022e1f0  _bn_sqr_comba4
Module: U:\tmp\ldconv_libcrypto_a_99560c9c37f156ab8.lib(asn_moid.obj)
0001:0022e550  _ASN1_add_oid_module
Module: U:\tmp\ldconv_libcrypto_a_99560c9c37f156ab8.lib(asn_mstbl.obj)
0001:0022ea40  _ASN1_add_stable_module
Module: U:\tmp\ldconv_libcrypto_a_99560c9c37f156ab8.lib(eng_cnf.obj)
0001:0022f0f0  _ENGINE_add_conf_module
Module: U:\tmp\ldconv_libcrypto_a_99560c9c37f156ab8.lib(evp_cnf.obj)
0001:0022f320  _EVP_add_alg_module
Module: U:\tmp\ldconv_libcrypto_a_99560c9c37f156ab8.lib(mdc2dgst.obj)
0001:0022f470  _MDC2_Init
0001:0022f4b0  _MDC2_Update
0001:0022f590  _MDC2_Final
Module: U:\tmp\ldconv_libcrypto_a_99560c9c37f156ab8.lib(rmd_dgst.obj)
0001:0022f620  _RIPEMD160_Update
0001:0022f780* _RIPEMD160_Transform
0001:0022f7b0  _RIPEMD160_Final
0001:0022f8f0  _RIPEMD160_Init
Module: U:\tmp\ldconv_libcrypto_a_99560c9c37f156ab8.lib(wp_dgst.obj)
0001:0022f950  _WHIRLPOOL_Init
0001:0022f990* _WHIRLPOOL_BitUpdate
0001:0022fe00  _WHIRLPOOL_Update
0001:0022feb0  _WHIRLPOOL_Final
0001:00230100* _WHIRLPOOL
Module: U:\tmp\ldconv_libcrypto_a_99560c9c37f156ab8.lib(sm3.obj)
0001:002301f0  _sm3_init
0001:00230260* _sm3_block_data_order
0001:00232b20  _sm3_update
0001:00232c80* _sm3_transform
0001:00232cb0  _sm3_final
Module: U:\tmp\ldconv_libcrypto_a_99560c9c37f156ab8.lib(blake2b.obj)
0001:0023b630  _BLAKE2b_Init
0001:0023b740  _BLAKE2b_Update
0001:0023b820  _BLAKE2b_Final
Module: U:\tmp\ldconv_libcrypto_a_99560c9c37f156ab8.lib(blake2s.obj)
0001:0023d0a0  _BLAKE2s_Init
0001:0023d110  _BLAKE2s_Update
0001:0023d1d0  _BLAKE2s_Final
Module: U:\tmp\ldconv_libcrypto_a_99560c9c37f156ab8.lib(keccak1600.obj)
0001:0023da70  _SHA3_absorb
0001:0023dbf0  _SHA3_squeeze
Module: U:\tmp\ldconv_libcrypto_a_99560c9c37f156ab8.lib(xcbc_enc.obj)
0001:0023df20  _DES_xcbc_encrypt
Module: U:\tmp\ldconv_libcrypto_a_99560c9c37f156ab8.lib(sm4.obj)
0001:0023e490  _SM4_set_key
0001:0023e590  _SM4_encrypt
0001:0023f0a0  _SM4_decrypt
Module: U:\tmp\ldconv_libcrypto_a_99560c9c37f156ab8.lib(bf-586.obj)
0001:00240130  _BF_encrypt
0001:00240550  _BF_decrypt
0001:00240970  _BF_cbc_encrypt
Module: U:\tmp\ldconv_libcrypto_a_99560c9c37f156ab8.lib(bf_skey.obj)
0001:00240bb0  _BF_set_key
Module: U:\tmp\ldconv_libcrypto_a_99560c9c37f156ab8.lib(bf_cfb64.obj)
0001:00241d50  _BF_cfb64_encrypt
Module: U:\tmp\ldconv_libcrypto_a_99560c9c37f156ab8.lib(bf_ofb64.obj)
0001:00241ec0  _BF_ofb64_encrypt
Module: U:\tmp\ldconv_libcrypto_a_99560c9c37f156ab8.lib(bf_ecb.obj)
0001:00241fd0* _BF_options
0001:00241fe0  _BF_ecb_encrypt
Module: U:\tmp\ldconv_libcrypto_a_99560c9c37f156ab8.lib(cast-586.obj)
0001:00242040  _CAST_encrypt
0001:002424e0  _CAST_decrypt
0001:00242970  _CAST_cbc_encrypt
Module: U:\tmp\ldconv_libcrypto_a_99560c9c37f156ab8.lib(c_skey.obj)
0001:00242bc0  _CAST_set_key
0001:00244000* _CAST_S_table5
0001:00243c00* _CAST_S_table6
0001:00244400* _CAST_S_table4
0001:00243800* _CAST_S_table7
0001:00244800  _CAST_S_table3
0001:00244c00  _CAST_S_table2
0001:00245000  _CAST_S_table1
0001:00245400  _CAST_S_table0
Module: U:\tmp\ldconv_libcrypto_a_99560c9c37f156ab8.lib(c_cfb64.obj)
0001:00245800  _CAST_cfb64_encrypt
Module: U:\tmp\ldconv_libcrypto_a_99560c9c37f156ab8.lib(c_ofb64.obj)
0001:00245970  _CAST_ofb64_encrypt
Module: U:\tmp\ldconv_libcrypto_a_99560c9c37f156ab8.lib(c_ecb.obj)
0001:00245a70  _CAST_ecb_encrypt
Module: U:\tmp\ldconv_libcrypto_a_99560c9c37f156ab8.lib(store_lib.obj)
0001:00245af0* _OSSL_STORE_open
0001:00245cd0* _OSSL_STORE_ctrl
0001:00245d00* _OSSL_STORE_vctrl
0001:00245d30* _OSSL_STORE_expect
0001:00245db0* _OSSL_STORE_find
0001:00245e40* _OSSL_STORE_error
0001:00245e50* _OSSL_STORE_eof
0001:00245e60* _OSSL_STORE_close
0001:00245eb0  _OSSL_STORE_INFO_new_NAME
0001:00245f30* _OSSL_STORE_INFO_set0_NAME_description
0001:00245f90  _OSSL_STORE_INFO_new_PARAMS
0001:00246000  _OSSL_STORE_INFO_new_PKEY
0001:00246070  _OSSL_STORE_INFO_new_CERT
0001:002460e0  _OSSL_STORE_INFO_new_CRL
0001:00246150  _OSSL_STORE_INFO_get_type
0001:00246160* _OSSL_STORE_INFO_get0_NAME
0001:00246180* _OSSL_STORE_INFO_get1_NAME
0001:00246220* _OSSL_STORE_INFO_get0_NAME_description
0001:00246240* _OSSL_STORE_INFO_get1_NAME_description
0001:002462f0* _OSSL_STORE_INFO_get0_PARAMS
0001:00246310* _OSSL_STORE_INFO_get1_PARAMS
0001:00246370* _OSSL_STORE_INFO_get0_PKEY
0001:00246390* _OSSL_STORE_INFO_get1_PKEY
0001:002463f0* _OSSL_STORE_INFO_get0_CERT
0001:00246410* _OSSL_STORE_INFO_get1_CERT
0001:00246470* _OSSL_STORE_INFO_get0_CRL
0001:00246490* _OSSL_STORE_INFO_get1_CRL
0001:002464f0  _OSSL_STORE_INFO_free
0001:002465f0* _OSSL_STORE_load
0001:00246680* _OSSL_STORE_supports_search
0001:002466c0* _OSSL_STORE_SEARCH_by_name
0001:00246730* _OSSL_STORE_SEARCH_by_issuer_serial
0001:002467d0* _OSSL_STORE_SEARCH_by_key_fingerprint
0001:00246930* _OSSL_STORE_SEARCH_by_alias
0001:002469b0* _OSSL_STORE_SEARCH_free
0001:002469e0  _OSSL_STORE_SEARCH_get_type
0001:002469f0  _OSSL_STORE_SEARCH_get0_name
0001:00246a00* _OSSL_STORE_SEARCH_get0_serial
0001:00246a10* _OSSL_STORE_SEARCH_get0_bytes
0001:00246a30* _OSSL_STORE_SEARCH_get0_string
0001:00246a40* _OSSL_STORE_SEARCH_get0_digest
0001:00246a50  _ossl_store_info_new_EMBEDDED
0001:00246b40  _ossl_store_info_get0_EMBEDDED_buffer
0001:00246b60  _ossl_store_info_get0_EMBEDDED_pem_name
0001:00246b80* _ossl_store_attach_pem_bio
0001:00246c50* _ossl_store_detach_pem_bio
Module: U:\tmp\ldconv_libcrypto_a_99560c9c37f156ab8.lib(poly1305-x86.obj)
0001:00246c90  _poly1305_init
0001:00246cf0  _poly1305_blocks
0001:00246ed0  _poly1305_emit
Module: U:\tmp\ldconv_libcrypto_a_99560c9c37f156ab8.lib(rsa_gen.obj)
0001:002479e0* _RSA_generate_key_ex
0001:00247a60  _RSA_generate_multi_prime_key
Module: U:\tmp\ldconv_libcrypto_a_99560c9c37f156ab8.lib(rsa_pss.obj)
0001:00247b00* _RSA_verify_PKCS1_PSS
0001:002480c0  _RSA_verify_PKCS1_PSS_mgf1
0001:00248680* _RSA_padding_add_PKCS1_PSS
0001:00248ac0  _RSA_padding_add_PKCS1_PSS_mgf1
Module: U:\tmp\ldconv_libcrypto_a_99560c9c37f156ab8.lib(rsa_saos.obj)
0001:00248f50  _RSA_sign_ASN1_OCTET_STRING
0001:002490b0* _RSA_verify_ASN1_OCTET_STRING
Module: U:\tmp\ldconv_libcrypto_a_99560c9c37f156ab8.lib(rsa_sign.obj)
0001:00249380  _RSA_sign
0001:00249510  _int_rsa_verify
0001:00249930  _RSA_verify
Module: U:\tmp\ldconv_libcrypto_a_99560c9c37f156ab8.lib(dh_kdf.obj)
0001:002499c0  _DH_KDF_X9_42
Module: U:\tmp\ldconv_libcrypto_a_99560c9c37f156ab8.lib(dsa_gen.obj)
0001:00249de0  _dsa_builtin_paramgen
0001:0024a7f0* _DSA_generate_parameters_ex
0001:0024a8d0  _dsa_builtin_paramgen2
Module: U:\tmp\ldconv_libcrypto_a_99560c9c37f156ab8.lib(dh_rfc5114.obj)
0001:0024b5b0  _DH_get_1024_160
0001:0024b620  _DH_get_2048_224
0001:0024b690  _DH_get_2048_256
Module: U:\tmp\ldconv_libcrypto_a_99560c9c37f156ab8.lib(dh_rfc7919.obj)
0001:0024b720  _DH_new_by_nid
0001:0024b850* _DH_get_nid
Module: U:\tmp\ldconv_libcrypto_a_99560c9c37f156ab8.lib(dsa_key.obj)
0001:0024b980  _DSA_generate_key
Module: U:\tmp\ldconv_libcrypto_a_99560c9c37f156ab8.lib(ecdh_kdf.obj)
0001:0024bc20  _ecdh_KDF_X9_63
0001:0024bca0* _ECDH_KDF_X9_62
Module: U:\tmp\ldconv_libcrypto_a_99560c9c37f156ab8.lib(pbe_scrypt.obj)
0001:0024c4a0  _EVP_PBE_scrypt
Module: U:\tmp\ldconv_libgcc_a_99560c9c382191438.lib(_udivdi3.obj)
0001:0024cc20  ___udivdi3
Module: U:\tmp\ldconv_libcrypto_a_99560c9c37f156ab8.lib(siphash.obj)
0001:0024cd20* _SipHash_ctx_size
0001:0024cd30  _SipHash_hash_size
0001:0024cd40  _SipHash_set_hash_size
0001:0024cdb0  _SipHash_Init
0001:0024ce90  _SipHash_Update
0001:0024d300  _SipHash_Final
Module: U:\tmp\ldconv_libcrypto_a_99560c9c37f156ab8.lib(sm2_crypt.obj)
0001:0024d900* _d2i_SM2_Ciphertext
0001:0024ec64* _SM2_Ciphertext_it
0001:0024d930* _i2d_SM2_Ciphertext
0001:0024d960* _SM2_Ciphertext_new
0001:0024d980* _SM2_Ciphertext_free
0001:0024d9c0  _sm2_plaintext_size
0001:0024dac0  _sm2_ciphertext_size
0001:0024db80  _sm2_encrypt
0001:0024e420  _sm2_decrypt
Module: U:\tmp\ldconv_libcrypto_a_99560c9c37f156ab8.lib(sm2_sign.obj)
0001:0024f400  _sm2_compute_z_digest
0001:0024fba0* _sm2_do_sign
0001:0024fc10* _sm2_do_verify
0001:0024fc70  _sm2_sign
0001:0024fd50  _sm2_verify
Module: U:\tmp\ldconv_libcrypto_a_99560c9c37f156ab8.lib(bio_md.obj)
0001:00250400  _BIO_f_md
Module: U:\tmp\ldconv_libcrypto_a_99560c9c37f156ab8.lib(bio_enc.obj)
0001:00250e60  _BIO_f_cipher
0001:00250e70* _BIO_set_cipher
Module: U:\tmp\ldconv_libcrypto_a_99560c9c37f156ab8.lib(bss_null.obj)
0001:00251070  _BIO_s_null
Module: U:\tmp\ldconv_libcrypto_a_99560c9c37f156ab8.lib(pk7_attr.obj)
0001:002510f0* _PKCS7_add_attrib_smimecap
0001:00251180* _PKCS7_get_smimecap
0001:002511e0* _PKCS7_simple_smimecap
0001:00251300* _PKCS7_add_attrib_content_type
0001:00251370  _PKCS7_add0_attrib_signing_time
0001:002513f0  _PKCS7_add1_attrib_digest
Module: U:\tmp\ldconv_libcrypto_a_99560c9c37f156ab8.lib(dsa_sign.obj)
0001:00251460  _DSA_do_sign
0001:00251470* _DSA_sign_setup
Module: U:\tmp\ldconv_libcrypto_a_99560c9c37f156ab8.lib(dsa_vrf.obj)
0001:00251480  _DSA_do_verify
Module: U:\tmp\ldconv_libcrypto_a_99560c9c37f156ab8.lib(ct_prn.obj)
0001:002514a0* _SCT_validation_status_string
0001:002515a0* _SCT_print
0001:002519e0  _SCT_LIST_print
Module: U:\tmp\ldconv_libgcc_eh_a_99560c9c382174360.lib(unwind-dw2-fde.obj)
0001:002528cc* ___register_frame_info_bases
0001:002528f2* ___register_frame_info
0001:00252916* ___register_frame
0001:0025294f* ___register_frame_info_table_bases
0001:002529b2* ___register_frame_info_table
0001:002529dc  ___register_frame_table
0001:00252a0f* ___deregister_frame_info_bases
0001:00252ae0* ___deregister_frame_info
0001:00252ae5  ___deregister_frame
0001:00252b07* __Unwind_Find_FDE
Module: U:\tmp\ldconv_libcrypto_a_99560c9c37f156ab8.lib(cms_lib.obj)
0001:00252c70  _d2i_CMS_ContentInfo
0001:00252ca0  _i2d_CMS_ContentInfo
0001:00252cd0  _CMS_ContentInfo_new
0001:00252cf0  _CMS_ContentInfo_free
0001:00252d10* _CMS_ContentInfo_print_ctx
0001:00252d50* _CMS_get0_type
0001:00252d70* _cms_Data_create
0001:00252ed0* _cms_content_bio
0001:00253000  _CMS_dataFinal
0001:002532b0  _CMS_get0_content
0001:002533b0  _CMS_dataInit
0001:00253550  _CMS_get0_eContentType
0001:00253610* _CMS_set1_eContentType
0001:00253720* _CMS_is_detached
0001:00253800* _CMS_set_detached
0001:00253970  _cms_DigestAlgorithm_init_bio
0001:00253a70  _cms_DigestAlgorithm_find_ctx
0001:00253b80* _CMS_add0_CertificateChoices
0001:00253c50* _CMS_add0_cert
0001:00253d80  _CMS_add1_cert
0001:00253db0* _CMS_add0_RevocationInfoChoice
0001:00253e80* _CMS_add0_crl
0001:00253f70* _CMS_add1_crl
0001:00254060* _CMS_get1_certs
0001:00254160* _CMS_get1_crls
0001:00254260  _cms_ias_cert_cmp
0001:002542b0  _cms_keyid_cert_cmp
0001:002542f0  _cms_set1_ias
0001:002543c0  _cms_set1_keyid
Module: U:\tmp\ldconv_libcrypto_a_99560c9c37f156ab8.lib(cms_att.obj)
0001:00254470  _CMS_signed_get_attr_count
0001:00254480  _CMS_signed_get_attr_by_NID
0001:00254490* _CMS_signed_get_attr_by_OBJ
0001:002544a0* _CMS_signed_get_attr
0001:002544b0* _CMS_signed_delete_attr
0001:002544c0* _CMS_signed_add1_attr
0001:002544f0* _CMS_signed_add1_attr_by_OBJ
0001:00254530  _CMS_signed_add1_attr_by_NID
0001:00254570* _CMS_signed_add1_attr_by_txt
0001:002545b0  _CMS_signed_get0_data_by_OBJ
0001:002545c0* _CMS_unsigned_get_attr_count
0001:002545d0* _CMS_unsigned_get_attr_by_NID
0001:002545e0* _CMS_unsigned_get_attr_by_OBJ
0001:002545f0* _CMS_unsigned_get_attr
0001:00254600* _CMS_unsigned_delete_attr
0001:00254610* _CMS_unsigned_add1_attr
0001:00254640* _CMS_unsigned_add1_attr_by_OBJ
0001:00254680* _CMS_unsigned_add1_attr_by_NID
0001:002546c0* _CMS_unsigned_add1_attr_by_txt
0001:00254700* _CMS_unsigned_get0_data_by_OBJ
0001:00254730  _CMS_si_check_attributes
Module: U:\tmp\ldconv_libcrypto_a_99560c9c37f156ab8.lib(cms_enc.obj)
0001:002549f0  _cms_EncryptedContent_init_bio
0001:00255060  _cms_EncryptedContent_init
0001:00255110* _CMS_EncryptedData_set1_key
0001:00255320  _cms_EncryptedData_init_bio
Module: U:\tmp\ldconv_libcrypto_a_99560c9c37f156ab8.lib(aes_wrap.obj)
0001:00255350  _AES_wrap_key
0001:00255390  _AES_unwrap_key
Module: U:\tmp\ldconv_libcrypto_a_99560c9c37f156ab8.lib(cms_pwri.obj)
0001:002553f0* _CMS_RecipientInfo_set0_password
0001:00255480* _CMS_add0_recipient_password
0001:00255910  _cms_RecipientInfo_pwri_crypt
Module: U:\tmp\ldconv_libcrypto_a_99560c9c37f156ab8.lib(cms_io.obj)
0001:00256110  _CMS_stream
0001:002561a0* _d2i_CMS_bio
0001:002561d0* _i2d_CMS_bio
0001:00256200* _PEM_read_bio_CMS
0001:00256240* _PEM_read_CMS
0001:00256280* _PEM_write_bio_CMS
0001:002562e0* _PEM_write_CMS
0001:00256340* _BIO_new_CMS
0001:00256370* _i2d_CMS_bio_stream
0001:002563b0* _PEM_write_bio_CMS_stream
0001:002563f0* _SMIME_write_CMS
0001:00256460* _SMIME_read_CMS
Module: U:\tmp\ldconv_libcrypto_a_99560c9c37f156ab8.lib(ec_print.obj)
0001:002564b0  _EC_POINT_point2bn
0001:00256530* _EC_POINT_bn2point
0001:002566e0* _EC_POINT_point2hex
0001:002567e0* _EC_POINT_hex2point
Module: U:\tmp\ldconv_libcrypto_a_99560c9c37f156ab8.lib(scalar.obj)
0001:00257330  _curve448_scalar_mul
0001:00257360  _curve448_scalar_sub
0001:002576a0  _curve448_scalar_add
0001:00257b80* _curve448_scalar_decode
0001:00258d40* _curve448_scalar_one
0001:00257d40  _curve448_scalar_destroy
0001:00257d60  _curve448_scalar_decode_long
0001:00258d00  _curve448_scalar_zero
0001:00258810  _curve448_scalar_encode
0001:00258990  _curve448_scalar_halve
Module: U:\tmp\ldconv_libcrypto_a_99560c9c37f156ab8.lib(curve448_tables.obj)
0002:00004760  _curve448_wnaf_base
0002:00004764  _curve448_precomputed_base
Module: U:\tmp\ldconv_libcrypto_a_99560c9c37f156ab8.lib(f_impl.obj)
0001:0025e1c0  _gf_mul
0001:0025e870  _gf_mulw_unsigned
0001:0025ead0  _gf_sqr
Module: U:\tmp\ldconv_libcrypto_a_99560c9c37f156ab8.lib(f_generic.obj)
0001:0025eaf0* _gf_strong_reduce
0001:0025f0c0  _gf_serialize
0001:0025f220  _gf_lobit
0001:0025f2b0* _gf_hibit
0001:0025f4c0  _gf_deserialize
0001:0025f8f0  _gf_sub
0001:0025fb30  _gf_add
0001:0025fd50  _gf_eq
0001:00260070  _gf_isr
Module: U:\tmp\ldconv_libcrypto_a_99560c9c37f156ab8.lib(x86-gf2m.obj)
0001:00260650  _bn_GF2m_mul_2x2
Module: U:\tmp\ldconv_libcrypto_a_99560c9c37f156ab8.lib(rmd-586.obj)
0001:00260710  _ripemd160_block_asm_data_order
Module: U:\tmp\ldconv_libcrypto_a_99560c9c37f156ab8.lib(wp_block.obj)
0001:00261c00  _whirlpool_block
Module: U:\tmp\ldconv_libcrypto_a_99560c9c37f156ab8.lib(bn_dh.obj)
0001:00263e20  __bignum_ffdhe8192_p
0001:00263e34  __bignum_ffdhe6144_p
0001:00263e48  __bignum_ffdhe4096_p
0001:00263e5c  __bignum_ffdhe3072_p
0001:00263e70  __bignum_ffdhe2048_p
0001:00263e84  __bignum_dh2048_256_q
0001:00263e98  __bignum_dh2048_256_g
0001:00263eac  __bignum_dh2048_256_p
0001:00263ec0  __bignum_dh2048_224_q
0001:00263ed4  __bignum_dh2048_224_g
0001:00263ee8  __bignum_dh2048_224_p
0001:00263efc  __bignum_dh1024_160_q
0001:00263f10  __bignum_dh1024_160_g
0001:00263f24  __bignum_dh1024_160_p
0001:00263f38  __bignum_const_2
Module: U:\tmp\ldconv_libgcc_a_99560c9c382191438.lib(gthr-os2.obj)
0001:0026536b* ___gthread_os2_mutex_init
0001:0026539e* ___gthread_os2_mutex_destroy
0001:002653be  ___gthread_os2_mutex_lock
0001:002653d2* ___gthread_os2_mutex_trylock
0001:002653e3  ___gthread_os2_mutex_unlock
0001:00265403* ___gthread_os2_cond_init
0001:002655c5* ___gthread_os2_cond_destroy
0001:00265603* ___gthread_os2_cond_wait
0001:00265628* ___gthread_os2_cond_wait_recursive
0001:0026564f* ___gthread_os2_create
0001:00265739* ___gthread_os2_join
0001:002657b1* ___gthread_os2_detach
0001:002657ef* ___gthread_os2_equal
0001:00265800* ___gthread_os2_self
0001:00265805* ___gthread_os2_yield
0001:0026581b* ___gthread_os2_mutex_timedlock
0001:00265840* ___gthread_os2_recursive_mutex_timedlock
0001:00265868* ___gthread_os2_cond_signal
0001:002658d9* ___gthread_os2_cond_broadcast
0001:0026592c* ___gthread_os2_cond_timedwait
Module: U:\tmp\ldconv_libcrypto_a_99560c9c37f156ab8.lib(cms_dd.obj)
0001:00265970* _cms_DigestedData_create
0001:002659f0  _cms_DigestedData_init_bio
0001:00265a20  _cms_DigestedData_do_final
Module: U:\tmp\ldconv_libcrypto_a_99560c9c37f156ab8.lib(bio_ndef.obj)
0001:00265e60  _BIO_new_NDEF
Module: U:\tmp\ldconv_libcrypto_a_99560c9c37f156ab8.lib(asn_mime.obj)
0001:002670f0  _SMIME_read_ASN1
0001:00267670* _SMIME_crlf_copy
0001:002678a0  _i2d_ASN1_bio_stream
0001:00267b20  _PEM_write_bio_ASN1_stream
0001:00267e20  _SMIME_write_ASN1
0001:00268600* _SMIME_text
Module: U:\tmp\ldconv_libcrypto_a_99560c9c37f156ab8.lib(bio_asn1.obj)
0001:00269040  _BIO_f_asn1
0001:00269050  _BIO_asn1_set_prefix
0001:00269090* _BIO_asn1_get_prefix
0001:002690e0  _BIO_asn1_set_suffix
0001:00269120* _BIO_asn1_get_suffix


                        +----------------------+
                        |   Imported Symbols   |
                        +----------------------+

Symbol                              Module
======                              ======

___libc_ForkRegisterModule          libcn0
___init_app                         libcx0
__CRT_init                          libcn0
__atfork_callback                   libcn0
_pthread_setspecific                pthr01
_pthread_key_create                 pthr01
_pthread_getspecific                pthr01
_close                              libcx0
_read                               libcx0
_getnameinfo                        libcx0
__exit                              libcn0
_getservbyname                      tcpip32
_pthread_detach                     pthr01
__errno                             libcn0
___libc_GLocaleCtype                libcn0
___stderrp                          libcn0
_getpwnam                           libcn0
_poll                               libcx0
_pthread_exit                       pthr01
_getaddrinfo                        libcx0
_freeaddrinfo                       libcx0
_pthread_self                       pthr01
_pthread_create                     pthr01
_pthread_join                       pthr01
_pthread_attr_init                  pthr01
_pthread_attr_setstacksize          pthr01
_pthread_attr_destroy               pthr01
_fcntl                              libcx0
_wait                               libcx0
_waitpid                            libcx0
DosLoadModule                       doscalls
DosGetInfoBlocks                    doscalls
DosQueryModuleName                  doscalls
DosQueryProcAddr                    doscalls
DosFreeModule                       doscalls
__std_exit                          libcn0
__std_calloc                        libcn0
__std_free                          libcn0
_pthread_atfork                     pthr01
_pthread_rwlock_init                pthr01
_pthread_rwlock_rdlock              pthr01
_pthread_rwlock_wrlock              pthr01
_pthread_rwlock_unlock              pthr01
_pthread_rwlock_destroy             pthr01
_pthread_once                       pthr01
_pthread_key_delete                 pthr01
_pthread_equal                      pthr01
__std_strlen                        libcn0
__std_strcpy                        libcn0
__std_realloc                       libcn0
__std_memset                        libcn0
__std_vsnprintf                     libcn0
__std_open                          libcn0
__std_write                         libcn0
___libc_FH                          libcn0
__libsocket_setsockopt              tcpip32
__libsocket_set_errno               tcpip32
__libsocket_sock_errno              tcpip32
_os2_sock_errno                     tcpip32
__std_longjmp                       libcn0
__std_environ                       libcn0
__std_fork                          libcn0
__std_dup2                          libcn0
__std_signal                        libcn0
__std_execve                        libcn0
__std_sleep                         libcn0
__libsocket_bind                    tcpip32
__libsocket_getsockname             tcpip32
__std_memcmp                        libcn0
__std_setjmp                        libcn0
__libsocket_getpeername             tcpip32
__libsocket_send                    tcpip32
__libsocket_recv                    tcpip32
__std_ioctl                         libcn0
__std_memmove                       libcn0
__libsocket_shutdown                tcpip32
__std_strchr                        libcn0
__std_strcmp                        libcn0
__std_fcntl                         libcn0
__std_close                         libcn0
__std_time                          libcn0
__std_sprintf                       libcn0
__std_ctime_r                       libcn0
__std_strstr                        libcn0
__std_writev                        libcn0
__getprogname                       libcn0
__std_getpid                        libcn0
__std_strerror                      libcn0
__std_localtime_r                   libcn0
__std_snprintf                      libcn0
__std_abort                         libcn0
__std_fputs                         libcn0
__std_fflush                        libcn0
__std_stricmp                       libcn0
__std_opendir                       libcn0
__std_malloc                        libcn0
__std_readdir                       libcn0
__std_closedir                      libcn0
__std_qsort                         libcn0
__std_strtol                        libcn0
__std_stat                          libcn0
__std_strtok                        libcn0
__std_getgrnam                      libcn0
__std_strrchr                       libcn0
_stpcpy                             libcn0
__std_realpath                      libcn0
__libsocket_socket                  tcpip32
___libc_TcpipAllocFH44              libcn0
__libsocket_soclose                 tcpip32
__libsocket_getsockopt              tcpip32
__std_strnicmp                      libcn0
__libsocket_connect                 tcpip32
__libsocket_listen                  tcpip32
_fread                              libcx0
__libsocket_sendto                  tcpip32
__std_bsearch                       libcn0
__std_getrlimit                     libcn0
__libsocket_accept                  tcpip32
__libsocket_socketpair              tcpip32
___libc_FHClose                     libcn0
__std_lchown                        libcn0
__std_lstat                         libcn0
__std_unlink                        libcn0
__std_strcat                        libcn0
__std_chroot                        libcn0
__std_chdir                         libcn0
__std_fprintf                       libcn0
___stdinp                           libcn0
__std_memcpy                        libcn0
_mmap                               libcx0
_mprotect                           libcx0
_munmap                             libcx0
__std_strncmp                       libcn0
DosTIB                              doscalls
DosSetExceptionHandler              doscalls
DosUnsetExceptionHandler            doscalls
__lmalloc                           libcn0
_gethostbyname                      tcpip32
__std_fileno                        libcn0
__std_fstat                         libcn0
__std_setbuf                        libcn0
__std_ferror                        libcn0
__std_fclose                        libcn0
__std_clearerr                      libcn0
__std_fdopen                        libcn0
__std_chmod                         libcn0
__std_fwrite                        libcn0
__std_strdup                        libcn0
__std_atexit                        libcn0
__std_strncpy                       libcn0
__std_fgets                         libcn0
__std_fseek                         libcn0
__std_ftell                         libcn0
__std_feof                          libcn0
__std_atoi                          libcn0
__std_memchr                        libcn0
__std_strtoul                       libcn0
__std_sscanf                        libcn0
___ctordtorInit1                    libcn0
___ctordtorTerm1                    libcn0
__std_strspn                        libcn0
__std_strcspn                       libcn0
__std_sigaction                     libcn0
__std_tcsetattr                     libcn0
__std_fputc                         libcn0
__std_fopen                         libcn0
__std_tcgetattr                     libcn0
__std_random                        libcn0
__std_usleep                        libcn0
__std_gettimeofday                  libcn0
__std_sysconf                       libcn0
__std_getenv                        libcn0
__std_vfprintf                      libcn0
_gai_strerror                       libcx0
__std_gmtime_r                      libcn0
__std_getuid                        libcn0
__std_geteuid                       libcn0
__std_getgid                        libcn0
__std_getegid                       libcn0
DosRequestMutexSem                  doscalls
DosQueryMutexSem                    doscalls
__assert                            libcn0
___libc_GpFIBLIS                    libcn0
___fmutex_request_internal          libcn0
DosCreateMutexSem                   doscalls
DosReleaseMutexSem                  doscalls
___fmutex_release_internal_must_complete libcn0
___fmutex_request_internal_must_complete libcn0
___fmutex_release_internal          libcn0
DosCloseEventSem                    doscalls
DosWaitEventSem                     doscalls
DosPostEventSem                     doscalls
DosCloseMutexSem                    doscalls
DosCreateEventSem                   doscalls
DosResetEventSem                    doscalls
__beginthread                       libcx0
__gettid                            libcn0
DosSleep                            doscalls


                        +--------------------+
                        |   Libraries Used   |
                        +--------------------+

U:\tmp\ldconv_libssl_a_99560c9c37e1aece0.lib
U:\tmp\ldconv_libcrypto_a_99560c9c37f156ab8.lib
U:\extras\lib\pthreads.lib
U:\extras\lib\libcx.lib
U:\tmp\ldconv_ssp_a_99560c9c38216f540.lib
U:\tmp\ldconv_libgcc_eh_a_99560c9c382174360.lib
U:\tmp\ldconv_libgcc_a_99560c9c382191438.lib
U:\usr\lib\libc_alias.lib
U:\usr\lib\libc_dll.lib
U:\usr\lib\libos2.lib
U:\usr\lib\libend.lib


                        +-----------------------+
                        |   Linker Statistics   |
                        +-----------------------+

Stack size:  007d0000 (8192000.)
Memory size:  00a469f0 (10775024.)
Entry point address: 0001:00000000
Link time: 00:00.65
